:0200000490006A
:100000006825002001C40590DD220590DF220590BF
:10001000E1220590E3220590E52205900000000012
:10002000000000000000000000000000B972009015
:10003000E7220590000000005D720090E922059023
:1000400029E205902DE2059031E2059035E2059018
:1000500039E205903DE2059041E2059045E20590C8
:1000600049E205904DE2059051E2059055E2059078
:1000700059E205905DE2059061E2059065E2059028
:1000800069E205906DE2059071E2059075E20590D8
:1000900079E205907DE2059081E2059085E2059088
:1000A00089E205908DE2059091E2059095E2059038
:1000B00099E205909DE20590A1E20590A5E20590E8
:1000C000A9E20590ADE20590B1E20590B5E2059098
:1000D000B9E20590BDE20590C1E20590C5E2059048
:1000E000F3220590C9E20590CDE20590D1E205909A
:1000F000D5E20590D9E20590DDE20590E1E20590B8
:10010000E5E20590E9E20590EDE20590F1E2059067
:10011000F5E20590F9E20590C5D60290FDE2059062
:1001200001E3059005E3059009E305900DE30590D3
:10013000FB2205900000000000000000000000000D
:1001400000000000000000000000000011E3059026
:1001500015E305900323059019E305901DE3059031
:1001600021E3059025E3059029E305902DE3059013
:1001700031E30590ED2205900000000035E3059085
:1001800039E305903DE3059041E3059045E3059093
:1001900049E305904DE305900000000051E3059010
:1001A00000000000000000000000000055E3059082
:1001B00059E305905DE30590000000000000000099
:1001C000000000000000000000000000000000002F
:1001D00000000000000000000000000061E3059046
:1001E000000000000000000000000000000000000F
:1001F00000000000000000000000000000000000FF
:1002000000000000000000000000000000000000EE
:1002100000000000000000000000000000000000DE
:10022000000000000000000000000000000003804B
:10023000000380000380000380000380000380002F
:100240000380000380000380000100000100000023
:100250000000000000038000038000000000000098
:10026000000000000000000000000000000000008E
:100270000000000000000000000E70000E70000E74
:10028000700004200004200004200004200000006E
:10029000000000000000000000000000000000005E
:1002A000000000000000000000000000000000004E
:1002B00000000000000000000000000000000660D8
:1002C000000660000660000660000660003FF8005F
:1002D0003FF8000660000CC0003FF8003FF8000C3B
:1002E000C0000CC0000CC0000CC0000CC00000001E
:1002F00000000000000000000000000000000000FE
:1003000000000001800001800007B0000FF000181D
:1003100070001870001C00000F800007E00000F063
:10032000001830001C30001C70001FE0001BC000D3
:1003300001800001800001800001800000000000B9
:100340000000000000000000000000000000078026
:10035000000FC0001CE0001860001860001CE000E6
:100360000FF80007E0001FF000073800061800062D
:10037000180007380003F00001E000000000000052
:10038000000000000000000000000000000000006D
:1003900000000000000000000000000003F0000763
:1003A000F0000C60000C00000C00000600000700CC
:1003B000000F9C001DFC0018F0001870000FFC00DE
:1003C00007DC00000000000000000000000000004A
:1003D000000000000000000000000000000000001D
:1003E0000003800003800003800001000001000082
:1003F00001000001000000000000000000000000FB
:1004000000000000000000000000000000000000EC
:1004100000000000000000000000000000000000DC
:10042000000000000000001800003800007000000C
:10043000F00000E00000E00001C00001C00001C0C9
:100440000001C00001C00001C00000E00000E000A9
:10045000007000007000003800001800000000006C
:100460000000000000000000000000000000180074
:10047000001C00000E00000E000007000007000036
:1004800003800003800003800003800003800003DA
:1004900080000700000700000F00000E00001C0095
:1004A0000018000000000000000000000000000034
:1004B0000000000000000180000180000180001D9C
:1004C000B8001FF80007E00003C00003C00006608A
:1004D00000066000000000000000000000000000B6
:1004E000000000000000000000000000000000000C
:1004F00000000000000000000000000000000000FC
:1005000000000000018000018000018000018000E7
:100510000180003FFC003FFC0001800001800001E1
:100520008000018000018000000000000000000049
:1005300000000000000000000000000000000000BB
:1005400000000000000000000000000000000000AB
:10055000000000000000000000000000000000009B
:100560000000000000000000000000E00000C000EB
:1005700001C00001800001800003000003000000B2
:10058000000000000000000000000000000000006B
:10059000000000000000000000000000000000005B
:1005A0000000001FF8001FF800000000000000001D
:1005B000000000000000000000000000000000003B
:1005C000000000000000000000000000000000002B
:1005D000000000000000000000000000000000001B
:1005E000000000000000000000000000000000000B
:1005F0000000000000000000000003C00003C00075
:1006000003C0000000000000000000000000000027
:100610000000000000000000001800001800003872
:100620000000300000700000600000600000C000AA
:1006300000C00001800001800003000003000006EC
:1006400000000600000E00000C00001C0000180056
:100650000018000000000000000000000000000082
:1006600000000000000003C00007E0000C30000C98
:10067000300018180018180018180018180018185A
:10068000001818001818000C30000C300007E000AB
:1006900003C0000000000000000000000000000097
:1006A00000000000000000000000000000000080CA
:1006B000000780001F80001D800001800001800075
:1006C00001800001800001800001800001800001A4
:1006D00080000180001FF8001FF8000000000000EB
:1006E000000000000000000000000000000000000A
:1006F00000000000000007C0001FF000383000308C
:10070000180030180000180000300000600001C020
:10071000000380000600000C00001800003FF800F5
:100720003FF8000000000000000000000000000092
:10073000000000000000000000000000000003C0F6
:10074000000FE0000C70000030000030000060007E
:1007500003C00003E0000070000018000018000053
:1007600018001838001FF0000FC000000000000043
:100770000000000000000000000000000000000079
:1007800000000000000000E00001E00001E00003C4
:1007900060000660000660000C60000C60001860DD
:1007A000003060003FF8003FF80000600003F800F0
:1007B00003F800000000000000000000000000003E
:1007C00000000000000000000000000000001FF01A
:1007D000001FF0001800001800001800001BC000E7
:1007E0001FF0001C30000018000018000018000066
:1007F00018003030003FF0000FC000000000000083
:1008000000000000000000000000000000000000E8
:1008100000000000000000F80003F8000700000ED0
:1008200000000C00001800001BC0001FF0001C306E
:10083000001818001818001818000C38000FF000E5
:1008400003E00000000000000000000000000000C5
:1008500000000000000000000000000000001FF881
:10086000001FF80018180018380000300000300091
:1008700000700000600000600000E00000C00000A8
:10088000C00001C0000180000180000000000000E5
:100890000000000000000000000000000000000058
:1008A00000000000000007E0000FF0001C380018F6
:1008B00018001818000C300007E00007E0000C30AA
:1008C000001818001818001818001C38000FF00045
:1008D00007E0000000000000000000000000000031
:1008E000000000000000000000000000000007C041
:1008F000000FF0001C30001818001818001818001D
:100900000C38000FF80003D8000018000030000079
:10091000700000E0001FC0001F0000000000000089
:1009200000000000000000000000000000000000C7
:1009300000000000000000000000000000000000B7
:10094000000003C00003C00003C00000000000005E
:100950000000000000000000000003C00003C00011
:1009600003C00000000000000000000000000000C4
:100970000000000000000000000000000000000077
:100980000000000000000000000000F00000F00087
:1009900000F0000000000000000000000000000067
:1009A000E00001C00001800001800003000002009F
:1009B0000000000000000000000000000000000037
:1009C000000000000000000000000000001C00000B
:1009D0003C0000F00003C0000F00003C0000F000ED
:1009E000003C00000F000003C00000F000003C00CD
:1009F000001C0000000000000000000000000000DB
:100A000000000000000000000000000000000000E6
:100A1000000000000000000000000000007FFC005B
:100A20007FFC000000000000007FFC007FFC000055
:100A300000000000000000000000000000000000B6
:100A400000000000000000000000000000000000A6
:100A500000000000000000000000000070000078AE
:100A600000001E000007800001E000007800001E6A
:100A70000000780001E0000780001E000078000000
:100A800070000000000000000000000000000000F6
:100A90000000000000000000000000000000000056
:100AA0000007C0000FE00018700018300018300078
:100AB00000700000E00003C000038000030000009D
:100AC0000000000000070000070000000000000018
:100AD0000000000000000000000000000000000016
:100AE00000000000000003E00007F0000E38000CDA
:100AF000180018780018F80019D8001998001998EB
:100B00000019980018F8001878001800000C000070
:100B10000E180007F80003E00000000000000000CD
:100B200000000000000000000000000000000000C5
:100B3000001F80001FC00001C000036000036000B0
:100B40000630000630000C30000FF8001FF80018C7
:100B50000C00300C00FC7F00FC7F00000000000057
:100B60000000000000000000000000000000000085
:100B70000000000000000000007FE0007FF000188F
:100B800038001818001818001838001FF0001FF857
:100B900000181C00180C00180C00180C007FF8003E
:100BA0007FF00000000000000000000000000000D6
:100BB0000000000000000000000000000000000035
:100BC0000003EC000FFC001C1C00180C00300C0093
:100BD000300000300000300000300000300000180D
:100BE0000C001C1C000FF80003F0000000000000C7
:100BF00000000000000000000000000000000000F5
:100C00000000000000000000007FC0007FF000181E
:100C10003800181800180C00180C00180C00180CDC
:100C200000180C00180C001818001838007FF0008D
:100C30007FE0000000000000000000000000000055
:100C400000000000000000000000000000000000A4
:100C5000007FF8007FF80018180018180019980095
:100C60001980001F80001F8000198000199800184B
:100C700018001818007FF8007FF80000000000003E
:100C80000000000000000000000000000000000064
:100C90000000000000000000003FFC003FFC000CD2
:100CA0000C000C0C000CCC000CC0000FC0000FC0DE
:100CB000000CC0000CC0000C00000C00003FC00085
:100CC0003FC0000000000000000000000000000025
:100CD0000000000000000000000000000000000014
:100CE0000003EC000FFC001C1C00180C00300C0072
:100CF00030000030000030FE0030FE00300C0038C4
:100D00000C001C1C000FFC0003F0000000000000A1
:100D100000000000000000000000000000000000D3
:100D20000000000000000000007E7E007E7E0018B3
:100D300018001818001818001818001FF8001FF8DD
:100D4000001818001818001818001818007E7E00E7
:100D50007E7E000000000000000000000000000097
:100D60000000000000000000000000000000000083
:100D7000001FF8001FF800018000018000018000C2
:100D800001800001800001800001800001800001DD
:100D900080000180001FF8001FF800000000000024
:100DA0000000000000000000000000000000000043
:100DB00000000000000000000007FE0007FE000029
:100DC00030000030000030000030000030003030D3
:100DD000003030003030003030003060003FE00044
:100DE0000F80000000000000000000000000000074
:100DF00000000000000000000000000000000000F3
:100E0000007F3E007F3E0018300018600018C000D0
:100E10001980001B80001FC0001CE0001870001823
:100E200030001838007F1F007F1F00000000000006
:100E300000000000000000000000000000000000B2
:100E40000000000000000000007F80007F80000C98
:100E500000000C00000C00000C00000C00000C0056
:100E6000000C0C000C0C000C0C000C0C007FFC00A7
:100E70007FFC0000000000000000000000000000F7
:100E80000000000000000000000000000000000062
:100E900000F00F00F81F00381C003C3C003C3C00F8
:100EA000366C00366C0033CC0033CC00318C003013
:100EB0000C00300C00FE7F00FE7F000000000000F0
:100EC0000000000000000000000000000000000022
:100ED00000000000000000000078FE0078FE001C0A
:100EE00018001E18001F18001B18001B980019D8A6
:100EF0000018D80018F8001878001838007F18007B
:100F00007F1800000000000000000000000000004A
:100F100000000000000000000000000000000000D1
:100F20000003C0000FF0001C3800181800381C0027
:100F3000300C00300C00300C00300C00381C001855
:100F400018001C38000FF00003C000000000000073
:100F50000000000000000000000000000000000091
:100F60000000000000000000003FF0003FF8000C0F
:100F70001C000C0C000C0C000C0C000C18000FF8E2
:100F8000000FE0000C00000C00000C00003FC0004F
:100F90003FC0000000000000000000000000000052
:100FA0000000000000000000000000000000000041
:100FB0000003C0000FF0001C3800181800381C0097
:100FC000300C00300C00300C00300C00381C0018C5
:100FD00018001C38000FF00007C00007CC000FFC01
:100FE000000C3800000000000000000000000000BD
:100FF0000000000000000000007FE0007FF000180B
:1010000038001818001818001838001FF0001FC00A
:101010000018E0001870001830001838007F1E001B
:101020007F0E000000000000000000000000000033
:1010300000000000000000000000000000000000B0
:101040000007D8000FF8001C380018180018180006
:101050001E00000FC00003F00000780018180018F0
:1010600018001C38001FF0001BE00000000000000A
:101070000000000000000000000000000000000070
:101080000000000000000000003FFC003FFC0031B9
:101090008C00318C00318C00318C0001800001808B
:1010A000000180000180000180000180000FF0003D
:1010B0000FF0000000000000000000000000000031
:1010C0000000000000000000000000000000000020
:1010D000007E7E007E7E0018180018180018180088
:1010E00018180018180018180018180018180018F8
:1010F00018000C30000FF00003C0000000000000DA
:1011000000000000000000000000000000000000DF
:101110000000000000000000007F7F007F7F0018BB
:101120000C000C18000C18000C18000630000630DB
:101130000003600003600003600001C00001C00004
:10114000008000000000000000000000000000001F
:10115000000000000000000000000000000000008F
:1011600000FE3F80FE3F80300600300600308600E3
:1011700019CC0019CC001B6C001B6C001E7C000EEF
:1011800038000E38000C18000C1800000000000099
:10119000000000000000000000000000000000004F
:1011A0000000000000000000007E7E007E7E00182F
:1011B00018000C300006600003C0000180000180B0
:1011C0000003C0000660000C30001818007E7E008E
:1011D0007E7E000000000000000000000000000013
:1011E00000000000000000000000000000000000FF
:1011F000007C7E007C7E001818000C300006600029
:1012000006600003C0000180000180000180000131
:1012100080000180000FF0000FF0000000000000CF
:1012200000000000000000000000000000000000BE
:101230000000000000000000001FF8001FF8001868
:10124000180018300018600018C00001800003006A
:10125000000618000C18001818003018003FF8009D
:101260003FF8000000000000000000000000000047
:10127000000000000000000000000000000001F07D
:101280000001F00001800001800001800001800069
:1012900001800001800001800001800001800001C8
:1012A000800001800001800001800001800001F0C9
:1012B0000001F0000000000000000000000000003D
:1012C0001800001800001C00000C00000E000006B2
:1012D0000000060000030000030000018000018000
:1012E0000000C00000C0000060000060000070004E
:1012F0000030000038000018000018000000000056
:1013000000000000000000000000000000000F804E
:10131000000F80000180000180000180000180003A
:101320000180000180000180000180000180000137
:1013300080000180000180000180000180000F809A
:10134000000F80000000000000000000000000000E
:1013500000000000800001C00003E00007700006EC
:1013600030000C1800180C001004000000000000F1
:10137000000000000000000000000000000000006D
:10138000000000000000000000000000000000005D
:10139000000000000000000000000000000000004D
:1013A000000000000000000000000000000000003D
:1013B000000000000000000000000000000000002D
:1013C000000000000000000000000000000000001D
:1013D00000000000000000000000FFFF00FFFF0011
:1013E00000000003000003800000E0000060000037
:1013F00000000000000000000000000000000000ED
:1014000000000000000000000000000000000000DC
:1014100000000000000000000000000000000000CC
:1014200000000000000000000000000000000000BC
:10143000000000000000000000000FC0001FE000DE
:1014400000300000300007F0001FF000383000309E
:1014500030003070001FFC000FBC000000000000D6
:10146000000000000000000000000000000000007C
:10147000000000000000780000780000180000184C
:1014800000001BE0001FF8001C1800180C00180CCE
:1014900000180C00180C00180C001C18007FF80035
:1014A0007BE00000000000000000000000000000E1
:1014B000000000000000000000000000000000002C
:1014C0000000000000000000000003EC000FFC0022
:1014D0001C1C00380C00300C0030000030000038BC
:1014E0000C001C1C000FF80003F0000000000000BE
:1014F00000000000000000000000000000000000EC
:1015000000000000000000780000780000180000D3
:10151000180007D8001FF8001838003018003018DD
:10152000003018003018003018001838001FFE0076
:1015300007DE0000000000000000000000000000C6
:10154000000000000000000000000000000000009B
:101550000000000000000000000007E0001FF8008D
:10156000181800300C003FFC003FFC003000003039
:101570000000180C001FFC0007F000000000000035
:10158000000000000000000000000000000000005B
:1015900000000000000001FC0003FC000600000643
:1015A00000003FF8003FF8000600000600000600BB
:1015B000000600000600000600000600003FF000E4
:1015C0003FF00000000000000000000000000000EC
:1015D000000000000000000000000000000000000B
:1015E0000000000000000000000007DE001FFE00F9
:1015F000183800301800301800301800301800304B
:1016000018001838001FF80007D80000180000184C
:10161000000038000FF0000FC000000000000000C4
:10162000000000000000780000780000180000189A
:1016300000001BE0001FF0001C38001818001818EC
:10164000001818001818001818001818007E7E00DE
:101650007E7E00000000000000000000000000008E
:1016600000000000000000000000000000000180F9
:10167000000180000000000000001F80001F8000AB
:1016800001800001800001800001800001800001D4
:1016900080000180003FFC003FFC000000000000D3
:1016A000000000000000000000000000000000003A
:1016B00000000000000000C00000C00000000000AA
:1016C00000001FF0001FF00000300000300000306C
:1016D000000030000030000030000030000030001A
:1016E0000030000030000030000070001FE0001FDC
:1016F00080000000000000000000000000003C002E
:10170000003C00000C00000C00000CF8000CF8007D
:101710000CC0000D80000F80000F00000F80000D36
:10172000C0000CE0003C7C003C7C0000000000009D
:1017300000000000000000000000000000000000A9
:101740000000000000001F80001F800001800001D9
:101750008000018000018000018000018000018084
:10176000000180000180000180000180003FFC003A
:101770003FFC00000000000000000000000000002E
:101780000000000000000000000000000000000059
:1017900000000000000000000000F77800FFFC00DF
:1017A00039CC00318C00318C00318C00318C00310F
:1017B0008C00318C00FDEF00FDEF00000000000008
:1017C0000000000000000000000000000000000019
:1017D0000000000000000000000000000000000009
:1017E00000007BE0007FF0001C380018180018187B
:1017F000001818001818001818001818007E7E002D
:101800007E7E0000000000000000000000000000DC
:1018100000000000000000000000000000000000C8
:101820000000000000000000000003C0000FF000F6
:101830001C3800381C00300C00300C00300C003814
:101840001C001C38000FF00003C000000000000066
:101850000000000000000000000000000000000088
:101860000000000000000000000000000000000078
:1018700000007BE0007FF8001C1800180C00180C1A
:1018800000180C00180C00180C001C18001FF800A1
:101890001BE0001800001800001800007F00007F07
:1018A0000000000000000000000000000000000038
:1018B0000000000000000000000007DE001FFE0026
:1018C0001838003018003018003018003018003078
:1018D00018001838001FF80007D80000180000187A
:1018E0000000180000FE0000FE00000000000000E4
:1018F00000000000000000000000000000000000E8
:1019000000003E78003EFC0007CC00070000060007
:10191000000600000600000600000600003FF00080
:101920003FF0000000000000000000000000000088
:1019300000000000000000000000000000000000A7
:101940000000000000000000000007F8000FF80091
:101950001818001818001F80000FF00000F8001879
:1019600018001838001FF0001FE000000000000001
:101970000000000000000000000000000000000067
:101980000000000000000C00000C00000C00000C27
:1019900000003FF0003FF0000C00000C00000C00C5
:1019A000000C00000C00000C00000C1C0007FC00E8
:1019B00003F0000000000000000000000000000034
:1019C0000000000000000000000000000000000017
:1019D0000000000000000000000078780078780027
:1019E00018180018180018180018180018180018EF
:1019F00018001838000FFE0007DE0000000000008D
:101A000000000000000000000000000000000000D6
:101A100000000000000000000000000000000000C6
:101A200000007C3E007C3E001818001818000C30A6
:101A3000000C300006600006600007E00003C000F4
:101A400003C00000000000000000000000000000D3
:101A50000000000000000000000000000000000086
:101A600000000000000000000000783C00783C000E
:101A70003118003398003398001AB0001EF0001E91
:101A8000F0001C60000C60000C6000000000000012
:101A90000000000000000000000000000000000046
:101AA0000000000000000000000000000000000036
:101AB00000003E7C003E7C000C300006600003C04D
:101AC0000001800003C0000660000C30003E7C0076
:101AD0003E7C00000000000000000000000000004C
:101AE00000000000000000000000000000000000F6
:101AF000000000000000000000007E1F007E1F00AC
:101B0000180C000C18000C180006300006300003FA
:101B1000600003E00001C00000C0000180000180FF
:101B2000000300003FC0003FC000000000000000B4
:101B300000000000000000000000000000000000A5
:101B400000001FF8001FF80018300018600000C0E7
:101B5000000180000300000618000C18001FF800A8
:101B60001FF800000000000000000000000000005E
:101B7000000000000000000000000000000000E085
:101B80000001E00001800001800001800001800070
:101B90000180000180000380000700000380000135
:101BA000800001800001800001800001800001E0D0
:101BB0000000E00000000000000000000000000045
:101BC0000000000000000180000180000180000191
:101BD0008000018000018000018000018000018000
:101BE0000001800001800001800001800001800070
:101BF00001800001800001800001800000000000E1
:101C000000000000000000000000000000000700CD
:101C10000007800001800001800001800001800039
:101C200001800001800001C00000E00001C000014F
:101C30008000018000018000018000018000078099
:101C4000000700000000000000000000000000008D
:101C50000000000000000000000000000000000084
:101C600000000000000000000E00001F18003BB83C
:101C70000031F00000E00000000000000000000063
:101C80000000000000000000000000000000000054
:101C90000000000000000000000000000000000044
:101CA0000000000000000000000000000000000034
:101CB0000000000000000000000000000000000024
:101CC00000000700070007000700070007000700E3
:101CD00002000200000000000700070000000000F2
:101CE0000000000000000000000000001CE01CE0FC
:101CF0001CE0084008400840000000000000000010
:101D000000000000000000000000000000000000D3
:101D10000CC00CC00CC00CC00CC03FF03FF00CC09D
:101D20000CC03FF03FF00CC00CC00CC00CC00CC08D
:101D300000000000000000000300030007E00FE0C7
:101D4000186018001F000FC000E0186018601FC066
:101D50001F800300030003000000000000000000DB
:101D600000001C002200220022001C6001E00F8005
:101D70003C0031C002200220022001C0000000000F
:101D8000000000000000000000000000000003E070
:101D90000FE00C000C0006000F301FF019E018C017
:101DA0001FF007B00000000000000000000000006D
:101DB0000000000003800380038001000100010097
:101DC0000000000000000000000000000000000013
:101DD0000000000000000000000000C000C0018002
:101DE00001800180030003000300030003000300DF
:101DF00001800180018000C000C0000000000000E0
:101E000000000C000C0006000600060003000300A2
:101E100003000300030003000600060006000C0098
:101E20000C0000000000000000000300030003009D
:101E30001B601FE0078007800FC00CC0000000007F
:101E40000000000000000000000000000000000092
:101E500000000000000003000300030003003FF047
:101E60003FF0030003000300030000000000000037
:101E70000000000000000000000000000000000062
:101E800000000000000000000000000000000380CF
:101E9000030003000600060004000000000000002C
:101EA00000000000000000000000000000003FE013
:101EB0003FE0000000000000000000000000000003
:101EC0000000000000000000000000000000000012
:101ED000000000000000000000000000000003807F
:101EE00003800380000000000000000000000000EC
:101EF0000060006000C000C000C0018001800300DD
:101F00000300060006000C000C000C00180018006E
:101F1000000000000000000000000F801FC018C07B
:101F2000306030603060306030603060306018C0E9
:101F30001FC00F8000000000000000000000000033
:101F4000000003001F001F00030003000300030044
:101F500003000300030003001FE01FE00000000077
:101F6000000000000000000000000F801FC038E0EB
:101F70003060006000C00180030006000C00180003
:101F80003FE03FE000000000000000000000000013
:101F900000000F803FC030E0006000E007C007C0D5
:101FA00000E00060006060E07FC03F800000000053
:101FB0000000000000000000000001C003C003C0DA
:101FC00006C00CC00CC018C030C03FE03FE000C0ED
:101FD00003E003E00000000000000000000000003B
:101FE00000001FC01FC0180018001F801FC018E08D
:101FF00000600060006030E03FC01F800000000013
:102000000000000000000000000003E00FE01E00E0
:102010001800380037803FC038E03060306018E08A
:102020001FC007800000000000000000000000004A
:1020300000003FE03FE03060006000C000C000C032
:102040000180018001800300030003000000000004
:10205000000000000000000000000F801FC038E0FA
:10206000306038E01FC01FC038E03060306038E0BA
:102070001FC00F80000000000000000000000000F2
:1020800000000F001FC038C03060306038E01FE033
:102090000F6000E000C003C03F803E000000000071
:1020A0000000000000000000000000000000000030
:1020B0000000038003800380000000000000038014
:1020C000038003800000000000000000000000000A
:1020D0000000000000000000000001C001C001C0BD
:1020E000000000000000038003000600060004005A
:1020F00000000000000000000000000000000030B0
:1021000000F003C007001C0078001C00070003C09B
:1021100000F000300000000000000000000000009F
:10212000000000000000000000007FF07FF00000D1
:1021300000007FF07FF000000000000000000000C1
:10214000000000000000000000000000000030005F
:102150003C000F00038000E0007800E003800F00E7
:102160003C00300000000000000000000000000003
:10217000000000000F801FC018601860006001C0E0
:1021800003800300000000000700070000000000BB
:102190000000000000000000000003800C800840E8
:1021A0001040104011C012401240124011C01000E7
:1021B0000800084007800000000000000000000048
:1021C000000000001F801F80038006C006C00CC0F6
:1021D0000C601FE01FE03030787878780000000055
:1021E0000000000000000000000000003F803FC031
:1021F0001860186018E01FC01FE018701830183001
:102200003FF03FE000000000000000000000000080
:102210000000000007B00FF01C70383030003000B4
:102220003000300038301C700FE007C000000000A4
:102230000000000000000000000000007F807FC060
:1022400030E030703030303030303030307030E0AE
:102250007FC07F8000000000000000000000000040
:10226000000000003FF03FF01830183019801F8048
:102270001F801980183018303FF03FF00000000038
:102280000000000000000000000000003FF03FF0F0
:102290001830183019801F801F801980180018000E
:1022A0003F003F00000000000000000000000000B0
:1022B0000000000007B01FF0187030303000300010
:1022C00031F831F8303018301FF007C0000000003E
:1022D0000000000000000000000000003CF03CF0A6
:1022E0001860186018601FE01FE018601860186020
:1022F0003CF03CF000000000000000000000000086
:10230000000000001FE01FE00300030003000300C3
:1023100003000300030003001FE01FE000000000B3
:1023200000000000000000000000000003F803F8B7
:10233000006000600060006030603060306030E05D
:102340003FC00F80000000000000000000000000FF
:10235000000000003EF83EF818E019801B001F0046
:102360001D8018C018C018603E783E38000000007C
:102370000000000000000000000000003F003F00DF
:102380000C000C000C000C000C000C300C300C305D
:102390003FF03FF0000000000000000000000000DF
:1023A000000000007878787838703CF034B037B0AE
:1023B00037B03330333030307CF87CF80000000028
:1023C00000000000000000000000000039F03DF0B7
:1023D0001C601E601E601B601B6019E019E018E0A5
:1023E0003EE03E6000000000000000000000000031
:1023F0000000000007800FC01CE038703030303023
:102400003030303038701CE00FC007800000000012
:102410000000000000000000000000003FC03FE09E
:1024200018701830183018701FE01FC018001800FE
:102430003F003F000000000000000000000000001E
:102440000000000007800FC01CE0387030303030D2
:102450003030303038701CE00FC0078007B00FF00C
:102460000CE0000000000000000000003FC03FE062
:102470001870183018701FE01FC018E0186018702E
:102480003E383E1800000000000000000000000080
:10249000000000000FB01FF03870303038001F808F
:1024A00007E00070303038703FE037C000000000B7
:1024B0000000000000000000000000003FF03FF0BE
:1024C00033303330333003000300030003000300D4
:1024D0000FC00FC00000000000000000000000005E
:1024E000000000003CF03CF01860186018601860B4
:1024F0001860186018601CE00FC007800000000022
:1025000000000000000000000000000078F078F0FB
:102510003060306018C018C00D800D800D8007003D
:10252000070007000000000000000000000000009D
:10253000000000007C7C7C7C301833983398339802
:1025400036D816D01C701C701C70183000000000AB
:1025500000000000000000000000000078F078F0AB
:10256000306018C00D80070007000D8018C0306073
:1025700078F078F00000000000000000000000008B
:10258000000000003CF03CF018600CC007800780A1
:1025900003000300030003000FC00FC00000000091
:1025A0000000000000000000000000001FE01FE02D
:1025B000186018C001800300030006000C6018605A
:1025C0001FE01FE00000000000000000000000000D
:1025D000000003C003C00300030003000300030066
:1025E000030003000300030003000300030003C013
:1025F00003C0000000000000180018000C000C00D0
:102600000C0006000600030003000180018000C0EA
:1026100000C000C00060006000000000000000007A
:1026200000000F000F00030003000300030003007D
:1026300003000300030003000300030003000F0076
:102640000F000000000000000000020007000D80E5
:1026500018C03060202000000000000000000000D2
:10266000000000000000000000000000000000006A
:10267000000000000000000000000000000000005A
:10268000000000000000000000000000000000004A
:1026900000000000FFFCFFFC0000040003000080BD
:1026A000000000000000000000000000000000002A
:1026B000000000000000000000000000000000001A
:1026C000000000000000000000000FC01FE00060DC
:1026D0000FE01FE0386030E03FF01F7000000000A6
:1026E00000000000000000000000700070003000DA
:1026F000300037803FE03860303030303030386084
:102700007FE0778000000000000000000000000073
:102710000000000000000000000007B01FF01830AB
:1027200030303000300038301FF00FC000000000A3
:102730000000000000000000000000700070003089
:10274000003007B01FF01870303030303030387043
:102750001FF807B8000000000000000000000000A3
:102760000000000000000000000007801FE018606B
:102770003FF03FF0300018301FF007C000000000AD
:102780000000000000000000000003F007F0060059
:1027900006001FE01FE00600060006000600060017
:1027A0001FE01FE00000000000000000000000002B
:1027B0000000000000000000000007B81FF81870BB
:1027C00030303030303018701FF007B000300070FB
:1027D0000FE00FC0000000000000380038001800B3
:1027E00018001BC01FE01C6018601860186018609B
:1027F0003CF03CF000000000000000000000000081
:10280000000003000300000000001F001F00030081
:1028100003000300030003001FE01FE000000000AE
:1028200000000000000000000000030003000000A2
:1028300000001FC01FC000C000C000C000C000C01A
:1028400000C000C000C001C03F803F000000000089
:10285000000038003800180018001BE01BE01B00C7
:102860001E001E001B00198039F039F00000000026
:10287000000000000000000000001F001F00030017
:102880000300030003000300030003000300030030
:102890001FE01FE00000000000000000000000003A
:1028A000000000000000000000007EE07FF03330F8
:1028B00033303330333033307BB87BB80000000026
:1028C0000000000000000000000000000000000008
:1028D00000003BC03FE01C60186018601860186082
:1028E0003CF03CF000000000000000000000000090
:1028F0000000000000000000000007801FE01860DA
:1029000030303030303018601FE0078000000000A9
:1029100000000000000000000000000000000000B7
:10292000000077807FE03860303030303030386001
:102930003FE03780300030007C007C000000000069
:102940000000000000000000000007B81FF8187029
:1029500030303030303018701FF007B000300030A9
:1029600000F800F800000000000000000000000077
:1029700000003CE03DF00F300E000C000C000C009D
:102980003FC03FC000000000000000000000000049
:102990000000000000000000000007E01FE01860D9
:1029A0001E000FC001E018601FE01F800000000043
:1029B0000000000000000000000000000C000C00FF
:1029C0000C003FE03FE00C000C000C000C000C3051
:1029D0000FF007C000000000000000000000000031
:1029E0000000000000000000000038E038E018603F
:1029F00018601860186018E01FF00F7000000000E9
:102A000000000000000000000000000000000000C6
:102A1000000078F078F0306018C018C00D800D808C
:102A20000700070000000000000000000000000098
:102A30000000000000000000000078F078F0326034
:102A4000326037E01DC01DC018C018C00000000073
:102A50000000000000000000000000000000000076
:102A600000003CF03CF00CC00780030007800CC065
:102A70003CF03CF0000000000000000000000000FE
:102A80000000000000000000000078F078F03060E6
:102A900018C018C00D800F800700060006000C004B
:102AA0007F007F0000000000000000000000000028
:102AB00000001FE01FE018C00180030006000C604A
:102AC0001FE01FE000000000000000000000000008
:102AD000000001C003C00300030003000300030063
:102AE00007000E000700030003000300030003C0FB
:102AF00001C000000000000000000300030003000C
:102B000003000300030003000300030003000300AD
:102B100003000300030003000300000000000000A6
:102B200000001C001E00060006000600060006004D
:102B300007000380070006000600060006001E00CE
:102B40001C00000000000000000000000000000069
:102B5000000000000E003F3033F001E000000000F4
:102B60000000000000000000000000000000000065
:102B70000000000000000000000000000010101025
:102B80001010000010000000006C48480000000019
:102B900000000000001414287C287C2850500000FD
:102BA00000103840403848701010000000205020BD
:102BB0000C70081408000000000000182020544881
:102BC0003400000000101010100000000000000091
:102BD0000008081010101010100808000020201025
:102BE000101010101020200000107C102828000069
:102BF000000000000000101010FE10101000000077
:102C0000000000000000001810302000000000004C
:102C1000007C000000000000000000000000003008
:102C200030000000000404080810102020400000BC
:102C3000003844444444444438000000003010103C
:102C4000101010107C0000000038440408102044CC
:102C50007C000000003844041804044438000000DC
:102C6000000C141424447E040E000000003C2020BC
:102C70003804044438000000001C204078444444D8
:102C800038000000007C4404080808101000000010
:102C90000038444438444444380000000038444478
:102CA000443C040870000000000000303000003098
:102CB000300000000000001818000018302000004C
:102CC00000000C10608060100C000000000000008C
:102CD0007C007C00000000000000C02018041820C8
:102CE000C00000000000182404081000300000009C
:102CF0003844444C54544C404438000000301028B0
:102D000028287C44EE00000000F844447844444401
:102D1000F8000000003C44404040404438000000BF
:102D200000F0484444444448F000000000FC445093
:102D300070504044FC000000007E222838282020EB
:102D400070000000003C4440404E44443800000005
:102D500000EE44447C444444EE000000007C10102B
:102D6000101010107C000000003C0808084848487B
:102D70003000000000EE444850704844E600000077
:102D800000702020202024247C00000000EE6C6CC9
:102D900054544444EE00000000EE64645454544C17
:102DA000EC0000000038444444444444380000002F
:102DB0000078242424382020700000000038444487
:102DC00044444444381C000000F8444444784844D7
:102DD000E200000000344C40380404645800000055
:102DE00000FE9210101010103800000000EE444455
:102DF000444444443800000000EE4444282828108D
:102E00001000000000EE44445454545428000000C4
:102E100000C6442810102844C600000000EE4428D4
:102E20002810101038000000007C440810102044C6
:102E30007C000000003820202020202020203800A6
:102E40000040202020101008080800000038080862
:102E5000080808080808380000101028440000007E
:102E6000000000000000000000000000000000FE64
:102E70000010080000000000000000000000003802
:102E8000443C44443E00000000C040586444444474
:102E9000F80000000000003C4440404438000000BE
:102EA000000C04344C4444443E0000000000003850
:102EB000447C40403C000000001C207C202020205E
:102EC0007C000000000000364C4444443C043800C0
:102ED00000C0405864444444EE00000000100070FC
:102EE000101010107C00000000100078080808087E
:102EF0000808700000C0405C48705048DC000000CA
:102F000000301010101010107C000000000000E8CD
:102F100054545454FE000000000000D8644444445B
:102F2000EE00000000000038444444443800000033
:102F3000000000D8644444447840E00000000036BB
:102F40004C4444443C040E000000006C302020201F
:102F50007C0000000000003C44380444780000007D
:102F60000000207C202020221C000000000000CC5B
:102F70004444444C36000000000000EE444428283D
:102F800010000000000000EE4454545428000000DB
:102F9000000000CC48303048CC000000000000EEBB
:102FA00044242818101078000000007C48102044A9
:102FB0007C000000000810101010201010100800F5
:102FC0000010101010101010101000000020101031
:102FD00010100810101020000000000000245800FD
:102FE000000000004178007807E08278C17842EA6A
:102FF00001214278007842EA012140EA012070472D
:103000000170090A417070470170090A4170090A8C
:103010008170090AC17070472AB111F8013B521E34
:1030200000F8013BF9D17047521E00F8011BFBD19B
:10303000704700E0401C0278130018BF8A42F9D1A3
:103040001046704700B9704780B5006901F0E8FE8E
:1030500000B1012002BD00281CBF0C290B2904D09F
:103060000F291CBF006901F0E5BE7047F0B50022D2
:103070000023834C04EB03152E685EB10768BE4243
:1030800002BF6E688768BE4202BFAD684669B5423E
:1030900001D103E001225B1C022BEBD3022B04D1F4
:1030A00062B902290AD01220F0BD29B904EB03103D
:1030B0008089B0F5807F01D11020F0BD0020F0BDE7
:1030C000F0B5002203686E4C876804EB02152E6889
:1030D0009E4204BF6E68BE4202BFAD684669B542FB
:1030E00002D0521C022AF0D3022A10D125680022F5
:1030F000002D1EBF01222569002D0DD104EB021504
:103100002B6083686B604069A8600020A88104EB95
:103110000210838929B10BB10020F0BD4FF48071FA
:1031200000E0591C8181501CF0BD401E022810B5E2
:1031300013D2000152490A189389B3F5807F01D058
:103140001C0002D10023938103E05B1E93819BB29C
:103150000BB900220A50002010BD022010BD10B58E
:103160000021474A0B01D458844204BF0024D450A4
:10317000491C0229F6D310BDF8B505460024E878AD
:10318000F0B16E6B6878012305F13801324601F029
:1031900077FE08B1012413E0E870A86A296A301AA2
:1031A00088420DD2AF7809E0286A012305F1380181
:1031B0007F1E86196878324601F062FE022FF3D234
:1031C0002046F2BD70B504460D46606B0026854270
:1031D00010D02046FFF7D0FF06000BD16078012306
:1031E0002A4604F1380101F045FE10B14FF0FF35D9
:1031F00001266563304670BD38B50446FFF7BCFF55
:1032000005003AD12078032804BF207901282DD168
:1032100001F0E4FD04F13800FFF706FF4AF65521FE
:1032200004F23620FFF7ECFE164904F13800FFF7F0
:10323000EBFE4FF4077014492044FFF7E5FEA16947
:103240004FF408702044FFF7DFFE61694FF4097006
:103250002044FFF7D9FE606A012304F13801421CC3
:103260006078626301F00CFE00202071607800221B
:10327000002101F013FE00B10125284632BD0000F7
:103280003CEE03205252614172724161C269891E53
:10329000921E914201D3002070474289006B02FBCD
:1032A000010070472DE9F0410C46022C056849D316
:1032B000E869844246D228784FF0FF36012804D0CE
:1032C00040D303282ED01ED33CE0A86A04EB540759
:1032D00000F0C3FC002836D1C7F30800284490F85A
:1032E0003880A86A7F1C00F0B8FC60BBC7F30800F8
:1032F000284490F8380048EA0021E00754BFC1F3A1
:103300000B060E091FE0A86A00EB142100F0A7FCD1
:10331000C8B96000C0F3080028443830FFF762FEE7
:10332000064610E0A86A00EBD41100F098FC50B9F2
:10333000A000C0F3080028443830FFF756FE20F004
:10334000704600E001263046BDE8F0812DE9F041ED
:103350000F46022F044615464FF0020865D3E06978
:10336000874262D22078012804D05ED3032841D05E
:103370002FD35AE0A06A07EB570600F045FC5FEA3E
:10338000000852D1C6F3080020443830761CF907F3
:1033900043BF017801F00F0141EA05112946017090
:1033A0000120E070A06A00F02FFC5FEA00083CD129
:1033B000C6F3080020443830F90748BF290906D46D
:1033C00001782A0A02F00F0201F0F00111430170A6
:1033D00029E0A06A00EB172100F018FC5FEA000862
:1033E00023D17800C0F308002044A9B23830FFF799
:1033F00007FE18E0A06A00EBD71100F007FC5FEAB7
:10340000000812D1B800C0F30800271807F13800EF
:10341000FFF7EBFD25F0704100F07040014307F12C
:103420003800FFF7F1FD0120E0704046BDE8F08173
:10343000F8B504460F46022F1146256811D3E869F6
:1034400087420ED231B14FF0FF322846FFF77EFFA0
:10345000010023D1394600F03FF906001DD0012EAE
:1034600001D10220F2BD16F1010F01D10120F2BD00
:10347000002239462846FFF769FF01000ED1E869AE
:10348000A969821E914205D2491CA961297941F09E
:103490000101297137468742DCD30020F2BD2DE9B6
:1034A000F0410D008046D8F8004006D1676917B199
:1034B000E06987420ED301270CE0FFF7F3FE0228F4
:1034C00038BF01203DD310F1010F3AD0E1698842A5
:1034D00037D32F463E46E069761C864202D3022649
:1034E000022F26D331464046FFF7DCFED0B94FF01D
:1034F000FF3231462046FFF729FF28B92DB1324669
:1035000029462046FFF722FFA8B9E169A069666154
:10351000891E814224BF401EA061207940F0010035
:1035200020710DE0012818BF10F1010F09D0BE4233
:10353000D1D1002005E001280CBF4FF0FF36012655
:103540003046BDE8F081C26A0068490A4089121D10
:10355000B1FBF0F001E0401A0832116809B900200F
:1035600070478842F7D25168081870472DE9F0413A
:103570000D460446B5F5001F26682ED215F01F0F24
:103580002BD1A76865611FB93078032801DBF76A82
:103590002FB93189680988421FD2F06A19E0708911
:1035A0004FEA402801E0A5EB0805454539460DD313
:1035B00000F092F8074617F1010F01D1012017E042
:1035C000022F0AD3F0698742EDD306E03046FFF7B9
:1035D0005DFEE061E069A76108B9022008E000EB48
:1035E0005520E061C5F308003044383020620020E7
:1035F000BDE8F0812DE9F04104460E46606925687A
:1036000000F12007E06908B3B7F5001F1ED2F905E5
:1036100059D1A169401CE06121B929897809884202
:1036200051D311E06889401E10EA572F4BD100F0AA
:1036300053F88046B8F1020F16D318F1010F36D0B7
:10364000E869804538D31EB90020E061042041E0DC
:10365000A1692046FFF723FF5FEA000808BF0720A3
:1036600038D0B8F1010F01D1022033E018F1010F79
:103670001DD02846FFF780FDC8B901F0AFFB05F16A
:1036800038000026FFF7D0FC41462846FFF7FEFD34
:1036900002E0686B761C401C68636889864208D229
:1036A0000120E8702846FFF767FD0028F1D00120CF
:1036B00010E0686B801B6863C4F818804146284698
:1036C000FFF7E4FDE061C7F3080028443830676184
:1036D00020620020BDE8F0812046E3E570B5044695
:1036E0000D4605F11A00FFF77DFC064620780328F9
:1036F00005D105F11400FFF775FC46EA0046304697
:1037000070BD70B504460D461646B1B205F11A00FB
:10371000FFF776FC2078032805D1310C05F1140061
:10372000BDE870406CE470BD7CB5164604461D468D
:103730000B22FFF771FC062D12D3308880B136F8CA
:10374000020B102100F00102400802EB4505EA03DC
:1037500044BF85F4883585F02105491EF2D1ECE798
:10376000072005F00F023032D2B23A2AA8BFD21D8C
:103770000DF80020401E2D09F3D17E220DF8002007
:10378000002200E0521C824202D2A35C202BF9D11D
:1037900013465A1C08283ABF1DF80050401C20252B
:1037A000082AE554F4D373BD00210B220B46C9014E
:1037B00001EB530110F8013B5918521EC9B2F5D163
:1037C000084670472DE9F24F82B005462868FF276A
:1037D00004240090BB46E969002965D001F009FB8B
:1037E000040061D1286A017809B904245EE0C27A34
:1037F000E52918BF2E2902F03F02AA7159D022F004
:103800002003082B029E0CBF01230023B34250D19A
:103810000F2A50D14A0606D590F80DB001F0BF012D
:103820006A690F462A63FAB2914204BF427B93450C
:103830003FD104460098D0F80C8004F11A00FFF73D
:10384000D1FBB0BB20780D214FF0010A002620F0FB
:103850004000401E01FB00F90FF29C30805D2044C7
:10386000FFF7C0FBBAF1000F09D0B9F1FF0F3EBF5F
:10387000824628F819A009F1010904D319E04FF68E
:10388000FF71884215D1761C0D2EE5D320784006B5
:1038900005D5B9F1FF0F0CD2002028F819007F1EC2
:1038A00000F0BAF8040096D0200001D00020E861B2
:1038B000AFE0FF27F4E74FF0FF36FFB20FB12E6302
:1038C000F6E7FFF771FF8345F2D0F8E72DE9F04FF7
:1038D00083B005462868002101902846FFF746FE80
:1038E00004000FD1FF20FF2600904FF0FF30286327
:1038F000E9690198FFF766FC040003D1286A0178A2
:1039000009B9042485E0C27AE52902F03F02AA71D0
:1039100076D0130702D50F2A72D101E00F2A56D1B3
:1039200095F82F2052066FD44A0606D5427B01F047
:10393000BF010E4600926A692A63F2B2914202BF49
:103940000099427B914240D104460198D0F80C90F6
:1039500004F11A00FFF746FBB8BB20780D214FF0A9
:10396000010B002700F03F00401E01FB00F80FF2A2
:103970008820C05D2044FFF735FBBBF1000F824675
:1039800010D0B8F1FF0F20D201F0B6FA834639F813
:10399000180008F1010801F0AFFA834508BFD346CB
:1039A00004D012E04FF6FF7082450ED17F1C0D2F20
:1039B000DDD32078400606D5BBF1000F1CBF39F8D7
:1039C0001800002801D1761E1EE0FF261CE0F6B28A
:1039D00026B9009EFFF7E8FE86421AD095F82F0020
:1039E000C0070DD4286A05F124010B2210F8013B11
:1039F00011F8016B9B1B521E01D0002BF6D043B176
:103A00004FF0FF30FF26286300F006F804003FF473
:103A10006FAF2046BDE8FE8F00212846EAE52DE97C
:103A2000F04F87B005462868A021009095F82F0038
:103A3000084218BF062040F0DC80002600E0761C1B
:103A40000098C06830F816000028F8D10C2205F163
:103A5000240103A803AFFFF7DFFAF87AC00720D5E7
:103A60004020012485F82F000098234603A9C2684E
:103A700005F12400FFF758FE2846FFF727FF5FEA0D
:103A8000000802D1641C642CEED3642C08BF07200C
:103A900000F0AF80B8F1040F40F0AA80F87A85F802
:103AA0002F00F87A800706D506F10C000D21B0FB37
:103AB000F1F0461C00E001262C6800212846FFF7A3
:103AC00055FD010015D10027E96900F09FF80100BC
:103AD0000FD1296A0978E5291CBF0029002702D1E6
:103AE0007F1CB74208D001212846FFF783FD010063
:103AF000EAD0042808BF07205FEA00085DD1761EDF
:103B00005ED06869A0EB46112846FFF72FFD5FEAFB
:103B1000000852D105F124004FF6FF77FFF744FE6D
:103B20008DF8080001F064F95FEA000845D10098BB
:103B30002C6A00215FFA86F84FF0000AC0680190F5
:103B40009DF8080060730F20E0720020207304F1DC
:103B50001A00FFF755FAA8F101000D2101FB00F949
:103B600001E0BB4504D0019830F819B009F1010912
:103B70000FF28400594610F80A000AF1010A2018D1
:103B8000FFF73EFABBF1000F08BFBB46BAF10D0FBD
:103B9000E7D3BB451DBF019830F81900002848F055
:103BA000400884F8008000F035FDFFF735FF5FEA3C
:103BB000000802D1761EB5D102E05FEA080017D1F5
:103BC00001F016F95FEA000812D1286A20220021CC
:103BD000FFF72AFA286A0B2205F12401FFF71CFAE5
:103BE00095F82F00296A00F01800087300F012FD04
:103BF000404601F087B8000001030507090E1012C6
:103C00001416181C1E00000000EB56212046FFF77A
:103C1000D9BA70B50446216B2568666911F1010FA8
:103C20000CBF0020FFF7A2FC010015D1E16900F0F4
:103C300016F801000DD1226AE52111700121E97009
:103C40006169B14208D200212046FFF7D3FC010090
:103C5000ECD0042808BF022070BD00EB5721284695
:103C6000FFF7B0BA2DE9F04105460C462E6800205A
:103C7000A075E869002861D0286B10F1010F17D0FA
:103C80004FF00008002702E0E1197F1C8875F068FA
:103C900030F8180008F10108010006D0002101F0F9
:103CA0000DF908B1FF2FEFD300270020E119887527
:103CB00000230022A17D286A865C521C202E21D080
:103CC000052E08BFE526092A06D1E01809B92E27D6
:103CD00087752E275B1C4772E7187E7289B9A6F19B
:103CE00041001A280CD2286A092A007B2CBF4FF009
:103CF000100C4FF0080C10EA0C0F1CBF2036F6B267
:103D0000BE755B1C0B2AD6D331B90020E11888752B
:103D1000286A007B00B900230020E1184872286A55
:103D2000C07A2072286A1C30FFF75FF92060286A89
:103D30001630FFF75AF9E080000CA080BDE8F08152
:103D40002DE9F14F82B000680C460025D4F80080C0
:103D50000026D0F80CA00FF2B81911E0FF2D35D2D3
:103D60000121384601F0AAF807002FD0802F04DA8D
:103D700039464846FFF75DF940BB2AF815706D1CBF
:103D800018F80670761C202F0ADB2F2F18BF5C2F27
:103D9000E4D118F806002F2814BF5C28761CF8D050
:103DA000202F08EB06002060ACBF0024042400E0B4
:103DB0006D1E3DB10AEB450030F8027C202F18BF84
:103DC0002E2FF5D000202AF815000DB906205EE050
:103DD00002980B222021002624300090FFF724F9BE
:103DE00000E0761C3AF81600202818BF2E28F8D0DC
:103DF0000EB144F003040AEB450030F8020C2E2803
:103E000001D06D1EF7D14FF00009CB464FF00808E6
:103E100000E004463AF81670761C7FB1202F44F07B
:103E20000300F6D02E2F01D1AE42F2D1C34501D20C
:103E3000AE423CD1B8F10B0F2BD10446009800786C
:103E4000E52802D1009A05201070B8F1080F08BFCC
:103E50004FEA890909F00C000C2819BF09F003008A
:103E6000032844F00204E4B2A0070DD409F00300D3
:103E7000012809F00C0004BF44F01004E4B2042847
:103E800004BF44F00804E4B20098C4720020BDE806
:103E9000FE8FAE4218BF0446B54221BF2E464FF0FA
:103EA000080B4FF00B084FEA8909B3D2C6E7802F01
:103EB0000EDB0021384601F001F8070004D00FF2B4
:103EC0005C00C01910F8807C44F00204E4B22FB109
:103ED00039460FF2C800FFF7ACF820B144F00304F4
:103EE0005F27E4B20DE0A7F141001A2838BF49F07E
:103EF000020906D3A7F161001A283CBF49F0010965
:103F0000203F029858440BF1010B80F8247081E7A0
:103F1000222A3A3C3E3F7C7F000000004355454149
:103F20004141414345454549494941414592924FA7
:103F30004F4F5555594F554F9C4F9E9F41494F5597
:103F4000A5A5A6A7A8A9AAABACADAEAFB0B1B2B3B8
:103F5000B4414141B8B9BABBBCBDBEBFC0C1C2C308
:103F6000C4C54141C8C9CACBCCCDCECFD1D14545BE
:103F70004549494949D9DADBDCDD49DF4FE14F4F9B
:103F80004F4FE6E8E85555555959EEEFF0F1F2F389
:103F9000F4F5F6F7F8F9FAFBFCFDFEFF2B2C3B3DA0
:103FA0005B5D000032B50446256802E00098401CC5
:103FB0000090009800782F2818BF5C28F6D00020C9
:103FC000A06000980078202811D28020002184F879
:103FD0002F002046FFF7CAFA32BD6069C0F308001F
:103FE000284400F138012846FFF778FBA0606946B5
:103FF0002046FFF7A5FE010012D12046FFF766FC20
:1040000094F82F10020001F0040104D0042808BF26
:10401000002905D103E019B9A079C006DDD4052037
:1040200032BD10B502684FF0FF31BAB1134600E05F
:104030005B1C1C78202C01D33A2CF9D13A2C0CD1E2
:1040400012F8014B303C0A2C08D29A4208BF002CCF
:1040500004D15A1C0021026000E00021084610BD76
:1040600038B504460020E07004F134054FF0FF300D
:104070002860FFF7CBFD08B1042032BD04F23620E2
:10408000FEF7B0FF4AF65521884201D0032032BD29
:104090002879E92804D0EB2804BFA879902813D107
:1040A00004F16E00FEF7A1FF20F07F40DFF84C1511
:1040B000884207D004F18A00FEF797FFDFF8401529
:1040C000884201D1002032BD022032BD2DE9F043EB
:1040D0000D4685B0002114462960FFF7A2FF0700B6
:1040E00048BF0B2006D4DFF81C8508EB8700466824
:1040F0000EB90C2013E13046FEF7A4FF08B90F20DB
:104100000DE12E60307804F0FE0448B1707800F0C4
:1041100099FEC10704D4002C01D040070DD4FDE066
:10412000002030707770707800F095FEC10748BFAE
:10413000032003D41CB1400701D50A20EFE0002181
:104140003046FFF78DFF00270446022C23D10024C0
:1041500006EB04104FF4FB710844017919B10830E3
:10416000FEF743FF00E000204DF82400641C042CFF
:10417000EED3B9465DF8297027B139463046FFF7CE
:104180006FFF00E003200446022C04DB09F1010963
:10419000B9F1040FEED3042C08BF0120CED0022CBD
:1041A00080F27F8006F14300FEF71CFFB0F5007F30
:1041B00077D106F14E00FEF715FF050004D106F198
:1041C0005C00FEF712FF0546356206F14500C17836
:1041D0000129B17018BF022963D14D430078010055
:1041E00070815ED0411E08425BD106F14900FEF7A6
:1041F000F9FE0F210842308153D106F14B00FEF742
:10420000F1FE040004D106F15800FEF7EEFE04466C
:1042100006F14600FEF7E6FE002842D031892A1852
:1042200002EB111294423CD3A31A7489B3FBF4F34A
:10423000BBB303244FF6F67C634540F6F67C776209
:1042400038BF0224634538BF0124C0199B1CB062EB
:10425000D019032CF36130630FD106F16200FEF731
:10426000C1FE002804BF308900281AD106F164007D
:10427000FEF7BBFEF16989000CE091B1B06AF1690B
:104280002818022C0FBF490001EB410201F0010187
:1042900001EB5201F062306A01F2FF11B0EB512FD5
:1042A00001D20D203BE04FF0FF30B0617061802003
:1042B000032C307128D106F16800FEF793FE012827
:1042C00022D1791C3046FEF77DFFE8B9307106F245
:1042D0003620FEF787FE4AF65521884214D106F1B2
:1042E0003800FEF782FEC84988420DD14FF40770AE
:1042F0003044FEF77AFEC549884205D14FF4097073
:104300003044FEF772FE70613470B8F80000401C53
:10431000A8F80000F0803046FEF721FF002005B02D
:10432000BDE8F08338B505000C461CBF286800289E
:104330000AD0017841B1C188AA88914204D140785D
:1043400000F080FDC00703D500202060092032BDA9
:10435000286820602868FEF775FE08B90F2032BD76
:10436000002032BDF3B581B0144600916846FFF7D6
:1043700058FE050001D50B20FEBDA24800EB8506C6
:10438000776847B13846FEF7EAFE386900F043FD2A
:1043900078B100203870019808B9706011E0019977
:1043A00000200870019800F11001E8B200F024FD2F
:1043B00008B90220FEBD01987060019808B1012C77
:1043C00001D00020FEBD002201A902A8FFF77EFE59
:1043D000044601982146FEF73EFE2046FEBD2DE92B
:1043E000F24304008EB008BF092013D002F03F074B
:1043F0003A4669460EA8FFF769FE060040F0F180D4
:104400000098019000F076FC5FEA000803D100F00C
:1044100075FC1120EEE00098C0F80C800E9901A800
:10442000FFF7C0FD06000DD19DF83300000648BF20
:10443000062607D417F0FE0101A818BF0121FEF7D8
:1044400015FE06461C20074200F09B80300000F05D
:104450008E80042E48D16E48016800291EBF006975
:104460000028122603D101A8FFF7D9FA064630002A
:1044700047F0080737D138073BD500F01DFD05464A
:10448000099829460E30FEF7BFFD099829461630D7
:10449000FEF7BAFD09992020C872DDF82490009833
:1044A0004946FFF71BF90546009800224946FFF7E9
:1044B00028F9099800211C30FEF7A6FD00F0AAF8A3
:1044C0009DB1009800222946D0F8349001A8FEF74B
:1044D000AFFF060007D100984946FEF773FE00992A
:1044E0000646681E4861300078D1380748BF47F05B
:1044F0004007009817F0FE01406B60620998A062C7
:1045000001A818BF0121FEF7DBFD206168B3099DFA
:1045100000982946FFF7E2F8A06005F11C00FEF7BD
:1045200064FDE0600020E0620098206000F055FC2F
:10453000C0882775A080002060752062A06104F10A
:104540003000FEF771FDB80648D5E768002F45D06A
:10455000A761009840894502A068BD421FD3F905B4
:10456000E0613BD000F01FFB60BB022636E09DF807
:104570000A001121084210D178077FF57CAF082688
:104580002CE03000AFD19DF80A00C10648BF0426D8
:1045900024D4B907A9D5C007A7D507261EE0014630
:1045A000FFF79AF8022801D2022609E010F1010F64
:1045B00003D101264FF0FF3002E07F1B3100CCD049
:1045C000E0610BE000EB572201232262009804F126
:1045D0003001407800F04EFC00B10126404600F06A
:1045E0002DFC300031461CBF002020600098FEF7F3
:1045F00032FD30460FB0BDE8F08300004641540064
:104600004641543358F00320525261417272416165
:104610003CEE032000990120C87070472DE9F04757
:10462000044682B000F064F90746002804BF677DA5
:10463000002F05D000983946FEF70DFD38467BE087
:10464000207DC00703D400F028F9072074E0E0685B
:10465000A169401AA84215D8054613E0C4F820A065
:1046600000F027F988BF0F4600F130013A46404676
:10467000FEF7D2FCA069B844ED1B3818A061306881
:1046800038183060002D54D0A169C805E8D100F079
:10469000FEF811D109B9A06808E0E06A18B1204617
:1046A000FEF751FF02E0E169FFF716F8022807D391
:1046B00010F1010F39D0E061E16900F075FA18B925
:1046C00000F010F9022037E06F0A09EB000A1CD055
:1046D00000F0E7F838BFA0EB090700983B464078A8
:1046E00000F0C8FB08BB207D00060CD5206AA0EBBB
:1046F0000A00B84207D208EB40204FF4007204F1E0
:104700003001FEF789FC7F02B4E7226A5245A5D04A
:10471000207D000605D5009800F0DEF828B900F0ED
:1047200035F900F0CFF8002898D000F0E9F8012022
:1047300002E000F047F90020BDE8F6872DE9F047D8
:10474000044682B000F0D4F80746002804BF677D15
:10475000002F05D000983946FEF77DFC384694E0DE
:10476000207D800703D400F098F807208DE0A06931
:10477000291881421FD24FF0FF310D1A1BE0C4F8F7
:1047800020A000F096F888BF0F463A4641463030E8
:10479000FEF742FC207D40F080002075E168A069B2
:1047A000B84438188142A06138BF0146E1603068E2
:1047B000ED1B38183060002D5ED0A169C805E0D12E
:1047C00000F065F818D111B9A06850B906E0E06AA8
:1047D00018B12046FEF7B7FE03E0E1692046FEF778
:1047E0005EFE002848D0012813D010F1010F3FD001
:1047F000A168E06101B9A060207D000605D500F048
:1048000069F8002834D100F0C1F8E16900F0CCF972
:1048100018B900F067F8022037E06F0A09EB000AC8
:104820001BD000F03EF838BFA0EB090700983B46CC
:10483000407800F025FBD8B9206AA0EB0A00B84206
:1048400009D208EB40214FF4007204F13000FEF76A
:10485000E3FB00F09BF87F02A0E7206A50458ED072
:10486000A069E16888428AD200F02CF8002886D03E
:1048700000F046F8012008E0207D002140F04000D3
:1048800020750098FEF7E7FB0020BDE8F68700984A
:104890004089401E10EA5129704700980721FEF711
:1048A000DABB009807EB090152464089884241462D
:1048B0007047A0692F46C0F30800C0F500718D4213
:1048C0002044704700980123524604F1300140789B
:1048D00000F0D0BA0098226A012304F13001407838
:1048E00000F0CEBA0220022160750098FEF7B3BB3B
:1048F0001E4600208846306015466946204611E570
:104900000120012160750098FEF7A5BB70B582B04B
:1049100000F0B5F9050035D1207D410632D50006FD
:104920000AD5FFF7D7FF28B100980121FEF793FBC6
:10493000012076BD00F02AF800F0BEFA0646616A52
:1049400000F057FA05001DD1A56AE87A40F0200072
:10495000E872A26820682946FEF7D3FEE16805F1F7
:104960001C00FEF751FB314600F033FA002105F13F
:104970001200FEF745FB00F035FA0546207D00F0F9
:10498000BF00207500F0C1F9284676BD207D00F0FB
:104990007F002075704738B50446FFF7B7FF050064
:1049A0000ED169462046FFF7BDFC050008D12069FD
:1049B000FEF7BBFB050004BF0020206000F002F8FA
:1049C000284632BD00980021FEF745BB2DE9F84F7F
:1049D0000F4600F054F95FEA000808BF94F815800C
:1049E0005FEA080034D1E66A002E5ED017F1010FAD
:1049F0002FD1A06856F8047B4FF00209F8B10546A4
:104A00004FF0000A09F102098346014620460AF1E7
:104A1000010AFEF747FC0228C0F0998010F1010F4F
:104A20006BD00BF101018842EED04F4503D3C6F89D
:104A300000A0756008360099C9698842DFD3E06A32
:104A40004F45C0F8009032BF4FF011080020306091
:104A5000A2E0E068B84298BF0746002FA761F7D0F0
:104A60007F1E39462046FEF76EFDE06100F09BF8A0
:104A700006006CD000984089401E00EA5720861935
:104A8000A069C0051CBF226A9642E1D0207D0006C5
:104A900006D50098FFF720FF002878D1FFF776FFB2
:104AA00000F085F8002872D175E0E068B84203D2C2
:104AB000217D890758BF0746A0690021002FA16109
:104AC0004BD0009949894D0268B1401E7A1EB0FB57
:104AD000F5F1B2FBF5F28A4205D3691E8843A06165
:104AE0003F1AE1690CE0A16849B92046FEF7D7FCFE
:104AF000014601292BD011F1010F48D0A160E161DD
:104B000069B92AE0FEF7CEFB014611F1010F3ED054
:104B100002291CD30098C069814218D2E161BD42CC
:104B20000CD2A0697F1B2818A061207D8007204639
:104B3000E8D5FEF7B4FC0100E7D10027A0693818DA
:104B4000A061F80509D000F02FF8060003D1FFF7A7
:104B5000C9FE022025E000EB5726A069E1688142EA
:104B600004D2217DE06041F040012175C0051CBFE9
:104B7000226A964210D0207D000605D50098FFF7E6
:104B8000ABFE20B9FFF702FF00F011F818B1FFF7F4
:104B9000B7FE012005E0266200984146FEF75BFA69
:104BA0004046BDE8F28F01460098FEF76FBB0098C3
:104BB0000123324604F13001407800F05BB973B54F
:104BC000040001D1092076BD0022694601A8FFF743
:104BD0007DFA06003AD10098206000F08BF80500BD
:104BE00003D100F08BF8112076BD0098C5600199C3
:104BF0002046FFF7D7F9060021D194F82F000006D0
:104C000007D4A079C00617D5216A0098FEF766FD83
:104C1000A06000980021C088A0802046FEF7A6FC76
:104C200006000CD1A06848B100212046FEF748FAE2
:104C3000206120B9122602E0052600E02061284606
:104C400000F0FCF8042E08BF052601D0300001D08A
:104C50000020206000F04AF8304676BD38B500F0FC
:104C60000EF8050009D1206918B1FEF75EFA0500BB
:104C700001D100202060FFF7A5FE284632BD044682
:104C80006946FFF74FBBF8B50D46FFF7F8FF060082
:104C900028D12DB900212046FEF768FC064621E008
:104CA00000F028F8070003D100F028F81120F2BD29
:104CB00000980021C7602046FEF784FD0646042EBA
:104CC00001D030000BD129462046FEF7CBFF002152
:104CD0002046FEF78FFC0646042E08BF0026384605
:104CE00000F0ACF800F002F83046F2BD0098314612
:104CF000FEF7B1B94FF4007000F09EB80098112192
:104D0000FEF7A9B907B0BDE8F08F00982946FEF775
:104D1000A2B971B59BB0022269461BA8FFF7D6F96C
:104D20000600009801904FD1FFF7E4FF040003D183
:104D3000FFF7E4FF11204AE00098C4601B9901A826
:104D4000FFF730F9060004D1022101A8FEF78EF921
:104D50000646300035D19DF83300000648BF0626D0
:104D60002FD49DF80A60F00715D409990098FEF732
:104D7000B5FC0546F00612D5009810950E9000215E
:104D80000EA8FEF7F3FB06001BD100210EA8FEF7CC
:104D900019FD060001D1072613E0042E11D101A848
:104DA000FEF737FF060006D13DB10022294601A8D3
:104DB000FEF73EFB0646300003D10098FEF71CFAD2
:104DC0000646204600F03AF8FFF790FF30461CB048
:104DD00070BD05F11600FEF717B900984FF4007288
:104DE0000021704700990120C8700098FEF704BAAE
:104DF000E9690098FEF7E6B910B50FF2440082B0F9
:104E000000680C4600900121684600F037FB2060E6
:104E100000B1012016BD80B500F0AAFB012002BD43
:104E200010B54FF47A71002400F03EFB00B9012464
:104E3000204610BD00F06CBB00F02ABC00F0ACBCFA
:104E40000000000001461B4A501802EB8101007A65
:104E5000496849680847174A0146535C002043B92E
:104E600001205054501802EB8101007A496809680A
:104E70000847704738B500F009F8A468A04732BD6C
:104E800038B500F003F8E468A04732BD0446094D88
:104E9000281905EB8404007A6468704710B503464E
:104EA000044CE01804EB8303007A5B681B69BDE8DF
:104EB0001040184708F0032000207047802800DACF
:104EC000704710B50FF2A80349B1FF2801DD00209B
:104ED00010BD03EB4000A0F58070008810BD33F8D2
:104EE0001140A04203D0491C89B28029F7DB01F1AF
:104EF000800000F0FF0010BDB0F5805F70B5ACBF62
:104F00000FF260320FF2681202E00BB902EB4402BA
:104F1000158855B3A84228DB5488121D230204F0DB
:104F2000FF041B0C6619B042EFDA082B1DD8DFE82E
:104F300003F005090E10121416181A00401B32F85F
:104F4000100012E0411B01F00101401A0DE0103881
:104F50000BE0203809E0303807E01A3805E0083067
:104F600003E0503801E0A0F5E35080B270BD0000CE
:104F7000C700FC00E900E200E400E000E500E70013
:104F8000EA00EB00E800EF00EE00EC00C400C50012
:104F9000C900E600C600F400F600F200FB00F900CC
:104FA000FF00D600DC00F800A300D800D700920173
:104FB000E100ED00F300FA00F100D100AA00BA0010
:104FC000BF00AE00AC00BD00BC00A100AB00BB0048
:104FD00091259225932502252425C100C200C000F9
:104FE000A9006325512557255D25A200A5001025A0
:104FF000142534252C251C2500253C25E300C30061
:105000005A25542569256625602550256C25A40060
:10501000F000D000CA00CB00C8003101CD00CE00A6
:10502000CF0018250C2588258425A600CC008025D6
:10503000D300DF00D400D200F500D500B500FE009B
:10504000DE00DA00DB00D900FD00DD00AF00B400B7
:10505000AD00B1001720BE00B600A700F700B800F1
:10506000B000A800B700B900B300B200A025A000AE
:1050700061001A03E0001703F8000703FF000100B6
:1050800078010001300132010601390110014A01A5
:105090002E017901060180014D0043028101820148
:1050A00082018401840186018701870189018A01C7
:1050B0008B018B018D018E018F0190019101910176
:1050C00093019401F60196019701980198013D0220
:1050D0009B019C019D0120029F01A001A001A20152
:1050E000A201A401A401A601A701A701A901AA0187
:1050F000AB01AC01AC01AE01AF01AF01B101B20136
:10510000B301B301B501B501B701B801B801BA01E6
:10511000BB01BC01BC01BE01F701C001C101C2015C
:10512000C301C401C501C401C701C801C701CA0147
:10513000CB01CA01CD011001DD0101008E01DE01AC
:105140001201F3010300F101F401F401F801280157
:10515000220212013A020900652C3B023B023D0289
:10516000662C3F0240024102410246020A015302FC
:10517000400081018601550289018A0158028F0190
:105180005A0290015C025D025E025F0293016102BD
:105190006202940164026502660267029701960149
:1051A0006A02622C6C026D026E029C017002710236
:1051B0009D01730274029F017602770278027902E0
:1051C0007A027B027C02642C7E027F02A6018102AD
:1051D0008202A9018402850286028702AE0144028E
:1051E000B101B20145028D028E028F02900291023E
:1051F000B7017B030300FD03FE03FF03AC030400C0
:105200008603880389038A03B1031103C2030200E2
:10521000A303A303C4030803CC0303008C038E037E
:105220008F03D8031801F2030A00F903F303F40310
:10523000F503F603F703F703F903FA03FA0330045F
:10524000200350041007600422018A043601C104BF
:105250000E01CF040100C004D004440161052604FE
:10526000000000007D1D0100632C001E9601A01EA1
:105270005A01001F0806101F0606201F0806301FCF
:105280000806401F0606511F0700591F521F5B1FCB
:10529000541F5D1F561F5F1F601F0806701F0E0002
:1052A000BA1FBB1FC81FC91FCA1FCB1FDA1FDB1FB6
:1052B000F81FF91FEA1FEB1FFA1FFB1F801F0806CC
:1052C000901F0806A01F0806B01F0400B81FB91FD2
:1052D000B21FBC1FCC1F0100C31FD01F0206E01F5E
:1052E0000206E51F0100EC1FF21F0100FC1F4E210A
:1052F0000100322170211002842101008321D02479
:105300001A05302C2F04602C0201672C0601752C25
:105310000201802C6401002D260841FF1A030000C1
:105320000021842818BFC11C08467047EFF3058090
:1053300000B10120C0B2704780B500F06BFC0020C6
:1053400002BD80B5FFF7F2FF18B1BDE8014000F0E3
:10535000F3BCBDE8014000F0EBBC3EB504460D4691
:10536000B4F90800FFF7DCFF02A90090019122695F
:10537000216860682B4692B200F062FA012801D0E1
:1053800000203EBD02983EBD00F051BE80B500F049
:105390001BFB002002BD80B500B9012000F04DFBD1
:1053A000002002BD0129134680B5006818BF002106
:1053B00000900A4601216AA000F0BBFF02BD7CB547
:1053C000002405460E46019406B90126FFF7AEFFFC
:1053D00068B1009401AB32460921284600F0DCFF99
:1053E00001280DD1019860B100F0B0F809E00090FB
:1053F000002332460421284600F0CEFF012800D0C9
:10540000FF24204676BD012001F097B938B5044647
:10541000002000900CB9802032BD002511F1010F51
:1054200008BF4FF0FF3500F064F838B100F05CF8C9
:10543000012809D100F061F8002032BD294620463C
:1054400001F04FFB0128F7D0FF2032BD38B500F046
:105450008BF860B16946204601F082FA012801D03C
:10546000FF2032BD009838B100F070F804E000F081
:1054700067F8012818BFFF25284632BD012910B55D
:105480000DD103220021012001F02CF9040004D0E9
:1054900000230022002101F08AF9204610BD0846B1
:1054A000BDE8104001F067B938B50446002000900F
:1054B0000CB9802032BD002511F1010F08BF4FF05B
:1054C000FF3500F016F838B100F00EF8012809D1C8
:1054D00000F013F8002032BD2946204601F001FB00
:1054E0000128F7D0FF2032BD6A460021204601F096
:1054F000B6BB01D001B10D4618E7009838B14FF0A6
:10550000805018490860BFF34F8FBFF36F8F70470B
:1055100038B500F029F860B16946204601F020FA5C
:10552000012801D0FF2032BD009838B100F00EF8FC
:1055300004E000F005F8012818BFFF25284632BD19
:10554000002300220021204601F031B94FF08050A5
:1055500004490860BFF34F8FBFF36F8F704700009F
:105560000000000004ED00E0002504460095DDE6A3
:1055700010B500F086F808B1822010BD204601F079
:10558000ACFB002010BD41680068002201F0AAB801
:1055900032B5044682B000201546009005B90125B9
:1055A000FFF7C4FE58B100236A4602A9204601F065
:1055B0008CF901280BD1FFF7A0FF00203EBD00238E
:1055C0002A4602A9204601F0F2F80128F5D0FF2072
:1055D0003EBD7FB504460D460020029501900DB9F1
:1055E000802025E0002612F1010F039008BF4FF044
:1055F000FF3600F022F870B103AA01A9284601F095
:105600002EFB01280CBF102000200090039880B1D1
:10561000FFF79CFF0DE0324601A9284601F0DBF9B7
:10562000012808BF102003D0002E0CBF002040200E
:10563000009068460EC80EC47FBD01D002B1164668
:1056400074E680B500F0F7FC012803D0BDE8014006
:1056500001F0C1BC01BD80B500F003FA002002BD1D
:1056600010B500F00EF80028204606D000F09DFA94
:10567000012804D1FFF76AFF01E000F069FA002079
:1056800010BD044652E60268531C03601170704757
:105690002DE9F8430446002500F0EBFA664FA946D1
:1056A000B868F0B9654A4FF40C4112F00703104690
:1056B00005D0D01DC008C000C0F50C415118091814
:1056C0000839C908C90038600A1A7D60B9604D60A0
:1056D0000D604260016040683861F8604FF0004042
:1056E000786178694FF05008044241D1002C3FD0D6
:1056F000083414F0070F1FBF04F1080004F007017D
:10570000441A14F0070F00F03CF88CB3F868A0427C
:105710002ED338463E6801E030460E467168A142FD
:1057200002D231680029F7D1B9688E4220D00168D1
:1057300001F10805316801607068011B112908D367
:10574000301910F0070200F01CF84160746000F09E
:105750004EF83A697068F968091A9142F96038BFE1
:105760003961796908437060C6F8009005F007094F
:1057700000F085FAB9F1000F00F003F82846BDE803
:10578000F28308D072B688F31188BFF34F8FBFF34E
:105790006F8F62B6FEE7704738B5F0B1A0F108042C
:1057A000254D606869695022084202D100F016F860
:1057B000FEE7236813B100F011F8FEE7884360604C
:1057C00000F057FAE86861680818E860204600F0C1
:1057D0000EF8BDE8314000F052BA31BD72B682F326
:1057E0001188BFF34F8FBFF36F8F62B670471249B6
:1057F00030B50A4600E01A4613688342FBD353686B
:10580000D418844203D14068C018506010464368E1
:105810001468C518A54208D189688C4204D0616813
:10582000C9184160246800E00C468242046018BF39
:10583000106030BD0000000024EF0320684D0220FE
:105840002DE9F0430446154685B088469946A800E0
:10585000FFF71EFF06001AD05C20FFF719FF0700B4
:1058600012D03E63002003900D9801900C98009098
:105870004B4602972A464146204600F00DF838462E
:1058800000F04DF8012004E03046FFF785FF4FF0AF
:10589000FF3005B0BDE8F0832DE9F8430A9C80464F
:1058A0000F4615469946A522206BA90001F0F4FB8E
:1058B000206B00EB8500001FC508ED0005F0070018
:1058C000395C221882F83410395C11B1401C102860
:1058D000F6D3002004F14C0784F84300089E0C2EF8
:1058E00028BF0B26E6623E607860201D01F0FEFBBB
:1058F00004F1180001F0FAFBC6F10C002461A0616C
:10590000002064624A46B86041463873284601F078
:10591000C3FA2060099800B10460BDE8F1832DE965
:10592000F0410446DFF8D05801F024FBE86C14265F
:10593000DFF8C888401CE864A86A28BBAC62E86C41
:10594000012827D1002706FB07F07F1C404401F007
:10595000C0FB0C2FF7D305F1740005F1880701F0A7
:10596000B8FB384601F0B5FB284601F0B2FB05F163
:10597000140001F0AEFB05F1380001F0AAFB05F1BF
:105980007400E8622F6305E0A86D18B900F017F8FD
:1059900028BFAC62A86E0122401CA8666064E06A61
:1059A000696D8240704300F0E2FB01F000FBA86DDE
:1059B00018B1A86AE16A00F04CFCBDE8F081E06A29
:1059C000A96AC96A8842704738B50546DFF8284891
:1059D00001F0D0FA05B9A56A281D01F0AFFB28B97E
:1059E000E86A00F07FF809B900F082F8A86A18B1F7
:1059F00005F1180001F0A2FBA06E401CA066A06A91
:105A0000854208D1291D04F1140001F072FB606B7E
:105A1000401C606307E0E06C401EE064284600F034
:105A2000EFFA00F0F7FA01F0C2FAA06D20B1A06A17
:105A3000854201D100F064F831BD10B504000DD0ED
:105A4000DFF8B407006F00F0D6F900F012F900217A
:105A5000204600F017FC00F012F908B900F0F0FB46
:105A600010BD70B50646DFF8904701F083FA06B91D
:105A7000A66A301D06F1280501F060FB28B96868A8
:105A800000F030F809B900F033F8286808B100F0E8
:105A90003FF9311D04F1380001F02BFB96F8580056
:105AA000012804BF002086F8580001F080FAA06D9C
:105AB00028B101F05FFA00F0ADFA01F078FAA06ABF
:105AC00086420ED1A06D10B100F01AF870BDA06B27
:105AD000E16C884202D10020A06270BDBDE8704038
:105AE00095E170BD1422DFF81417424389587047BE
:105AF000616D012202FA00F021EA00006065704742
:105B0000206F48B172B6502080F31188BFF34F8FD9
:105B1000BFF36F8F62B6FEE74FF08050DFF84C178F
:105B20000860BFF34F8FBFF36F8F704710B5002130
:105B300000F0F2F84369DFF8C02602F13804A3420E
:105B400004D1806A904201D000B90121084610BDFD
:105B500038B500F018F800F023F813D001F00AFA75
:105B60002046FFF7E3FF48B100F05DFB00F0C8F905
:105B700001F0BFFAFFF723FF00F037FABDE831402C
:105B800001F015BA31BD040009D172B6502080F37E
:105B90001188BFF34F8FBFF36F8F62B6FEE7704778
:105BA000DFF85456A86A84427047F8B504460025C9
:105BB00050272CB972B687F3118800F05DFBFEE721
:105BC00001F022FAEFF3118672B687F3118800F024
:105BD00053FB2046FFF7AAFFC0B1DFF80C77386F00
:105BE00078B9E06AB96AC96A884228BF012500F01D
:105BF0001AFBE06A796D00F094F97965211D104473
:105C000002E004F11801384601F073FA86F31188B6
:105C10002846F2BD1CB5DFF8D046002304F19C00F5
:105C200080220190002000900FF2CC610FF27930B9
:105C3000FFF706FE012808BF00F062FB5021012893
:105C40000FD100F090FA00F017FB4FF0FF30E06644
:105C50000120A06500202065BDE8134001F047B990
:105C600013BD10F1010FFBD100F07DFA00F004FB31
:105C7000FEE7DFF87406016F491C0167704770B5D5
:105C8000DFF874550026286F002400F045F801F075
:105C900071F9286F401E2867286F002834D1E86CFE
:105CA000B0B931E0E868C66800F032F8301D01F0A4
:105CB00045FAF06A696D00F034F96965311D1044E8
:105CC00001F017FAF06AFFF77BFE24BF0120286677
:105CD00028680028E6D10EB100F09CF9EE6D3EB1C7
:105CE00000F031F808B101202866761EF8D1EC6585
:105CF000286E48B14FF08050DFF87015012408601D
:105D0000BFF34F8FBFF36F8F01F051F9204670BD85
:105D100006F1180001F012BA48B972B6502080F3AB
:105D20001188BFF34F8FBFF36F8F62B6FEE77047E6
:105D3000DFF8B405006D704780B501F065F9DFF854
:105D4000A805006D02BD2DE9F843DFF8AC5400242E
:105D5000286F002844D1286D10F10109C5F8509032
:105D60000CD1E86A006800F046F8E86A296BE9623D
:105D70002863686E401C686600F04CF9E86E1427D2
:105D8000DFF86885814520D312E0301D01F0D6F997
:105D9000B06A08B1FFF7BCFFF06A00F031FA311DBC
:105DA000404401F0A6F9F06AFFF70AFE28BF01247B
:105DB000E86A006810B94FF0FF3005E0E86AC06893
:105DC000C66870688145E0D2E866A86AC06A784310
:105DD00058F800000228E86D28BF012428B902E025
:105DE000E86D401CE86501F0C5F9286E00B101249A
:105DF0002046BDE8F28348B172B6502080F3118886
:105E0000BFF34F8FBFF36F8F62B6FEE7704710B5D9
:105E1000DFF8E443206F10B10120206610BD20663A
:105E200001F0CEF9606D1421B0FA80F0C0F11F00CE
:105E30004843DFF8B8140A5812B900F019FAFEE71F
:105E4000084400F10802416849684160914204BF7A
:105E5000496841604068C068A062BDE8104001F038
:105E6000A4B910B50C4600F018F801F04EF9204620
:105E70000121BDE8104000F005BA38B50C461546C2
:105E800000F00BF801F035F90DB14FF0FF34294661
:105E90002046BDE8344000F0F5B948B972B650204C
:105EA00080F31188BFF34F8FBFF36F8F62B6FEE7A9
:105EB000DFF83414896A1831704738B5C068C4688F
:105EC00014B900F0D5F9FEE704F11800DFF8185412
:105ED00001F034F9286F20B900F0A5F900F010F8AE
:105EE00002E004F11801284601F003F9A86AE16A0A
:105EF000C06A884202D20120286632BD002032BD2D
:105F0000E06A696D01221423824058431143DFF88F
:105F1000DC236965211D1044704772B682F3118835
:105F2000704701221423824058431143DFF8BC23F9
:105F30007047DFF8B4134A6E0260096D4160704724
:105F4000F8B504460D4650201CB972B600F092F91F
:105F5000FEE71DB972B600F08DF9FEE701F00AF810
:105F6000DFF88403016D62682E688B1A16F1010F49
:105F70000CD0406E2768B84201D091420AD2B34299
:105F800006D2F01A28602046FFF7D3FF002402E073
:105F900000202860012401F00AF82046F2BD01200B
:105FA000DFF844130866704770B5944CDFF8385337
:105FB00011E000F0DFFF286AC668301D01F0BEF86E
:105FC000E86C401EE864686B401E686300F0EFFFF9
:105FD000304600F015F8686B0028EAD120680228E6
:105FE00000F003F801F0BEF8F5E708D34FF0805059
:105FF000DFF878120860BFF34F8FBFF36F8F7047E1
:1060000010B50446206BFFF7C7FB2046BDE81040E3
:10601000FFF7C2BB7848C16A096811B94FF0FF3178
:1060200003E0C16AC968C9684968C1667047DFF89A
:10603000B802806A7047DFF8B002816D09B90120AB
:106040007047006F08B902207047002070472DE9A3
:10605000F04104460020002C40D0674DE16AAA6A56
:10606000D26A914234D2A069002804D4A86AC06AD6
:10607000C0F10C00A061142760697943DFF86C62FD
:106080003144884220D1201D4FF0010801F056F81C
:10609000002801BFE06A07FB00F17158002905D113
:1060A000696D08FA00F021EA00006865A86AC06A14
:1060B000E062696D08FA00F2784311436965211DB9
:1060C000304401F016F808E0A86AC06AE06204E013
:1060D000E16CAA6AD26A914200D20120BDE8F08147
:1060E0002DE9F04104460020002C3AD0424D5021C9
:1060F000AA6A944204D000F036F800F0BDF8FEE73A
:10610000226D22B900F02FF800F0B6F8FEE7E36C3C
:10611000511EE26A21659A4223D011BB201D01263F
:106120001427DFF8C88101F009F8002801BFE06AF0
:1061300007FB00F158F80110002905D1696D06FA36
:1061400000F021EA00006865E06CE062C0F10C003C
:10615000A061E06A696D06FA00F2784300F007F882
:106160000120BDE8F08172B681F3118870471143B8
:106170006965211D404400F0BCBFF8B5040039D06A
:10618000206D00F044F8E36C8B4238BF0B46E16AA7
:1061900099422FD001282DD1FFF702FD04D1FFF73E
:1061A000BCFE00F069F8FEE7A069E362DFF83C613D
:1061B00000285CBFC3F10C00A0611427606979431B
:1061C0003144884216D100F02EF8002801BFE06A61
:1061D00007FB00F17158002906D1696D012202FA0E
:1061E00000F021EA00006865E06A00F009F8211D6E
:1061F00030447DE0F1BD00006CE6032070E3032035
:10620000696D0122824078431143696570475022CD
:1062100040B972B682F31188BFF34F8FBFF36F8F0F
:1062200062B6FEE77047201D00F088BFDFF8B800B7
:10623000816A19B1816A0A6D521C0A65806A7047C9
:106240004FF0805009490860BFF34F8FBFF36F8F45
:106250007047C06A884207D24FF0805003490860F7
:10626000BFF34F8FBFF36F8F7047000004ED00E066
:1062700072B6502080F31188BFF34F8FBFF36F8F3A
:1062800062B67047F8B5184C0646256DA06A0F46F1
:10629000001D00F053FF40B9A06A616D0122C06A81
:1062A00002FA00F021EA0000606516F1010F05D145
:1062B00027B1A06A011D04F1380019E0A06A76191F
:1062C000AE424660A06A05D2011D206BBDE8F440D5
:1062D00000F01BBF011DE06A00F017FFE06E864270
:1062E00038BFE666F1BD00006CE6032070E30320D2
:1062F000BDE8F44000F0FDBE49444C4500000000FC
:1063000000B583B000F083F9DFF84803816861B11C
:106310000C30002301900420009080220FF23C31C9
:106320000FF2C500FFF78CFA10B900F0F8F8FEE79D
:106330000EBD2DE9FC4104460D46164698462C201C
:10634000FFF7A6F9070008D0019708980090434688
:1063500032462946204600F003F83846BDE8F6816B
:106360002DE9F0410D0004461646984602D100F092
:10637000D6F8FEE7079F6FB100F049F93C60BD61B8
:10638000FE61C7F8208006987862381DBDE8F041AC
:1063900000F0ACBEBDE8F08170B51D4684B0044687
:1063A000002314B900F0BBF8FEE7AA4EB068C0B1F4
:1063B00006290091019202940EDAFFF73CFE0228B2
:1063C00003D1089AB068002302E0B06800230022DD
:1063D000694600F0ECF903E02A46694600F075FAD8
:1063E0000346184604B070BD80B506E0C0680021C1
:1063F000006800F00AF800F0B7F8964800680168F5
:106400000029F3D101210020F3E7F0B583B0044661
:106410000E46FFF72EFC01A800F044F8054601984F
:1064200000283CD18B4F26BBA54227D3FFF727FC82
:106430003868C068C668301D00F080FEF069012829
:1064400013D1B06923462A460119304600F071F88D
:1064500058B1002000230090224600213046FFF76B
:106460009BFF10B900F05BF8FEE7716A3046884781
:10647000F7BD78680068461EB641F60FB868324628
:10648000611B00F0E5FCFFF7FAFB50B94FF08050BC
:1064900071490860BFF34F8FBFF36F8FF7BDFFF7F0
:1064A000EEFBF7BD2DE9F04182B00446FFF740FC5A
:1064B0000546684E306985420BD30020206028468F
:1064C0003561BDE8F6817860391D3F61306800F0C4
:1064D0001CFE30680168E9B1C068C768D0F8008068
:1064E000381D00F02BFE796A38468847F869012884
:1064F000EFD1B86940448045E5D3002000230090E7
:10650000424600213846FFF747FF0028E1D100F05E
:1065100006F8FEE77168706031600120CEE772B660
:10652000502080F31188BFF34F8FBFF36F8F62B697
:10653000704738B500248A424160464D006106D359
:10654000D11A8269914206D2011D686807E09A4219
:1065500003D2994201D3012403E0011D286800F011
:10656000D4FD204632BD000010B586B004E081188D
:1065700013462046FFF7DDFF36480022806801A958
:1065800000F029FA002840D001980028F4D4039C98
:10659000606910B1201D00F0D1FD04A8FFF782FF53
:1065A000024601980928E7D8DFE800F0060606054C
:1065B000242B06060524DFE70298A1690346091883
:1065C0002046FFF7B6FF0028D6D0616A20468847EC
:1065D000E0690128D0D10020002300900298A16931
:1065E0000A1800212046FFF7D7FE0028C4D1FFF784
:1065F00096FFFEE70298A0610028B8D1FFF78FFF51
:10660000FEE72046FFF7C8F8B6E706B010BD10B5A4
:1066100000F0B0FC0F4CA068C0B904F1140000F009
:1066200058FD04F1280000F054FD04F1140000228C
:10663000206004F1280060600C210A2000F052F86C
:10664000A06018B10FF21C0100F0DBFBBDE81040A8
:1066500000F0ADBCDCEC032004ED00E0546D7220D2
:1066600053766300546D72510000000038B5040089
:106670000D4602D100F075F8FEE700F07BFCE16BFF
:10668000226C20685143084460600020A063E16BE5
:10669000226C2068A0602068491E514308444FF0D6
:1066A000FF31E06004F144000170417075B9206968
:1066B000A0B104F11000FFF700FC78B14FF080505A
:1066C000DFF88417086000F0C5FA07E004F1100055
:1066D00000F0FFFC04F1240000F0FBFC00F067FC7C
:1066E000012032BDF8B504000D46164602D100F077
:1066F00038F8FEE7002D0EBF502005FB04F05030A7
:10670000FEF7C6FF070007D00097334607F1500297
:106710002946204600F002F83846F2BD38B51C463E
:10672000049D01B92A462A60E863284629640121AC
:10673000FFF79CFF85F84C4031BD0246002110B5A3
:106740000120FFF7CFFF040009D000200023606084
:10675000002220600021E060204600F028F820465A
:1067600010BD72B6502080F31188BFF34F8FBFF376
:106770006F8F62B6704710B50C46502110B900F00B
:106780000DF8FEE7A04202D200F008F8FEE7022270
:106790000021FFF7A7FF00B1846310BD72B681F33B
:1067A0001188BFF34F8FBFF36F8F62B670472DE92B
:1067B000F74F804600245025B8F1000F8B461E4647
:1067C00002D100F085F9FEE7BBF1000F08F12407C4
:1067D00001D1F86960B9022E02D1B86901280AD145
:1067E000FFF729FC70B9029860B100F071F9FEE77B
:1067F00000F06EF9FEE700F06BF9FEE700F026FA14
:10680000FFF73DFA00F0B6FB7869B969DFF8389612
:106810004FF0805A884201D3022E14D13246594695
:10682000404600F067FA396821B13846FFF745FB6A
:1068300008B904E018B1C9F800A000F00BFA00F0A4
:10684000B6FB01203FE0029810B900F0B0FB39E040
:106850001CB968460124FFF76CFB00F0A8FBFFF7AA
:1068600008FA00F087FB00F0EAF904BF002101708C
:1068700000F0CEF904BF0021417000F098FB00F059
:10688000C3F9D8B900F076FB7869B96988420CBFC2
:106890000125002500F08BFB002DAFD0029908F1F7
:1068A0001000FFF7DEFA00F0D1F9FFF7E8F9002851
:1068B000A8D1C9F800A000F0CDF9A3E700F0C6F90F
:1068C000FFF7DDF90020BDE8FE8F2DE9F047804697
:1068D0005025B8F1000F894616461F4602D100F038
:1068E000F7F8FEE7B9F1000F08F1240401D1E069DF
:1068F00030BB022F02D1A069012824D100F084FB13
:10690000EFF3118A00F0E4F86069A169884201D3CD
:10691000022F20D198F945503A464946404600F0AA
:10692000E9F915F1010F11D1206890B12046FFF768
:10693000C4FA002818BF002E0BD00120306008E0F8
:1069400000F0C6F8FEE700F0C3F8FEE7681C88F820
:106950004500012000E000208AF31188BDE8F0879F
:10696000F8B504460D46502714B900F05FF9FEE76C
:10697000206C10B100F05AF9FEE7206808B9606891
:10698000E8B900F041FBEFF3118600F04FF9A06B7E
:10699000E16B88421BD294F94510401CA06311F1B1
:1069A000010F0FD1606A80B104F12400FFF785FA6E
:1069B000002818BF002D08D00120286005E000F055
:1069C00035F9FEE7481C84F84500012000E000206E
:1069D00086F31188F2BD2DE9F44783B004468A4658
:1069E0000027502514B900F073F8FEE7BAF1000F44
:1069F00004F1100601D1306B38B9FFF71CFB58B910
:106A0000039848B100F064F8FEE700F061F8FEE793
:106A100000F003F9FFF733F900F0ACFAB56ADFF8DC
:106A200028844FF080598DB15146204600F096F9E8
:106A3000681EB062306828B13046FFF73EFA08B1F0
:106A400000F006F900F0B3FA01203EE0039810B917
:106A500000F0ADFA38E01FB968460127FFF769FA80
:106A600000F0A5FAFFF705F900F084FA00F0D7F876
:106A700004BF0021017000F0CBF804BF0021417079
:106A800000F095FA03A96846FFF75AFA0028204655
:106A900011D100F0ABF90028BAD0039904F1240019
:106AA000FFF7DFF900F0B9F8FFF7E9F80028B3D1F4
:106AB00000F0CEF8B0E700F064F9FFF7E0F8204608
:106AC00000F094F90028A7D0002004B0BDE8F087BA
:106AD00072B685F31188BFF34F8FBFF36F8F62B625
:106AE00070472DE9F24382B0044600250026502766
:106AF00014B900F09BF8FEE7206C10B100F096F896
:106B0000FEE7FFF798FA40B9029830B100F08EF82E
:106B1000FEE700F082F8FFF7B2F800F02BFAA06B66
:106B2000DFF824834FF0805998B1401EA06320689D
:106B300010B9FFF77BFB6060206930B104F11000F1
:106B4000FFF7BBF908B100F083F800F030FA01203C
:106B500058E0029820B916B100F068F8FEE74EE060
:106B60001DB968460125FFF7E4F900F020FAFFF7A8
:106B700080F800F0FFF900F052F804BF0021017026
:106B800000F046F804BF0021417000F010FA00F058
:106B90003BF8002820461BD100F028F90028B8D087
:106BA000206838B900F0E6F96068FFF750FA064649
:106BB00000F0FDF9029904F12400FFF752F900F00A
:106BC0002CF8FFF75CF80028A7D100F041F8A4E703
:106BD00000F0D7F8FFF753F8204600F007F9002837
:106BE0009BD076B100F0C6F9606A00281DBF206B0B
:106BF0000068C0F10C0100216068FFF7BEFA00F0E8
:106C0000D6F90020BDE8FE8302A96846FFF798B9CF
:106C100090F9011011F1010F70472046B1E004F125
:106C2000440090F9001011F1010F704772B687F31C
:106C30001188BFF34F8FBFF36F8F62B6704708F1B3
:106C4000440090F9001011F1010F7047404698E0A0
:106C5000C8F80090BFF34F8FBFF36F8F70472DE9D7
:106C6000F047044689461646502514B9FFF730FF11
:106C7000FEE7B9F1000F04F1100701D1386B60B9DC
:106C800000F0C2F9EFF31188FFF722FFBD6A3DB9AA
:106C9000002088F31188BDE8F087FFF719FFFEE7B1
:106CA00094F944A04946204600F058F8681E1AF1AD
:106CB000010FB8620BD1386868B13846FFF7FDF8AC
:106CC000002818BF002E06D00120306003E00AF132
:106CD000010084F844000120DBE710B5040002D174
:106CE000FFF73FFDFEE700F09CF82046BDE81040AE
:106CF000FEF752BDF8B504461746A56B226C002678
:106D000042B9206830BB6068FFF7EAF90646002008
:106D100060601FE067B9A06800F064FAA068216CA9
:106D200008446168A060884214D32068A06011E024
:106D3000E06800F057FA206CE16840420144E160ED
:106D40002268914202D261680844E060022F01D1BA
:106D500005B16D1E681CA0633046F2BD10B5026C13
:106D60000B466AB14468C1681144C160A14224BFA6
:106D70000168C160C1681846BDE8104000F032BA31
:106D800010BDF8B5044604F1440500F0F3F895F998
:106D9000016004F1100707E004F12400FFF78DF80B
:106DA00008B1FFF7FCF8761E76B2012E02DB786997
:106DB0000028F1D14FF0FF346C7000F0F8F800F0CB
:106DC000D9F895F9006006E03846FFF776F808B183
:106DD000FFF7E5F8761E76B2012E02DB3868002850
:106DE000F2D12C70BDE8F14000F0E1B810B50446D6
:106DF00000F0C0F8A06B441EA44100F0D8F8E00FEA
:106E000010BD10B50022114B53F832402CB943F895
:106E1000321003EBC201486010BD521C082AF3D3A4
:106E200010BD10B50021094A02EBC1035C68844221
:106E300004D1002042F83100586010BD491C0829D7
:106E4000F2D310BD0000000004ED00E05CEC032074
:106E5000F8B504460D46164604F1380700F08AF8E6
:106E600097F90C0010F1010F04BF0020387397F957
:106E70000D0010F1010F04BF0020787300F097F8A7
:106E8000386828B93246294604F12400FEF7F5FF98
:106E90002046BDE8F24074E74908490010B5A0F16A
:106EA00020034FF0807499610FF2150159616FF062
:106EB0000201DC611A6040F8241D203810BD00007A
:106EC00064495020496811F1010F72B607D080F370
:106ED0001188BFF34F8FBFF36F8F62B6FEE780F369
:106EE0001188BFF34F8FBFF36F8F62B6FEE71CB5FB
:106EF0005948584C01780191FF21017001788DF8B3
:106F000000109DF8001001F0500121700721A160D0
:106F100006E0491EA1609DF8001049008DF80010A0
:106F2000A1689DF800201206F3D4C1F10702042ADB
:106F300002D000F05EF8FEE7090201F4E061A16012
:106F4000019901704548016841F4700101600168D0
:106F500041F07041016000F08BF80020606000F0AB
:106F6000C9F93F48016841F04041016000F0B2F9C1
:106F7000002016BD72B6502080F31188BFF34F8FEA
:106F8000BFF36F8F62B633494A68521C012A4A60C8
:106F90000CD134490968090608D072B680F311880B
:106FA000BFF34F8FBFF36F8F62B6FEE7704729487C
:106FB000416849B972B6502080F31188BFF34F8FF2
:106FC000BFF36F8F62B6FEE7491E416004BF002029
:106FD00080F31188704780B500F00BF8FEF7B3FE20
:106FE00018B14FF080501F490860002080F31188CD
:106FF00001BD72B6502080F31188BFF34F8FBFF3ED
:107000006F8F62B670470000EFF3058050211028A3
:10701000104A0DD3144B185C1378984208D272B6FC
:1070200081F31188BFF34F8FBFF36F8F62B6FEE716
:1070300090680E4A126802F4E062904208D272B67A
:1070400081F31188BFF34F8FBFF36F8F62B6FEE7F6
:10705000704700006800002000E400E020ED00E040
:1070600034EF00E004ED00E0F0E300E00CED00E0C0
:107070000748002101604FF47A7281600549096870
:10708000B1FBF2F1491E416007210160704700BF6A
:1070900010E000E00001002062F30F2262F31F42C3
:1070A00000B500BF130096469446103928BFA0E8EB
:1070B0000C50FAD85FEA417C28BF0CC048BF40F8AA
:1070C000042BC90728BF20F8022B48BF00F8012B6A
:1070D00000BD00F1080141604FF0FF31816000F117
:1070E0000801C16001610021016070470021016158
:1070F000704742684A6093688B60936859609160FA
:1071000008610168491C0160704730B50A6812F1D6
:10711000010F08BF036907D000F1080300E0234610
:107120005C682568AA42FAD25A684A6091608B600E
:10713000596008610168491C016030BD43680169FC
:1071400082689A60836842685A604A68824204BFD3
:1071500082684A60002202610868401E0860086870
:107160007047000010B51E4C206810B9FEF75FFF95
:10717000206010BD1A4840F2E93341694A1C994227
:1071800011DB01690022994224BF4FF47A71016139
:107190000169642359434FF47A73B1FBF3F1C1F1F0
:1071A0006401416002614261704710B5FEF73FFF24
:1071B0000B4C2168884202D1FEF7BEFDA06010BDD5
:1071C00010B5FEF734FF064C2168884207D1FEF760
:1071D000B3FDA168401A2169E0604018206110BD2C
:1071E0000CEF032062B38B0708D0521E11F8013B4D
:1071F00000F8013B00F024808B07F6D1830740F0B4
:10720000208000BF103A07D330B4B1E83810103AEC
:10721000A0E83810F9D230BC530724BFB1E80810F9
:10722000A0E8081044BF51F8043B40F8043BD207E3
:1072300024BF31F8022B20F8022B44BF0B780370D7
:107240007047083A07D3B1E80810083A40F8043B01
:1072500040F804CBF7D25307E4E70000EFF30980CE
:10726000BFF36F8F274B1A681EF0100F08BF20ED79
:10727000108A20E9F04F106009B44FF0500072B648
:1072800080F31188BFF34F8FBFF36F8F62B6FEF7A5
:10729000BEFD4FF0000080F3118809BC1968086832
:1072A000B0E8F04F1EF0100F08BFB0EC108A80F36A
:1072B0000988BFF36F8F7047124B19680868B0E8F0
:1072C000F04F80F30988BFF36F8F4FF0000080F319
:1072D000118870470C480068006880F308884FF0F8
:1072E000000080F3148862B661B6BFF34F8FBFF31E
:1072F0006F8F00DFDFF81400016841F47001016056
:107300007047000094E6032008ED00E088ED00E0FF
:107310004FF4E07210440268914203D343681A4468
:10732000914202D380680028F5D17047DFF85C07EE
:10733000016891B94FF4803181604FF48051416010
:107340004FF0FF31C16001610421DFF84427416142
:10735000C2F8BC11DFF83C1701600120704701F151
:10736000080313F0070305D001F10803C3F1080374
:1073700003F007031944D21A8161C26042F001038D
:107380004B60114428234B60DFF800170969C16185
:1073900070472DE9F84F064601F1080010F007008C
:1073A00008BF884607D001F10800C0F1080000F0CE
:1073B000070001EB000802F1080010F0070006D0FA
:1073C00002F10800C0F1080000F007000244154671
:1073D000A5EB0800A0EB030908EB030B43F0030047
:1073E000C8F80400AB4528BF01F00CFA2879C007A3
:1073F00058BF01F007FAB9F1100F38BF01F002FAD7
:10740000B069854209D1F0684844F060C6F818B008
:1074100040F00100CBF8040070E1706985420BD1A7
:10742000B0684844B060C6F814B040F00101CBF831
:1074300004104BF8000061E1686800F003010129C5
:1074400040F0AF80C008C0000190C00820283BD2A7
:10745000D5F808A0EF680090BD4208BF01F0D2F94E
:10746000554508BF01F0CEF968680099C008C00012
:10747000B0EBC10F18BF01F0C5F9009806EBC000D2
:1074800000F128018A4508D031698A45C0F084801E
:10749000DAF80C10A94240F07F80574506D1009AD7
:1074A0003068012191408843306077E0283087427E
:1074B00005D0306987426FD3B868A8426CD1CAF84A
:1074C0000C70C7F808A069E0EF68D5F818A0AF42C3
:1074D0000CD0A8683169884223D3C168A94204BF8F
:1074E000B968A9421DD1C760B8601CE005F114005D
:1074F000076837B905F110000768A7B101E0084631
:10750000076807F114010A68002A02BF07F1100199
:107510000A68002AF3D13169884202D30021016050
:1075200001E001F06FF9BAF1000F37D0E86906EB1E
:1075300080004FF49871084401688D4208D10760BB
:10754000A7B9EA697068012191408843706025E01D
:107550003069824508D3DAF81000A84214BFCAF88F
:107560001470CAF8107001E001F04CF9B7B130693D
:10757000874211D3C7F818A0296929B1814226BFD3
:1075800039618F6101F03EF9686938B1316988422B
:1075900002D37861876101E001F034F90198054474
:1075A000814468684008400068604FEAD90549F0A6
:1075B0000100CBF804004BF80990202D23D206EBF4
:1075C000C50000F12807BA46B9F1100F38BF01F025
:1075D00019F9306820FA05F1C90704D40121A9403E
:1075E0000843306006E0B868316988422CBF8246A3
:1075F00001F008F9C7F808B0CAF80CB0CBF808A039
:10760000CBF80C707AE05FEA192108BF002023D084
:10761000B1F5803F28BF1F201ED2A1F58070000C5D
:1076200000F008008140A1F58052120C02F0040223
:107630009140A1F580431B0CC0F10E0003F0020342
:10764000801AC01A994000EBD130C11D29FA01F20D
:1076500002F0010101EB400006EB80014FF498724B
:107660001144CBF81C000022CBF81420CBF81020DA
:10767000726822FA00F3DB0707D4012303FA00F053
:1076800010437060C1F800B01DE009681F281DBFDD
:107690004008C0F1190009FA00F0484600E0114620
:1076A0004A68D208D2004A4514D0C20F01EB8202C8
:1076B00002F1100340001A68002AF0D130698342B9
:1076C0001AD3C3F800B0CBF81810CBF80CB0CBF835
:1076D00008B013E032698868914228BF90420BD30A
:1076E000C0F80CB0C1F808B0CBF80800CBF80C100B
:1076F0000020CBF8180001E001F084F808F1080040
:10770000BDE8E68F2DE9FA4D0546DFF880030068F5
:1077100082B008B9FFF70AFEDFF8700302998068AB
:1077200041182F31401E21EA00000299814280F069
:10773000A9814FF4D8716E18B16839B132688018D8
:10774000824280F09F818142C0F09C8101F05EF80E
:1077500000281EBF0446D0F8008014F1010F00F08D
:1077600091813068716840448142306038BF014681
:107770007160A86980BB286908B1844200D22C617D
:107780000020F0613461C6F8148005F12801BF487B
:10779000006868624FF0FF3028620020C96089608D
:1077A00001F108024A610A61801C10312028F5D3DA
:1077B000B748854203D1A8F1280221462AE055F8AE
:1077C000040CC00805EBC000A0F1080104EB0800A0
:1077D000401AA0F128021DE04FF4E0702918084675
:1077E00000E08068D0B1026843681A449442F8D13E
:1077F000027B120712D4AA6903689A420ED3476823
:107800003B449A420AD208EB07014160E868A96943
:1078100008EB00022846FFF7A2FD1DE1286984421B
:10782000084638BF2C6104EB080100E0806880B195
:1078300002688A42FAD1017B09070AD404604168D0
:10784000414441602146029B284604B0BDE8F04D0A
:107850009FE5AF6939462846FFF75AFD4FF0000B08
:107860000168406808440190273810F00701019929
:107870000EBF0020C0F1080000F0070008442F38B8
:1078800007F11001884234BF00970090009804F17E
:10789000080100F1180A11F00701A8F1280005D02D
:1078A00004F10801C1F1080101F00701401A214467
:1078B000A961E86040F001024A6008442822426061
:1078C00072480069E8610098083010F0070018BF9E
:1078D00000F098FF00991B2048604FF4E0712944A4
:1078E000B1E80C5000980830A0E80C503461C6F89C
:1078F0001480C6F81CB000980830B061019801E00F
:107900000AF1040A0721CAF804100BF1010B0AF16D
:1079100008018142F4D3BBF1020FB8BF00F072FF3F
:107920000098B84200F09880C01B3918C4084A6813
:10793000520852004A6040F0010179603850202C12
:1079400020D205EBC40101F12806B046102838BF4B
:1079500000F058FF286820FA04F1C90704D4012177
:10796000A1400843286006E0B068296988422CBF1E
:10797000804600F047FFB760C8F80C70C7F8088071
:10798000FE6069E0010A23D0B1F5803F28BF1F21C6
:107990001ED2A1F58072120C02F008029140A1F5EE
:1079A00080531B0C03F004039940A1F58044240C80
:1079B000C2F10E0204F00204D21A121BA14002EB23
:1079C000D131CA1D20FA02F303F0010202EB41019A
:1079D00005EB81024FF498731A44F96100237B612F
:1079E0003B616B6823FA01F4E40705D40120884069
:1079F0001843686017601CE012681F291DBF490802
:107A0000C1F1190100FA01F1014600E01A4653687C
:107A1000DB08DB00834210D0CB0F02EB830303F1C2
:107A2000100449002368002BF0D12869844211D347
:107A30002760BA61FF60BF600EE0296990688A42E2
:107A400028BF884206D3C7609760B860FA600020FC
:107A5000B86101E000F0D6FEE8680299814211D2D7
:107A6000401AE860A969029A0A44AA6140F001003C
:107A70005060029840F00300486004B001F1080033
:107A8000BDE8F08D002004B0BDE8F08D6CEF032060
:107A900074E003206859883C2DE9F84F044600261D
:107AA00089465FEA1920C9F1000B08BF002123D0E5
:107AB000B0F5803F28BF1F211ED2A0F58071090CB0
:107AC00001F008018840A0F58052120C02F0040277
:107AD0009040A0F580431B0CC1F10E0103F002039E
:107AE000891AC91A984001EBD030C11D29FA01F258
:107AF00002F0010101EB400104EB8100D0F83001FC
:107B000018B31F290FBF4A464A08C2F1190209FAE1
:107B100002F2002300E052004568ED08ED00A5EBFD
:107B200009055D4503D25FEA050B06460BD04569A2
:107B3000D70F00EB8700002D00691CBF85422B4644
:107B40000028E8D11846B8BBC6BB012088404000D9
:107B5000414208436168084000F05D8141420840AD
:107B6000401E010B01F01001C840420902F008025A
:107B7000D040830803F00403D840450805F002050F
:107B80005118E8405918C0F3400729443944F840D7
:107B9000401804EB8000D0F830010DE00846416841
:107BA000C908C900A1EB090159453CBF8B460646EF
:107BB00001690029F2D140690028F0D1002E00F0BF
:107BC0002A81A068A0EB0900834580F02481206908
:107BD0008642C0F01E817068C00809EB0B08C00027
:107BE000404518BF00F00EFE06EB0905AE4280F0DE
:107BF0001081F768D6F818A0B7420CD0B068216998
:107C0000884223D3C168B14204BFB968B1421DD1D3
:107C1000C760B8601CE006F11400076837B906F1C8
:107C200010000768A7B101E00846076807F11401D2
:107C30000A68002A02BF07F110010A68002AF3D17E
:107C40002169884202D30021016001E000F0DAFDE1
:107C5000BAF1000F39D0F06904EB80004FF498714D
:107C6000084401688E4209D10760380014D1F269D6
:107C70006068012191408843606026E02069824568
:107C800008D3DAF81000B04214BFCAF81470CAF86A
:107C9000107001E000F0B6FDBFB12069874212D339
:107CA000C7F818A0306930B12169884226BF386111
:107CB000876100F0A7FD706938B12169884202D35D
:107CC0007861876101E000F09DFDBBF1100F09D2E2
:107CD00048F00300706006EB0800416841F00101C4
:107CE000416095E049F0030070604BF0010068606E
:107CF0004FEADB0045F80BB020281DD204EBC00191
:107D000001F12807216821FA00F2D207BB4605D409
:107D1000012202FA00F00843206006E0B8682169F9
:107D200088422CBF834600F06DFDBD60CBF80C503F
:107D3000C5F808B0EF606BE05FEA1B2023D0B0F518
:107D4000803F28BF1F201ED2A0F58071090C01F0D2
:107D500008018840A0F58052120C02F00402904005
:107D6000A0F580431B0CC1F10E0103F00203891A38
:107D7000C91A984001EBD030C11D2BFA01F202F074
:107D8000010101EB400004EB80014FF498721144B3
:107D9000E86100226A612A61626822FA00F3DB0767
:107DA00006D4012303FA00F0104360600D601CE06C
:107DB00009681F281DBF4008C0F119000BFA00F028
:107DC000584600E011464A68D208D2005A4510D001
:107DD000C20F01EB820202F1100340001A68002A70
:107DE000F0D12069834211D31D60A961ED60AD60BF
:107DF0000EE022698868914228BF904206D3C56090
:107E00008D60A860E9600020A86101E000F0FAFC44
:107E100008E100F0F7FC02E12DE9F84F044688463E
:107E2000606841420840401E010B01F01001C8404B
:107E3000420902F00802D040830803F00403D8404E
:107E4000450805F002055118E8405918C0F34006EE
:107E500029447118F040401804EB8000D0F830013C
:107E60004168C908C9000646A1EB080A09E00846AE
:107E70004168C908C900A1EB080151453CBF8A46C9
:107E8000064601690029F2D140690028F0D1206935
:107E90008642C0F0C2807068C00808EB0A09C000C2
:107EA000484518BF00F0AEFC06EB080B5E4580F0BD
:107EB000B480F768B569B7420CD0B06821698842D0
:107EC00023D3C168B14204BFB968B1421DD1C760B4
:107ED000B8601CE006F11400076837B906F110001D
:107EE0000768A7B101E00846076807F114010A68AE
:107EF000002A02BF07F110010A68002AF3D12169A4
:107F0000884202D30021016001E000F07BFC002DDB
:107F100035D0F06904EB80004FF498710844016893
:107F20008E4209D10760380011D1F26960680121E1
:107F300091408843606022E02069854205D328692A
:107F4000B04214BF6F612F6101E000F05BFCB7B17C
:107F50002069874211D3BD61306930B121698842FF
:107F600026BF3861876100F04DFC706938B1216926
:107F7000884202D37861876101E000F043FCBAF1E6
:107F8000100F09D249F00300706006EB0900416848
:107F900041F0010141603FE048F0030070604AF0A9
:107FA0000100CBF804004BF80AA0D4F808804FEA8F
:107FB000D805202D28BF00F025FCB8F1000F27D0F0
:107FC000D4F81490009504EBC50000F128052F4665
:107FD000B8F1100F38BF00F015FC2068009920FAA6
:107FE00001F2D10705D4009A012191400843206095
:107FF00006E0A868216988422CBF074600F002FC11
:10800000C5F80890C7F80C90C9F80870C9F80C506A
:10801000C4F808A0C4F814B004E000F0F3FB00209A
:10802000BDE8F28F06F10800BDE8F28F2DE9F04FB0
:1080300083B00546AFF30080F52DDFF8C04780F030
:1080400002810B2D31BF102705F10B00C708FF007F
:108050002068FE08F04010F0030F42D0C04300F04B
:108060000100861904EBC60000F12808F700D8F8D3
:1080700008506868C008C000B84218BF00F0C2FBD2
:10808000D5F80890454508BF00F0BCFB4D4508BF3A
:1080900000F0B8FB6868C008C000B84218BF00F024
:1080A000B1FBC84505D120680121B140884320605B
:1080B0000DE02069814508D3D9F80C00A84204D10D
:1080C000C8F80890C9F80C8001E000F09BFB47F06D
:1080D00003006860E8190835416841F0010141601A
:1080E000F9E0A168B94280F0C080002800F0A280C9
:1080F000012505FA06F149004A42B0401143084003
:1081000041420840401E010B01F01001C8404209E5
:1081100002F00802D040830803F00403D840460868
:1081200006F002065118F0405918C0F340087118C3
:10813000414420FA08F000EB010804EBC80000F10C
:1081400028094FEAC80AD9F808607068C008C0005A
:10815000504518BF00F056FBD6F808B04E4508BF92
:1081600000F050FB5E4508BF00F04CFB7068C00893
:10817000C000504518BF00F045FBD94505D1206827
:1081800005FA08F1884320600DE02069834508D393
:10819000DBF80C00B04204D1C9F808B0CBF80C9061
:1081A00001E000F02FFB47F003007060AAEB070826
:1081B000F019019048F0010001994860019840F8D9
:1081C0000880A7684FEAD70ABAF1200F28BF00F04D
:1081D00019FB47B3CDF800A004EBCA00D4F8149003
:1081E00000F1280AD346102F38BF00F00BFB20689F
:1081F000009920FA01F2D10705D4009905FA01F19E
:108200000843206007E0DAF80800216988422CBFA3
:10821000834600F0F7FACAF80890CBF80C90C9F83A
:1082200008B0C9F80CA0C4F8088006F10805019848
:10823000606150E06068C0B339462046FFF7ECFD4E
:10824000050012D047E015F1400F28BF4FF0FF376F
:108250000BD205F10B00C7086068FF0028B1394652
:108260002046FFF719FC050035D1A068B8421CD3A1
:10827000C11B626910290AD3D0196061A16041F065
:1082800001034360415047F0030050600AE00021C1
:10829000A160616140F0030151601044416841F008
:1082A0000101416002F1080515E0E06887420DD246
:1082B000C01BA169E060CA19A26140F001005060D2
:1082C00001F1080547F00300486004E03946204604
:1082D000FFF718FA0546AFF30080284603B0BDE863
:1082E000F08F00B970472DE9F047A0F10804AFF313
:1082F0000080DFF8085528698442C0F079826168FF
:1083000001F00302012A00F07382CA084FEAC20892
:10831000CA0704EB080937D4226811F0030F00F0F4
:10832000698251420C4484429044C0F06182696980
:108330008C4200F0D980D608202E70D2D4F80CA040
:10834000A768544508BF00F05DFABC4208BF00F0C2
:1083500059FA6068C008C000B0EBC60F18BF00F043
:1083600051FA05EBC60000F128018F4205D02969BA
:108370008F4251D3F968A1424ED1BA453DD1286808
:108380000121B140884328604C4580F03182D9F802
:108390000400C10740F12C82810700F17D81A969A9
:1083A000894540F0B680E868AC614044E86040F040
:1083B0000101616069698C4202D100216961A96093
:1083C000E969814280F01682DFF83404006808B958
:1083D000FEF7ACFFA969002900F00C82E8682928A3
:1083E00024BF2846FEF794FFE869E968884280F0D8
:1083F00001824FF0FF30E861FCE12830824506D071
:108400002869824508D3DAF80800A04204D1C7F8E9
:108410000CA0CAF80870B7E700F0F4F9B4E7E76811
:10842000A669A7420BD0A168814222D3C868A042A6
:1084300004BFB868A0421CD1CF60B9601BE004F152
:1084400014010F6837B904F110010F689FB101E002
:1084500011460F6807F114021368002B02BF07F1E1
:1084600010021368002BF3D1814202D30020086070
:1084700001E000F0C7F9002E86D0E06905EB80002E
:108480004FF49871084401688C4209D107603800A4
:1084900011D1E2696868012191408843686073E7FF
:1084A0002869864205D33069A04214BF77613761DD
:1084B00001E000F0A7F9002F3FF466AF286987427A
:1084C000AAD3BE61216929B1814226BF39618F617A
:1084D00000F098F9606900283FF456AF2969884296
:1084E0009AD3786187614FE799F8040000F00300A0
:1084F00003287FF449AFC5F80880D9F80400400884
:108500004000C9F8040048F00100606044F80880A9
:1085100070E16969894508D1A8686C614044A86028
:1085200040F001016160205064E1C008C0004FEAE2
:10853000D00ABAF1200F804437D2D9F80C70D9F89C
:108540000860B94508BF00F05DF9B14508BF00F00B
:1085500059F9D9F80400C008C000B0EBCA0F18BF21
:1085600000F050F905EBCA0000F128018E4207D057
:1085700029698E42C0F08380F168494540F07F80D0
:10858000B74206D12868012101FA0AF18843286020
:1085900077E02830874205D0286987426FD3B868D2
:1085A00048456CD1F760BE606BE0D9F80C70D9F823
:1085B00018604F450DD0D9F808002969884223D3A7
:1085C000C168494504BFB96849451DD1C760B86055
:1085D0001CE009F11400076837B909F110000768B9
:1085E000A7B101E00846076807F114010A68002AEC
:1085F00002BF07F110010A68002AF3D129698842F5
:1086000002D30021016001E000F0FCF8002E38D018
:10861000D9F81C0005EB80004FF4987108440168FC
:1086200089450AD10760380012D1D9F81C20686842
:10863000012191408843686023E02869864205D380
:108640003069484514BF7761376101E000F0DAF81E
:10865000BFB12869874212D3BE61D9F8101029B181
:10866000814226BF39618F6100F0CCF8D9F814003F
:1086700038B12969884202D37861876101E000F04E
:10868000C1F848F00100606044F8088068698442DD
:108690000BD1C5F80880ADE040084000C9F80400DF
:1086A00048F00100606044F808804FEAD807202FA6
:1086B00022D205EBC70000F128094E46B8F1100F91
:1086C00038BF00F09FF8286820FA07F1C90704D4E2
:1086D0000121B9400843286007E0D9F8080029695A
:1086E00088422CBF064600F08DF8C9F80840F460B7
:1086F000A660C4F80C907DE05FEA182008BF002156
:1087000023D0B0F5803F28BF1F211ED2A0F5807175
:10871000090C01F008018840A0F58052120C02F00B
:1087200004029040A0F580431B0CC1F10E0103F040
:108730000203891AC91A984001EBD030C11D28FAEA
:1087400001F202F0010101EB400105EB81004FF461
:1087500098721044002262612261E1616A6822FA23
:1087600001F3DB0706D4012303FA01F11143696029
:1087700004601CE000681F291DBF4908C1F11901F0
:1087800008FA01F1414600E010464268D208D200E2
:10879000424510D0CA0F00EB820202F110034900DB
:1087A0001A68002AF0D129698B4211D31C60A0619C
:1087B000E460A4600EE02A698168904228BF91427B
:1087C00006D3CC608460E060A1600020A06101E07D
:1087D00000F018F8286A401E28620BD1D5F8C801AD
:1087E00000E080680028FCD14FF0FF30286201E0F3
:1087F00000F008F8AFF30080BDE8F08774E00320D4
:108800006CEF0320012000F017B80000074908684A
:1088100008B1002070470648C008C000086005493C
:10882000C908C900091A0160704700BF54F103204C
:108830006F2500206845002080B5AFF30080024A14
:1088400011001820ABBEFBE7260002000001081053
:108850000902030A11182019120B04050C131A211E
:10886000283029221B140D06070E151C232A313827
:1088700039322B241D160F171E252C333A3B342D6D
:10888000261F272E353C3D362F373E3F3F3F3F3F8B
:108890003F3F3F3F3F3F3F3F3F3F3F3F00000000E4
:1088A00001000000020000000400000008000000B9
:1088B00010000000200000004000000080000000C8
:1088C0000001000000020000000400000008000099
:1088D0000010000000200000004000000000000028
:1088E000FFFFFFFFFDFFFFFFF9FFFFFFF1FFFFFFAE
:1088F000E1FFFFFFC1FFFFFF81FFFFFF01FFFFFF60
:1089000001FEFFFF01FCFFFF01F8FFFF01F0FFFF89
:1089100001E0FFFF01C0FFFF0180FFFF4DFFFFFFF0
:108920004EFFFFFF4FFFFFFF51FFFFFF52FFFFFF13
:1089300054FFFFFF55FFFFFF56FFFFFF58FFFFFFEC
:1089400059FFFFFF5BFFFFFF5CFFFFFF5DFFFFFFC6
:108950005FFFFFFF60FFFFFF62FFFFFF63FFFFFF9F
:1089600064FFFFFF66FFFFFF67FFFFFF69FFFFFF79
:108970006AFFFFFF6BFFFFFF6DFFFFFF6EFFFFFF53
:1089800070FFFFFF71FFFFFF72FFFFFF74FFFFFF2C
:1089900075FFFFFF77FFFFFF78FFFFFF79FFFFFF06
:1089A0007BFFFFFF7CFFFFFF7EFFFFFF7FFFFFFFDF
:1089B00080FFFFFF82FFFFFF83FFFFFF85FFFFFFB9
:1089C00086FFFFFF87FFFFFF89FFFFFF8AFFFFFF93
:1089D0008CFFFFFF8DFFFFFF8EFFFFFF90FFFFFF6C
:1089E00091FFFFFF93FFFFFF94FFFFFF95FFFFFF46
:1089F00097FFFFFF98FFFFFF9AFFFFFF9BFFFFFF1F
:108A00009CFFFFFF9EFFFFFF9FFFFFFFA1FFFFFFF8
:108A1000A2FFFFFFA3FFFFFFA5FFFFFFA6FFFFFFD2
:108A2000A8FFFFFFA9FFFFFFAAFFFFFFACFFFFFFAB
:108A3000ADFFFFFFAFFFFFFFB0FFFFFFB1FFFFFF85
:108A4000B3FFFFFFB4FFFFFFB6FFFFFFB7FFFFFF5E
:108A5000B8FFFFFFBAFFFFFFBBFFFFFFBDFFFFFF38
:108A6000BEFFFFFFC0FFFFFFC1FFFFFFC2FFFFFF11
:108A7000C4FFFFFFC5FFFFFFC7FFFFFFC8FFFFFFEA
:108A8000C9FFFFFFCBFFFFFFCCFFFFFFCEFFFFFFC4
:108A9000CFFFFFFFD0FFFFFFD2FFFFFFD3FFFFFF9E
:108AA000D5FFFFFFD6FFFFFFD7FFFFFFD9FFFFFF77
:108AB000DAFFFFFFDCFFFFFFDDFFFFFFDEFFFFFF51
:108AC000E0FFFFFFE1FFFFFFE3FFFFFFE4FFFFFF2A
:108AD000E5FFFFFFE7FFFFFFE8FFFFFFEAFFFFFF04
:108AE000EBFFFFFFECFFFFFFEEFFFFFFEFFFFFFFDE
:108AF000F1FFFFFFF2FFFFFFF3FFFFFFF5FFFFFFB7
:108B0000F6FFFFFFF8FFFFFFF9FFFFFFFAFFFFFF90
:108B1000FCFFFFFFFDFFFFFFFFFFFFFF0000000066
:108B20000100000003000000040000000600000037
:108B300007000000080000000A0000000B00000011
:108B40000D0000000E0000000F00000011000000EA
:108B500012000000140000001500000016000000C4
:108B600018000000190000001B0000001C0000009D
:108B70001D0000001F000000200000002200000077
:108B80002300000024000000260000002700000051
:108B9000290000002A0000002B0000002D0000002A
:108BA0002E00000030000000310000003200000004
:108BB00034000000350000003700000038000000DD
:108BC000390000003B0000003C0000003E000000B7
:108BD0003F00000040000000420000004300000091
:108BE0004500000046000000480000004900000069
:108BF0004A0000004C0000004D0000004F00000043
:108C0000500000005100000053000000540000001C
:108C10005600000057000000580000005A000000F5
:108C20005B0000005D0000005E0000005F000000CF
:108C300061000000620000006400000065000000A8
:108C40006600000068000000690000006B00000082
:108C50006C0000006D0000006F000000700000005C
:108C60007200000073000000740000007600000035
:108C700077000000790000007A0000007B0000000F
:108C80007D0000007E0000008000000081000000E8
:108C900082000000840000008500000087000000C2
:108CA00088000000890000008B0000008C0000009C
:108CB0008E0000008F000000900000009200000075
:108CC000930000009500000096000000970000004F
:108CD000990000009A0000009C0000009D00000028
:108CE0009E000000A0000000A1000000A300000002
:108CF000A4000000A5000000A7000000A8000000DC
:108D0000AA000000AB000000AC000000AE000000B4
:108D1000AF000000B1000000B200000000695B007D
:108D20002EB25A005CFB59008A445900B88D580095
:108D3000E6D65700142057004269560070B255001D
:108D40009EFB5400CC445400FA8D530028D75200A7
:108D50005620520084695100B2B25000E0FB4F002F
:108D60000E454F003C8E4E006AD74D0098204D00B6
:108D7000C6694C00F4B24B0022FC4A0050454A0040
:108D80007E8E4900ACD74800DA204800086A4700C8
:108D900036B3460064FC450092454500C08E440051
:108DA000EED743001C2143004A6A420078B34100D9
:108DB000A6FC4000D4454000028F3F0030D83E0062
:108DC0005E213E008C6A3D00BAB33C00E8FC3B00EB
:108DD00016463B00448F3A0072D83900A021390072
:108DE000CE6A3800FCB337002AFD360058463600FC
:108DF000868F3500B4D83400E2213400106B330084
:108E00003EB432006CFD31009A463100C88F30000C
:108E1000F6D82F0024222F00526B2E0080B42D0094
:108E2000AEFD2C00DC462C000A902B0038D92A001D
:108E300066222A00946B2900C2B42800F0FD2700A6
:108E40001E4727004C9026007AD92500A82225002D
:108E5000D66B240004B5230032FE220060472200B6
:108E60008E902100BCD92000EA222000186C1F003F
:108E700046B51E0074FE1D00A2471D00D0901C00C8
:108E8000FED91B002C231B005A6C1A0088B5190050
:108E9000B6FE1800E44718001291170040DA1600D9
:108EA0006E2316009C6C1500CAB51400F8FE130062
:108EB000264813005491120082DA1100B0231100E9
:108EC000DE6C10000CB60F003AFF0E0068480E0072
:108ED00096910D00C4DA0C00F2230C00206D0B00FB
:108EE0004EB60A007CFF0900AA480900D891080084
:108EF00006DB070034240700626D060090B605000B
:108F0000BEFF0400EC4804001A92030048DB020094
:108F100076240200A46D0100D2B60000000000001B
:108F20002E49FFFF5C92FEFF8ADBFDFFB824FDFFA8
:108F3000E66DFCFF14B7FBFF4200FBFF7049FAFF30
:108F40009E92F9FFCCDBF8FFFA24F8FF286EF7FFBA
:108F500056B7F6FF8400F6FFB249F5FFE092F4FF42
:108F60000EDCF3FF3C25F3FF6A6EF2FF98B7F1FFCA
:108F7000C600F1FFF449F0FF2293EFFF50DCEEFF53
:108F80007E25EEFFAC6EEDFFDAB7ECFF0801ECFFDB
:108F9000364AEBFF6493EAFF92DCE9FFC025E9FF64
:108FA000EE6EE8FF1CB8E7FF4A01E7FF784AE6FFEC
:108FB000A693E5FFD4DCE4FF0226E4FF306FE3FF75
:108FC0005EB8E2FF8C01E2FFBA4AE1FFE893E0FFFE
:108FD00016DDDFFF4426DFFF726FDEFFA0B8DDFF86
:108FE000CE01DDFFFC4ADCFF2A94DBFF58DDDAFF0F
:108FF0008626DAFFB46FD9FFE2B8D8FF1002D8FF97
:109000003E4BD7FF6C94D6FF9ADDD5FFC826D5FF1F
:10901000F66FD4FF24B9D3FF5202D3FF804BD2FFA7
:10902000AE94D1FFDCDDD0FF0A27D0FF3870CFFF30
:1090300066B9CEFF9402CEFFC24BCDFFF094CCFFB9
:109040001EDECBFF4C27CBFF7A70CAFFA8B9C9FF41
:10905000D602C9FF044CC8FF3295C7FF60DEC6FFC9
:109060008E27C6FFBC70C5FFEAB9C4FF1803C4FF52
:10907000464CC3FF7495C2FFA2DEC1FFD027C1FFDB
:10908000FE70C0FF2CBABFFF5A03BFFF884CBEFF63
:10909000B695BDFFE4DEBCFF1228BCFF4071BBFFEC
:1090A0006EBABAFF9C03BAFFCA4CB9FFF895B8FF75
:1090B00026DFB7FF5428B7FF8271B6FFB0BAB5FFFD
:1090C000DE03B5FF0C4DB4FF3A96B3FF68DFB2FF85
:1090D0009628B2FFC471B1FFF2BAB0FF2004B0FF0E
:1090E0004E4DAFFF7C96AEFFAADFADFFD828ADFF97
:1090F0000672ACFF34BBABFF6204ABFF904DAAFF1E
:10910000BE96A9FFECDFA8FF1A29A8FF4872A7FFA7
:1091100076BBA6FFA404A6FFD24DA5FF008D2C00B0
:10912000E6342C00CCDC2B00B2842B00982C2B00D6
:109130007ED42A00647C2A004A242A0030CC2900EC
:1091400016742900FC1B2900E2C32800C86B280004
:10915000AE13280094BB27007A632700600B27001A
:1091600046B326002C5B260012032600F8AA250031
:10917000DE522500C4FA2400AAA22400904A24004A
:1091800076F223005C9A23004242230028EA220060
:109190000E922200F4392200DAE12100C089210078
:1091A000A63121008CD9200072812000582920008E
:1091B0003ED11F0024791F000A211F00F0C81E00A5
:1091C000D6701E00BC181E00A2C01D0088681D00BD
:1091D0006E101D0054B81C003A601C0020081C00D2
:1091E00006B01B00EC571B00D2FF1A00B8A71A00EC
:1091F0009E4F1A0084F719006A9F19005047190002
:1092000036EF18001C971800023F1800E8E6170018
:10921000CE8E1700B43617009ADE16008086160030
:10922000662E16004CD61500327E15001826150045
:10923000FECD1400E4751400CA1D1400B0C513005F
:10924000966D13007C15130062BD12004865120074
:109250002E0D120014B51100FA5C1100E00411008B
:10926000C6AC1000AC54100092FC0F0078A40F00A4
:109270005E4C0F0044F40E002A9C0E0010440E00B9
:10928000F6EB0D00DC930D00C23B0D00A8E30C00D3
:109290008E8B0C0074330C005ADB0B0040830B00E8
:1092A000262B0B000CD30A00F27A0A00D8220A00FF
:1092B000BECA0900A47209008A1A090070C2080017
:1092C000566A08003C12080022BA0700086207002C
:1092D000EE090700D4B10600BA590600A001060045
:1092E00086A905006C51050052F9040038A104005C
:1092F0001E49040004F10300EA980300D040030073
:10930000B6E802009C9002008238020068E001008A
:109310004E880100343001001AD80000008000009F
:10932000E6270000CCCFFFFFB277FFFF981FFFFFBB
:109330007EC7FEFF646FFEFF4A17FEFF30BFFDFFD2
:109340001667FDFFFC0EFDFFE2B6FCFFC85EFCFFEA
:10935000AE06FCFF94AEFBFF7A56FBFF60FEFAFF01
:1093600046A6FAFF2C4EFAFF12F6F9FFF89DF9FF18
:10937000DE45F9FFC4EDF8FFAA95F8FF903DF8FF30
:1093800076E5F7FF5C8DF7FF4235F7FF28DDF6FF46
:109390000E85F6FFF42CF6FFDAD4F5FFC07CF5FF5E
:1093A000A624F5FF8CCCF4FF7274F4FF581CF4FF74
:1093B0003EC4F3FF246CF3FF0A14F3FFF0BBF2FF8B
:1093C000D663F2FFBC0BF2FFA2B3F1FF885BF1FFA3
:1093D0006E03F1FF54ABF0FF3A53F0FF20FBEFFFB9
:1093E00006A3EFFFEC4AEFFFD2F2EEFFB89AEEFFD2
:1093F0009E42EEFF84EAEDFF6A92EDFF503AEDFFE8
:1094000036E2ECFF1C8AECFF0232ECFFE8D9EBFFFE
:10941000CE81EBFFB429EBFF9AD1EAFF8079EAFF16
:109420006621EAFF4CC9E9FF3271E9FF1819E9FF2B
:10943000FEC0E8FFE468E8FFCA10E8FFB0B8E7FF45
:109440009660E7FF7C08E7FF62B0E6FF4858E6FF5A
:109450002E00E6FF14A8E5FFFA4FE5FFE0F7E4FF72
:10946000C69FE4FFAC47E4FF92EFE3FF7897E3FF8A
:109470005E3FE3FF44E7E2FF2A8FE2FF1037E2FF9F
:10948000F6DEE1FFDC86E1FFC22EE1FFA8D6E0FFB9
:109490008E7EE0FF7426E0FF5ACEDFFF4076DFFFCE
:1094A000261EDFFF0CC6DEFFF26DDEFFD815DEFFE5
:1094B000BEBDDDFFA465DDFF8A0DDDFF70B5DCFFFD
:1094C000565DDCFF3C05DCFF22ADDBFF0855DBFF12
:1094D000EEFCDAFFD4A4DAFFBA4CDAFFA0F4D9FF2D
:1094E000869CD9FF6C44D9FF52ECD8FF3894D8FF42
:1094F0001E3CD8FF04E4D7FFEA8BD7FFD033D7FF59
:10950000B6DBD6FF9C83D6FF822BD6FF68D3D5FF70
:109510004E7BD5FF3423D5FF1ACBD4FF1DFFFFFFB1
:109520001FFFFFFF21FFFFFF23FFFFFF24FFFFFFC0
:1095300026FFFFFF28FFFFFF2AFFFFFF2BFFFFFF94
:109540002DFFFFFF2FFFFFFF31FFFFFF32FFFFFF68
:1095500034FFFFFF36FFFFFF38FFFFFF3AFFFFFF3B
:109560003BFFFFFF3DFFFFFF3FFFFFFF41FFFFFF0F
:1095700042FFFFFF44FFFFFF46FFFFFF48FFFFFFE3
:1095800049FFFFFF4BFFFFFF4DFFFFFF4FFFFFFFB7
:1095900051FFFFFF52FFFFFF54FFFFFF56FFFFFF8A
:1095A00058FFFFFF59FFFFFF5BFFFFFF5DFFFFFF5E
:1095B0005FFFFFFF61FFFFFF62FFFFFF64FFFFFF31
:1095C00066FFFFFF68FFFFFF69FFFFFF6BFFFFFF05
:1095D0006DFFFFFF6FFFFFFF70FFFFFF72FFFFFFD9
:1095E00074FFFFFF76FFFFFF78FFFFFF79FFFFFFAC
:1095F0007BFFFFFF7DFFFFFF7FFFFFFF80FFFFFF80
:1096000082FFFFFF84FFFFFF86FFFFFF88FFFFFF52
:1096100089FFFFFF8BFFFFFF8DFFFFFF8FFFFFFF26
:1096200090FFFFFF92FFFFFF94FFFFFF96FFFFFFFA
:1096300097FFFFFF99FFFFFF9BFFFFFF9DFFFFFFCE
:109640009FFFFFFFA0FFFFFFA2FFFFFFA4FFFFFFA1
:10965000A6FFFFFFA7FFFFFFA9FFFFFFABFFFFFF75
:10966000ADFFFFFFAEFFFFFFB0FFFFFFB2FFFFFF49
:10967000B4FFFFFFB6FFFFFFB7FFFFFFB9FFFFFF1C
:10968000BBFFFFFFBDFFFFFFBEFFFFFFC0FFFFFFF0
:10969000C2FFFFFFC4FFFFFFC6FFFFFFC7FFFFFFC3
:1096A000C9FFFFFFCBFFFFFFCDFFFFFFCEFFFFFF97
:1096B000D0FFFFFFD2FFFFFFD4FFFFFFD5FFFFFF6B
:1096C000D7FFFFFFD9FFFFFFDBFFFFFFDDFFFFFF3E
:1096D000DEFFFFFFE0FFFFFFE2FFFFFFE4FFFFFF12
:1096E000E5FFFFFFE7FFFFFFE9FFFFFFEBFFFFFFE6
:1096F000EDFFFFFFEEFFFFFFF0FFFFFFF2FFFFFFB9
:10970000F4FFFFFFF5FFFFFFF7FFFFFFF9FFFFFF8C
:10971000FBFFFFFFFCFFFFFFFEFFFFFF000000005D
:109720000200000004000000050000000700000027
:10973000090000000B0000000C0000000E000000FB
:1097400010000000120000001300000015000000CF
:1097500017000000190000001B0000001C000000A2
:109760001E00000020000000220000002300000076
:109770002500000027000000290000002B00000049
:109780002C0000002E00000030000000320000001D
:1097900033000000350000003700000039000000F1
:1097A0003A0000003C0000003E00000040000000C5
:1097B0004200000043000000450000004700000098
:1097C000490000004A0000004C0000004E0000006C
:1097D000500000005200000053000000550000003F
:1097E00057000000590000005A0000005C00000013
:1097F0005E000000600000006100000063000000E7
:109800006500000067000000690000006A000000B9
:109810006C0000006E00000070000000710000008D
:109820007300000075000000770000007800000061
:109830007A0000007C0000007E0000008000000034
:109840008100000083000000850000008700000008
:10985000880000008A0000008C0000008E000000DC
:1098600090000000910000009300000095000000AF
:1098700097000000980000009A0000009C00000083
:109880009E0000009F000000A1000000A300000057
:10989000A5000000A7000000A8000000AA0000002A
:1098A000AC000000AE000000AF000000B1000000FE
:1098B000B3000000B5000000B7000000B8000000D1
:1098C000BA000000BC000000BE000000BF000000A5
:1098D000C1000000C3000000C5000000C600000079
:1098E000C8000000CA000000CC000000CE0000004C
:1098F000CF000000D1000000D3000000D500000020
:10990000D6000000D8000000DA000000DC000000F3
:10991000DD000000DF000000E100000000000000AA
:109920000000000000000000000000000000000037
:109930000000000000000000000000000000000027
:109940000000000000000000000000000000000017
:109950000000000000000000000000000000000007
:1099600000000000000000000000000000000000F7
:1099700000000000000000000000000000000000E7
:1099800000000000000000000000000000000000D7
:1099900000000000000000000000000000000000C7
:1099A00000000000000000000000000000000000B7
:1099B00000000000000000000000000000000000A7
:1099C0000000000000000000000000000000000097
:1099D0000000000000000000000000000000000087
:1099E0000000000000000000000000000000000077
:1099F0000000000000000000000000000000000067
:109A00000000000000000000000000000000000056
:109A10000000000000000000000000000001020340
:109A20000405060708090A0B0C0D0E0F101112137E
:109A30001415161718191A1B1C1D1E1F202122236E
:109A40002425262728292A2B2C2D2E2F303132335E
:109A50003435363738393A3B3C3D3E3F404142434E
:109A60004445464748494A4B4C4D4E4F505152533E
:109A70005455565758595A5B5C5D5E5F606162632E
:109A80006465666768696A6B6C6D6E6F707172731E
:109A90007475767778797A7B7C7D7E7F808182830E
:109AA0008485868788898A8B8C8D8E8F90919293FE
:109AB0009495969798999A9B9C9D9E9FA0A1A2A3EE
:109AC000A4A5A6A7A8A9AAABACADAEAFB0B1B2B3DE
:109AD000B4B5B6B7B8B9BABBBCBDBEBFC0C1C2C3CE
:109AE000C4C5C6C7C8C9CACBCCCDCECFD0D1D2D3BE
:109AF000D4D5D6D7D8D9DADBDCDDDEDFE0E1E2E3AE
:109B0000E4E5E6E7E8E9EAEBECEDEEEFF0F1F2F39D
:109B1000F4F5F6F7F8F9FAFBFCFDFEFFFFFFFFFF97
:109B2000FFFFFFFFFFFFFFFFFFFFFFFFFFFFFFFF45
:109B3000FFFFFFFFFFFFFFFFFFFFFFFFFFFFFFFF35
:109B4000FFFFFFFFFFFFFFFFFFFFFFFFFFFFFFFF25
:109B5000FFFFFFFFFFFFFFFFFFFFFFFFFFFFFFFF15
:109B6000FFFFFFFFFFFFFFFFFFFFFFFFFFFFFFFF05
:109B7000FFFFFFFFFFFFFFFFFFFFFFFFFFFFFFFFF5
:109B8000FFFFFFFFFFFFFFFFFFFFFFFFFFFFFFFFE5
:109B9000FFFFFFFFFFFFFFFFFFFFFFFFFFFFFFFFD5
:109BA000FFFFFFFFFFFFFFFFFFFFFFFFFFFFFFFFC5
:109BB000FFFFFFFFFFFFFFFFFFFFFFFFFFFFFFFFB5
:109BC000FFFFFFFFFFFFFFFFFFFFFFFFFFFFFFFFA5
:109BD000FFFFFFFFFFFFFFFFFFFFFFFFFFFFFFFF95
:109BE000FFFFFFFFFFFFFFFFFFFFFFFFFFFFFFFF85
:109BF000FFFFFFFFFFFFFFFFFFFFFFFFFFFFFFFF75
:109C0000FFFFFFFFFFFFFFFFFFFFFFFFFFFFFFFF64
:109C1000FFFFFFFFFFFFFFFFFFFFFFFF5DD0039090
:109C200095E3049091DE0590D5B00590000000000A
:109C30000000000014140101409C0090100A0D0067
:109C4000A000FF004C9C0090CCAC009005050100EA
:109C500094AC00900505010080AC00900A0A020057
:109C600058AC00900A0A020030AC00900A0A0200C8
:109C700008AC00900A0A0200E0AB00900404010066
:109C8000CCAB00900A0A0200A4AB009006060100CB
:109C900090AB00900D0D020068AB0090070701002B
:109CA00054AB00900A0A02002CAB00900B0B020090
:109CB00004AB009006060100F0AA00900D0D020012
:109CC000C8AA00900A0A0200A0AA00900707010093
:109CD0008CAA00900A0A020064AA009006060100FD
:109CE00050AA0090060601003CAA0090060601005A
:109CF00028AA00900A0A020000AA00900A0A02009C
:109D0000D8A9009005050100C4A90090060601002D
:109D1000B0A90090060601009CA900900707010069
:109D200088A900900A0A020060A900900F0F0200A3
:109D300038A900900F0F020010A900900F0F020029
:109D4000E8A800900B0B0200C0A800900D0D0200C7
:109D500098A800900D0D020070A800900D0D020053
:109D600048A800900D0D020020A800900D0D0200E3
:109D7000F8A700900D0D0200D0A70090121203006A
:109D800094A700900D0D02006CA700900C0C02002F
:109D900044A700900C0C02001CA700900C0C0200C1
:109DA000F4A600900C0C0200CCA600900505010062
:109DB000B8A6009005050100A4A6009005050100C5
:109DC00090A60090050501007CA600900D0D0200F4
:109DD00054A600900D0D02002CA600900E0E02005D
:109DE00004A600900E0E0200DCA500900E0E0200EC
:109DF000B4A500900E0E02008CA500900E0E02007D
:109E000064A500900B0B02003CA500900E0E020012
:109E100014A500900D0D0200ECA400900D0D0200A1
:109E2000C4A400900D0D02009CA400900D0D020032
:109E300074A400900C0C02004CA400900C0C0200C6
:109E400024A400900C0C0200FCA300900A0A02005B
:109E5000D4A300900A0A0200ACA300900A0A0200F0
:109E600084A300900A0A02005CA300900A0A020080
:109E700034A300900A0A02000CA300901010020004
:109E8000E4A200900A0A0200BCA200900A0A0200A2
:109E900094A200900A0A02006CA200900A0A020032
:109EA00044A200900A0A02001CA2009005050100CD
:109EB00008A2009005050100F4A10090050501002D
:109EC000E0A1009005050100CCA100900B0B020061
:109ED000A4A100900B0B02007CA100900B0B0200D0
:109EE00054A100900B0B02002CA100900B0B020060
:109EF00004A100900B0B0200DCA000900B0B0200F1
:109F0000B4A000900A0A02008CA000900B0B020083
:109F100064A000900B0B02003CA000900B0B020011
:109F200014A000900B0B0200EC9F00900B0B0200A2
:109F3000C49F00900A0A02009C9F00900B0B020035
:109F4000749F00900A0A02004C9F009000000000DD
:109F50000000198019800000E0C0E0C071C071C02D
:109F600031803B801B801F001F000E000E001C0074
:109F70007C0078000000000000007000700070009D
:109F800077007F807BC071C071C071C071C07BC021
:109F90007F8077007000700070007000000000008B
:109FA000070006000C000000E0C0E0C071C071C0F6
:109FB00031803B801B801F001F000E000E001C0024
:109FC0007C0078000000000000001980198000006B
:109FD00071C071C071C071C071C071C071C073C0F7
:109FE0007FC03DC000000000000000000000000035
:109FF00000000E001B00000071C071C071C071C074
:10A0000071C071C071C073C07FC03DC0000000004E
:10A010000000000000000000070006000C00000027
:10A0200071C071C071C071C071C071C071C073C0A6
:10A030007FC03DC0000000000000000000000000E4
:10A040001C000C000600000071C071C071C071C01E
:10A0500071C071C071C073C07FC03DC000000000FE
:10A060000000000000000000000000000000008070
:10A070001EC03F803B8073C077C07DC079C03B80ED
:10A080003F806F0020000000000000000000000082
:10A09000000000001C001C001C000000FF80FF806E
:10A0A000FF8000001C001C001C00000000000000DD
:10A0B000000000000000000000001980198000006E
:10A0C0001F003F807BC071C071C071C071C07BC078
:10A0D0003F801F00000000000000000000000000A2
:10A0E00000001C80138000001F003F807BC071C0F7
:10A0F00071C071C071C07BC03F801F0000000000B4
:10A10000000000000000000000000E001B00000026
:10A110001F003F807BC071C071C071C071C07BC027
:10A120003F801F0000000000000000000000000051
:10A13000070006000C0000001F003F807BC071C0BC
:10A1400071C071C071C07BC03F801F000000000063
:10A1500000000000000000000E00060003000000E8
:10A160001F003F807BC071C071C071C071C07BC0D7
:10A170003F801F0000000000000000000000000001
:10A1800000001C801380000077807FC079C071C000
:10A1900071C071C071C071C071C071C00000000099
:10A1A000000000000000000000000E800700098091
:10A1B0000F803FC03BC071C071C071C071C03B8097
:10A1C0003F801F000000000000000000000000D8D9
:10A1D000D800707070707070707070700000000047
:10A1E00000000070D80070707070707070707070C7
:10A1F00000000000000038306000707070707070F7
:10A2000070707070000000000000E060300070703E
:10A2100070707070707070700000000000000000BE
:10A2200000001980198000001F003F8071C071C0BC
:10A230007FC07FC0700071C03F801F000000000021
:10A24000000000000000000000000E001B000000E5
:10A250001F003F8071C071C07FC07FC0700071C09F
:10A260003F801F0000000000000000000000000010
:10A27000070006000C0000001F003F8071C071C085
:10A280007FC07FC0700071C03F801F0000000000D1
:10A2900000000000000000000E00060003000000A7
:10A2A0001F003F8071C071C07FC07FC0700071C04F
:10A2B0003F801F00000000000000000000000000C0
:10A2C00000000000000000001E003F007B807100C5
:10A2D0007000700071007B803F001E001E000600B1
:10A2E0003C00000000000000000000000000000032
:10A2F0001E783FFC638E078E0FFE3BFE738073CE8D
:10A300007FFC3C78000000000000000000000C0012
:10A31000120012000C0000001F003F8063800780C5
:10A320001F803B80738073807F803DC000000000F1
:10A3300000000000000000000000330033000000B7
:10A340001F003F80638007801F803B807380738085
:10A350007F803DC000000000000000000000000001
:10A3600000003900270000001F003F806380078045
:10A370001F803B80738073807F803DC000000000A1
:10A38000000000000000000000000E001B000000A4
:10A390001F003F80638007801F803B807380738035
:10A3A0007F803DC0000000000000000000000000B1
:10A3B000070006000C0000001F003F80638007803C
:10A3C0001F803B80738073807F803DC00000000051
:10A3D00000000000000000001C000C00060000004F
:10A3E0001F003F80638007801F803B8073807380E5
:10A3F0007F803DC000000000000000000000000061
:10A4000000001F003F8073807380770077007780A3
:10A4100073C071C070E074E07FE0778000000000DE
:10A4200000000000000000000000700070007F804D
:10A430007FC07FE070E070E070E07FE07FC07F80F1
:10A4400070007000000000000000000003800300A6
:10A4500006007070707038E01DC01DC00F800F8046
:10A4600007000700070007000700070000000000C2
:10A47000000000000CC00CC00000707070707070A4
:10A4800070707070707070707070707078F03FE005
:10A490003FE00F80000000000000000007000D807A
:10A4A000000070707070707070707070707070708C
:10A4B0007070707078F03FE03FE00F8000000000A7
:10A4C0000000000003800300060070707070707060
:10A4D00070707070707070707070707078F03FE0B5
:10A4E0003FE00F8000000000000000000E000600AA
:10A4F0000300707070707070707070707070707039
:10A500007070707078F03FE03FE00F800000000056
:10A51000000000000000000000080FCC1FF83FF012
:10A52000387870F871B8733876387C3878703FF0C6
:10A530007FE0CFC0400000000000000000000000ED
:10A540000000000000000000210073803F001E009A
:10A550001E003F007380210000000000000000008A
:10A56000000000000CC00CC0000007801FE03FF09E
:10A5700038707038703870387038703838703FF014
:10A580001FE0078000000000000000000E4009C02E
:10A59000000007801FE03FF0387070387038703866
:10A5A0007038703838703FF01FE0078000000000FE
:10A5B00000000000038006C0000007801FE03FF09D
:10A5C00038707038703870387038703838703FF0C4
:10A5D0001FE007800000000000000000038003006F
:10A5E000060007801FE03FF0387070387038703810
:10A5F0007038703838703FF01FE0078000000000AE
:10A600000000000007000300018007801FE03FF00A
:10A6100038707038703870387038703838703FF073
:10A620001FE0078000000000000000000E4009C08D
:10A630000000707078707C707C707E7076707770BF
:10A64000737073F071F071F070F0707000000000C2
:10A65000000000000000000000007F807FE07FE03D
:10A6600070F07070FE70FE707070707070F07FE04F
:10A670007FE07F800000000000000000D8D800705C
:10A68000707070707070707070707070000000008A
:10A6900070D80070707070707070707070707070C2
:10A6A00000000000383060707070707070707070F2
:10A6B0007070707000000000E0703070707070702A
:10A6C00070707070707070700000000019801980D8
:10A6D00000007FE07FE07FE0700070007FE07FE0BF
:10A6E0007FE0700070007FE07FE07FE0000000000E
:10A6F0000000000007000D8000007FE07FE07FE0A9
:10A70000700070007FE07FE07FE0700070007FE00D
:10A710007FE07FE0000000000000000003800300F5
:10A7200006007FE07FE07FE0700070007FE07FE068
:10A730007FE0700070007FE07FE07FE000000000BD
:10A74000000000000E00060003007FE07FE07FE0D5
:10A75000700070007FE07FE07FE0700070007FE0BD
:10A760007FE07FE00000000000000000000000002B
:10A77000000007801FE03FE038F07060700070005C
:10A780007000706038F03FE01FE0078007800180B4
:10A790000F00000000000000000000000007FF8024
:10A7A0000FFF800EFF801CE0001CE00038FF8038A7
:10A7B000FF803FFF807FE0007FE000E0FF80E0FF60
:10A7C00080C0FF80000000000000000000000000CA
:10A7D0000300048004800F800F800F801DC01DC007
:10A7E0001DC038E03FE03FE07FF070707070E038EF
:10A7F00000000000000000000CC00CC000000F8032
:10A800000F800F801DC01DC01DC038E03FE03FE03D
:10A810007FF070707070E0380000000000000000F1
:10A820000E4009C000000F800F800F801DC01DC0AA
:10A830001DC038E03FE03FE07FF070707070E0389E
:10A84000000000000000000007000D8000000F80E5
:10A850000F800F801DC01DC01DC038E03FE03FE0ED
:10A860007FF070707070E0380000000000000000A1
:10A870000380030006000F800F800F801DC01DC0E5
:10A880001DC038E03FE03FE07FF070707070E0384E
:10A8900000000000000000000E00060003000F8012
:10A8A0000F800F801DC01DC01DC038E03FE03FE09D
:10A8B0007FF070707070E038000000000000000051
:10A8C0000000000000000000000000000E000E006C
:10A8D0000E0000000E000E001E003C00780070000C
:10A8E00071C073C03F801F00000000000000703086
:10A8F000D860186030C01980D980730C031C061C06
:10A900000C2C0C4C187E180C0000000000000000FD
:10A9100000000000000030607060F0C031C0318085
:10A9200033003338066C060C0C1C18381870307C59
:10A93000000000000000000000000000000018609F
:10A94000386078C018C0198019801B0C031C061CC5
:10A95000062C0C4C0C7E180C0000000000000000BF
:10A960000000000000000000000000000000660081
:10A9700033003B801DC01DC03B80330066000000DB
:10A9800000000000000000000000003C66666666F3
:10A99000663C0000000000000000000000000030E5
:10A9A00070F0303030300000000000000000000087
:10A9B0000000000000000000000000000000000097
:10A9C0007818F000000000000000000070707000B7
:10A9D00000000000000000000000000000003FC078
:10A9E0007FC0FD80FD80FD807D803D800D800D80DD
:10A9F0000D800D800D800D800D800D800D8000007C
:10AA00000000000000000000000000007380738060
:10AA10007380738073807380738073807F807F8086
:10AA200070007000700070000000001C1830000002
:10AA300000000000000000000000000000000070A6
:10AA4000D8183018D8700000000000000000000086
:10AA500000000070D8183870E0F800000000000016
:10AA6000000000000000000000000E000E000E00BC
:10AA70007FC07FC07FC00E000E000E0000007FC0B0
:10AA80007FC07FC000000000000000000000003810
:10AA900044444438000000000000000000000000B2
:10AAA000FFC0FFC000000000000000000000000028
:10AAB0000000000000000000000000000000000096
:10AAC00000000000000000000000000000000F80F7
:10AAD000306060304F10888888888F08890888889F
:10AAE0004890603030600F800000000000000000DF
:10AAF000000000000000000000007C7C7C000000E2
:10AB00000000000000000000000000000000000045
:10AB10007FC07FC07FC001C001C001C001C0000074
:10AB20000000000000000000000000000000000025
:10AB300000000000000000000000198033007700D2
:10AB4000EE00EE00770033001980000000000000E6
:10AB50000000000000000078CC0C7CCCCC7C000015
:10AB600000000000000000000000000000000F8056
:10AB70003060603047908CC89808980898088CC856
:10AB80004790603030600F8000000000000000003F
:10AB9000000000CCCC00000000000000000000001D
:10ABA000000000000000000000003C007E00630088
:10ABB000600038007E00CF00C380E18071803F00DC
:10ABC0001E000700630073003F001E0000000060CD
:10ABD0006060606060600000006060606060606095
:10ABE000000000000000E0C071C071C03B803B80ED
:10ABF0001F007FC07FC00E007FC07FC00E000E0010
:10AC00000000000000000000000000000000000044
:10AC1000000021007F80FFC07380618061807380AD
:10AC2000FFC07F8021000000000000000000000045
:10AC30000000000000001E003F0073807380700061
:10AC4000FE00FE00380038007000FC80FFC0478026
:10AC50000000000000000000000000000000008074
:10AC6000010001001F003F807BC07200740074006F
:10AC700075C079C03F801F00100010001000200038
:10AC80000000000000007070700020207070707074
:10AC900070707070000000000000000000000000F4
:10ACA00000000000000000005DD0039095E30490D8
:10ACB00091DE0590D5B00590000000000000000076
:10ACC00014140101CCAC0090100A0D0020007E008D
:10ACD000D8AC00900000000005050100DCBC00902D
:10ACE00005050100C8BC009009090200A0BC009045
:10ACF0000A0A020078BC00900A0A020050BC0090C8
:10AD00001111030014BC00900D0D0200ECBB00906B
:10AD100004040100D8BB009006060100C4BB0090EB
:10AD200006060100B0BB0090070701009CBB009025
:10AD30000B0B020074BB00900505010060BB009086
:10AD4000060601004CBB00900505010038BB0090D1
:10AD50000505010024BB00900A0A0200FCBA00901D
:10AD60000A0A0200D4BA00900A0A0200ACBA0090A3
:10AD70000A0A020084BA00900A0A02005CBA009033
:10AD80000A0A020034BA00900A0A02000CBA0090C3
:10AD90000A0A0200E4B900900A0A0200BCB9009055
:10ADA0000A0A020094B900900707010080B90090D8
:10ADB000070701006CB900900B0B020044B900902A
:10ADC0000B0B02001CB900900B0B0200F4B80090B2
:10ADD0000B0B0200CCB800901212030090B8009048
:10ADE0000D0D020068B800900D0D020040B80090F3
:10ADF0000D0D020018B800900D0D0200F0B7009084
:10AE00000C0C0200C8B700900B0B0200A0B700901A
:10AE10000E0E020078B700900D0D020050B70090A2
:10AE2000050501003CB700900A0A020014B7009023
:10AE30000D0D0200ECB600900B0B0200C4B60090A2
:10AE40000F0F02009CB600900D0D020074B600902A
:10AE50000E0E02004CB600900C0C020024B60090BE
:10AE60000E0E0200FCB500900D0D0200D4B500904E
:10AE70000C0C0200ACB500900B0B020084B50090E6
:10AE80000D0D02005CB500900D0D020034B5009070
:10AE900011110300F8B400900C0C0200D0B4009023
:10AEA0000D0D0200A8B400900A0A020080B40090C0
:10AEB000060601006CB400900505010058B400902E
:10AEC0000606010044B400900B0B02001CB4009075
:10AED0000A0A0200F4B3009006060100E0B30090F5
:10AEE0000A0A0200B8B300900B0B020090B3009066
:10AEF0000A0A020068B300900B0B020040B30090F6
:10AF00000B0B020018B300900606010004B300907A
:10AF10000B0B0200DCB200900B0B0200B4B20090ED
:10AF200005050100A0B20090050501008CB200905B
:10AF30000A0A020064B200900505010050B20090B8
:10AF40001111030014B200900B0B0200ECB1009041
:10AF50000B0B0200C4B100900B0B02009CB10090DF
:10AF60000B0B020074B100900707010060B1009064
:10AF70000A0A020038B100900606010024B10090D0
:10AF80000B0B0200FCB000900B0B0200D4B0009041
:10AF90000F0F0200ACB000900B0B020084B00090C9
:10AFA0000B0B02005CB000900909020034B0009065
:10AFB0000707010020B00090040401000CB00090CD
:10AFC00007070100F8AF00900B0B0200D0AF009014
:10AFD00000000000000000000000000000007840B9
:10AFE000FFC0FFC0878000000000000000000000DC
:10AFF0000000000000000000000000E0F0303030F1
:10B000003030381C1C3830303030F0E00000006048
:10B010006060606060606060606060606060606030
:10B020000000000E1E1818181818387070381818FC
:10B0300018181E0E000000000000000000000000B4
:10B040007F007F0007000E001C001C00380070000D
:10B050007F007F00000000000000000000000000F2
:10B060000000000000000000E0E0E0E071C071C0FE
:10B0700031803B801B801F001F000E000E001C0053
:10B080007C007800000000000000000000000000CC
:10B0900071C03B803B801F000E000E001F003B80F4
:10B0A0003B8071C0000000000000000000000000B4
:10B0B0000000000000000000E38EE38E638C77DC6C
:10B0C00076DC36D83EF83C781C701C70000000001E
:10B0D0000000000000000000000000000000000070
:10B0E00071C071C071C03B803B801B001F001F00FE
:10B0F0000E000E0000000000000000000000000034
:10B10000000000000000000071C071C071C071C07B
:10B1100071C071C071C073C07FC03DC0000000002D
:10B1200000000000000000307070FCFC7070707057
:10B1300070707C3C00000000000000000000000077
:10B14000000000003F007F80738078003E001F00F9
:10B15000078073807F803F00000000000000000037
:10B16000000000000000767E787070707070707063
:10B1700000000000000000000000000000000000CF
:10B180001DC03FC07BC071C071C071C071C07BC0A9
:10B190003FC01DC001C001C001C001C000000000CF
:10B1A000000000000000000077007F807BC071C0BD
:10B1B00071C071C071C07BC07F807700700070006B
:10B1C000700070000000000000000000000000009F
:10B1D0001F003F807BC071C071C071C071C07BC057
:10B1E0003F801F0000000000000000000000000081
:10B1F000000000000000000077807FC079C071C0AF
:10B2000071C071C071C071C071C071C00000000018
:10B21000000000000000000000000000000000002E
:10B22000000000000000779E007FFF0079E70071BA
:10B23000C70071C70071C70071C70071C70071C72F
:10B240000071C700000000000000000000000000C6
:10B25000000000707070707070707070707070703E
:10B26000000000000000000000007000700070008E
:10B2700071C0738077007E007E007F00770073804E
:10B28000738071C00000000000000000000000702A
:10B290007000707070707070707070707070F0E02E
:10B2A000000000707000707070707070707070705E
:10B2B000000000000000000000007000700070003E
:10B2C00077807FC079C071C071C071C071C071C01A
:10B2D00071C071C00000000000000000000000000C
:10B2E00000000000000000001DC03FC07BC071C016
:10B2F00071C071C071C07BC03FC01DC001C071C0B2
:10B300007F803F000000003C7C70FCFC707070701F
:10B31000707070700000000000000000000000006D
:10B32000000000001F003F8071C071C07FC07FC05F
:10B33000700071C03F801F0000000000000000008E
:10B3400000000000000001C001C001C01DC03FC0DE
:10B350007BC071C071C071C071C07BC03FC01DC0D7
:10B3600000000000000000000000000000000000DD
:10B37000000000001E003F007B8071007000700024
:10B3800071007B803F001E000000000000000000F4
:10B3900000000000000070007000700077007F80E7
:10B3A0007BC071C071C071C071C07BC07F807700ED
:10B3B000000000000000000000000000000000008D
:10B3C000000000001F003F80638007801F803B80DB
:10B3D000738073807F803DC000000000000000008B
:10B3E000000000E0603000000000000000000000ED
:10B3F000000000000000000000000000000000004D
:10B40000000000000000000000000000000000003C
:10B410000000000000000000FFC0FFC000000000AE
:10B4200000000E000E001F001B003B80318071C029
:10B43000000000000000000000000000000000000C
:10B4400000000000000000F8F8F8383838383838C4
:10B450003838383838F8F8F8000000C0C06060604C
:10B460006070303030301818000000000000007CA0
:10B470007C7C70707070707070707070707C7C7C90
:10B480000000000000007FC07FC07FC00380070075
:10B490000E001E001C0038007000FFC0FFC0FFC07F
:10B4A00000000000000000000000000000007070BC
:10B4B000707038E01DC01DC00F800F8007000700AE
:10B4C0000700070007000700000000000000000060
:10B4D00000000000000070E070E039C019801F809B
:10B4E0000F000F000F001F80198039C070E070E05E
:10B4F000000000000000000000000000000000004C
:10B5000000E1C380E1C380E3E380736700736700F9
:10B510007777007777007637007637003E3E003E3B
:10B520003E003C1E003C1E00000000000000000029
:10B5300000000000000000000000E038E0387070FB
:10B540007070707038E038E01DC01DC01DC00F80E5
:10B550000F800F80000000000000000000000000CD
:10B5600000007070707070707070707070707070BB
:10B570007070707078F03FE03FE00F8000000000D6
:10B5800000000000000000000000FFE0FFE0FFE01E
:10B590000E000E000E000E000E000E000E000E003B
:10B5A0000E000E000000000000000000000000007F
:10B5B00000001F803FC07FE070E070007F003FC050
:10B5C0000FE000E070E07FE03FC01F80000000005F
:10B5D000000000000000000000007FC07FE07FF05E
:10B5E000707070707FF07FE07F8073C071E070E0FA
:10B5F00070F0707800000000000000000000000003
:10B6000000000FC01FE03FF038707038703870389D
:10B61000713873F839F83FF01FF00FB800100000D0
:10B62000000000000000000000007F807FC07FE07D
:10B6300070E070E07FE07FC07F807000700070007D
:10B64000700070000000000000000000000000001A
:10B65000000007801FE03FF0387070387038703895
:10B660007038703838703FF01FE00780000000002D
:10B6700000000000000000000000707078707C7016
:10B680007C707E7076707770737073F071F071F00B
:10B6900070F070700000000000000000000000006A
:10B6A0000000783C783C7C7C7C7C7C7C76DC76DCA6
:10B6B00076DC76DC739C739C739C711C000000002C
:10B6C000000000000000000000007000700070002A
:10B6D00070007000700070007000700070007FC01B
:10B6E0007FC07FC0000000000000000000000000DC
:10B6F000000070F071E071C0738077007F007F8080
:10B700007B8071C071C070E07070707000000000CC
:10B7100000000000000000000000038003800380A0
:10B7200003800380038003800380E380E380FF8045
:10B730007F003E00000000000000000000000070DC
:10B7400070707070707070707070707000000000B9
:10B750000000000000007070707070707070707089
:10B760007FF07FF07FF0707070707070707070702C
:10B77000000000000000000000000000000007C002
:10B780001FF03FF038787030700071F871F871F880
:10B7900038383FF81FF007C000000000000000002C
:10B7A0000000000000007FC07FC07FC070007000FC
:10B7B0007F807F807F80700070007000700070005C
:10B7C00000000000000000000000000000007FE01A
:10B7D0007FE07FE0700070007FE07FE07FE070003E
:10B7E00070007FE07FE07FE00000000000000000CC
:10B7F0000000000000007F807FE07FE070F070704C
:10B80000707070707070707070F07FE07FE07F809B
:10B8100000000000000000000000000000000780A1
:10B820001FE03FE038F070607000700070007060E2
:10B8300038F03FE01FE0078000000000000000003B
:10B840000000000000007FC07FE07FF0707070702B
:10B850007FE07FC07FE0707070707FF07FE07FC01E
:10B8600000000000000000000000000000000F8049
:10B870000F800F801DC01DC01DC038E03FE03FE0BD
:10B880007FF070707070E038000000000000000071
:10B8900000000000000000000001F80007FE001E8C
:10B8A0000F0019DB0033FB803639806E39806C3134
:10B8B000806C31806C73006C770067FE0037B800D5
:10B8C0003801C01E07800FFF0003FC0000000000CD
:10B8D00000001F003F8079C071C003C007800F00C7
:10B8E0000E000E0000000E000E000E000000000012
:10B8F0000000000000000000000000000000400008
:10B9000070007E001F8003C003C01F807E00700097
:10B9100040000000000000000000000000000000E7
:10B9200000000000000000007FC07FC07FC000005A
:10B9300000007FC07FC07FC000000000000000004A
:10B9400000000000000000000000000000000040B7
:10B9500001C00FC03F00780078003F000FC001C059
:10B960000040000000000000000000000000000097
:10B970000000383838000000003838380818300027
:10B980000000000000003838380000000038383867
:10B99000000000000000000000001E003F007300D7
:10B9A00073807380738073803F801F800380730077
:10B9B0003F001E000000000000000000000000002A
:10B9C00000001E003F007380738073803F001E00E4
:10B9D00033007380738073803F001E0000000000FE
:10B9E000000000000000000000007F807F800380D6
:10B9F000070006000E000C001C001C003800380078
:10BA000038003800000000000000000000000000C6
:10BA100000001F003F80338070007E007F00738035
:10BA200073807380738033803F001E00000000002D
:10BA3000000000000000000000001F001F00380090
:10BA400030003E003F0073800380038003807380DA
:10BA50003F001E0000000000000000000000000089
:10BA6000000007000F000F001F00370037006700BD
:10BA7000C700FFC0FFC0070007000700000000006C
:10BA8000000000000000000000001E003F00738066
:10BA9000738003800F000F00038003807380738026
:10BAA0003F001E0000000000000000000000000039
:10BAB00000001E003F0073807380038007000700B2
:10BAC0000E001C001C0038007F807F8000000000FA
:10BAD0000000000000000000000006000E003E0014
:10BAE0007E006E004E000E000E000E000E000E00D6
:10BAF0000E000E000000000000000000000000002A
:10BB000000001E003F0033007380738073807380D9
:10BB100073807380738033003F001E0000000000BC
:10BB200000000000000000181830303030706060F5
:10BB30006060C0C0000000000000000000000000C5
:10BB400000000000007070700000000000000000A5
:10BB50000000000000007C7C7C0000000000000071
:10BB60000000000000000000000000000070707085
:10BB700010306000000000000000000000000E0017
:10BB80000E000E007FC07FC07FC00E000E000E00B2
:10BB90000000000000000000000000000000003075
:10BBA000B4FC3078CC000000000000000000000071
:10BBB000000000607070303838383838383838381D
:10BBC000307070600000001838383070707070701D
:10BBD00070707070303038180000007070707070C5
:10BBE0000000000000000000000000000000000055
:10BBF00000000F003FC039C039C01D800F001F007A
:10BC00003FB073F071E071F03FF81F1000000000CA
:10BC1000000000000000000000000000003C1800D0
:10BC20006630006630006660006660003CC0000060
:10BC3000C000018000019E0003330003330006337F
:10BC4000000633000C1E0000000000000000000091
:10BC50000000000008003E007F00EB80E800E800E4
:10BC60007C003F000F800B80EB80EB807F003E006C
:10BC700008000800000000000000000000000CC0E8
:10BC80000CC01980FFC0FFC019803B803300FFC08B
:10BC9000FFC03300660066000000000000000000E6
:10BCA0000000000000007700770077007700770041
:10BCB0000000000000000000000000000000000084
:10BCC0000000000000000000000000707070707044
:10BCD00070702020007070700000000000000000F4
:10BCE0000000000000000000000000000000000054
:10BCF00047F288432DE9F04FC358AFB00990002BAD
:10BD000040F02F8247F20943C35C002B00F05282BF
:10BD100000F0E4FF002840F0668247F22043099AD1
:10BD2000D358099D47F20841012047F288426854E0
:10BD3000AB50099B03F5E9442368002B00F0C08752
:10BD4000079347F27443099CE05801F053F90D90B2
:10BD5000002800F04F8247F21843E358002B40F3CD
:10BD6000468247F2184301460020E31808900B93DF
:10BD70006D4B0A93034601EBC3110A9B80220EA868
:10BD80001B6898470DF1480E19E03EF9103C0EF182
:10BD9000100E9B001BB22EF8203C2EF81E3C2EF8F5
:10BDA0001C3C2EF81A3C2EF8183C2EF8163C2EF8A7
:10BDB000143C2EF8123C32AB734500F0AC803EF9D7
:10BDC0000E0C3EF90C5C3EF9062C3EF90A1C40EACA
:10BDD0000503564F02EB000A56183EF9089C0B4328
:10BDE0003EF9048C07FB06F63EF902CC49EA030350
:10BDF00005EB080402920CEB0007134301964CF28A
:10BE0000DF4241F2511648EA030318FB02FB06FB2E
:10BE100004F441F67E020CEB01065CEA0303444B9A
:10BE200005FB0245434A5C44009506EB0A0502FB0C
:10BE300007F742F2A15202FB05F503FB06563E4B03
:10BE400003FB0A55A1D03EF910BCBB19019A2F443F
:10BE50000EF1100E02EB050A0BEB09051644009AD1
:10BE60006D03C9EB0B0B02EB0508AD1A43F20B0295
:10BE70004FEA4B3B10FB027740F68E1204EB0B09A6
:10BE8000C4EB0B041CFB023C44F2B313BDF80820C6
:10BE900008EB0700C7EB080712FB03AB46F254237D
:10BEA00000F5806007F5806711FB036605EB0C0168
:10BEB00004EB0B03CCEB050509EB0602CBEB040B03
:10BEC000C6EB090601F5806105F5806502F5806223
:10BED00006F5806603F580630BF5806BC012DB12FC
:10BEE000FF122EF8200CC9122EF81C3CED122EF871
:10BEF000127CD2122EF81A1CF6122EF8185C4FEA99
:10BF0000EB2B2EF81E2C2EF8146C32AB2EF816BC30
:10BF100073457FF454AF0DF1380EDDF81C80082313
:10BF2000F346C44602932AE0B4030020FDADFFFFB0
:10BF30003BC1FFFF33E3FFFF84F3FFFFBBF900309A
:10BF400010335B11803383F30803DBB28CF80030CD
:10BF50008CF808308CF810308CF818308CF82030C1
:10BF60008CF828308CF830308CF83830029B0BF18C
:10BF7000020B0CF1010C013B029300F0ED85BBF9C3
:10BF800010E0BBF92010BBF930904EEA0102BBF97A
:10BF90004050BBF9504049EA0202BBF96030BBF99E
:10BFA00070002A430094019022431A430243C5D0F3
:10BFB00002460446944F01EB03084A44BBF900A033
:10BFC0001646009A02EB0E0004EB0E02344607FB05
:10BFD00002F741F251120444049742F2A15702FBC6
:10BFE00008F841F67E0207FB04F40AEB0507C5EBEF
:10BFF0000A0501FB02814CF2DF420695834D13FBDB
:10C0000002F343F20B0205FB00407D03049F43440F
:10C01000039507EB000A009D7D4F1EFB02A24D44D5
:10C0200007FB06447B4E1746059206FB05F5039E6B
:10C0300001EB060A049E28440AEB070E2644069FDD
:10C040002C440EF5003E324646F25425039E4FEA3C
:10C05000AE4E4FEA4738711A0EF1800E40F68E163A
:10C06000BDF8047019FB05441FFA8EFE17FB06226B
:10C07000BDF800700FFA8EF544F2B31617FB0600F8
:10C0800015F47F4F03EB0807C3EB080340F032853C
:10C090005FFA8EFE059D8CF800E0C5EB0A0606F5FA
:10C0A0000036B6148036B6B235B215F47F4F40F084
:10C0B0004D85F6B23D198CF8386005F50035AD14A4
:10C0C0008035ADB22EB216F47F4F40F03985EDB217
:10C0D0003C1B8CF8085004F50034A4148034A4B23E
:10C0E00025B215F47F4F40F02585E5B21C188CF879
:10C0F000305004F50034A4148034A4B225B215F4F1
:10C100007F4F40F01185E4B21B1A8CF8104003F504
:10C1100000339B1480339BB218B210F47F4F40F071
:10C12000FD84D8B28B188CF8280003F500339B14DB
:10C1300080339BB218B210F47F4F40F0E984DBB239
:10C140008A1A8CF8183002F500339B1480339BB2A6
:10C150001AB212F47F4F40F0D584DBB28CF8203055
:10C1600004E747F208420146825C002A7FF4E1AD11
:10C1700047F20A428A5C042A0ED8DFE812F02D0248
:10C1800057029D0305004D00DA0740F1F98447F29C
:10C190009442012109988154099E47F28441013B50
:10C1A00047F28844725800203351013A72502FB040
:10C1B000BDE8F08F00F032FFA8B9099947F220449A
:10C1C00047F284420B598A589A423FF7AAAD084673
:10C1D0000EA901F00FFE30B99DF83830D92B02D1ED
:10C1E000099B1B599DE501202FB0BDE8F08F0DA8DC
:10C1F00002F012F8099C002147F2884347F20842F6
:10C20000E358A1542146B3E733E3FFFF84F3FFFF74
:10C210003BC1FFFFFDADFFFFD907B8D4099E47F230
:10C22000204147F28C427458B058E41A00F0E2FE04
:10C2300047F290430D900546F05800F0DBFE072CC6
:10C240000E9000F3318506F5E9431A6802EBC40A43
:10C25000631047F20C41099CDB00615800290491EE
:10C2600040F3AB8103F5827305F120010AF1400A26
:10C27000DFF8B4B3D318029100F120010193E84B29
:10C2800000910AF18006029A504603969DE822002A
:10C2900095F83C70403015F804EC20320BEB870722
:10C2A00010F880CC0BEB8E0E0435D7F8D04420313B
:10C2B000DEF8D068D7F8D070DEF8D0EC34441F44F4
:10C2C00003EB24449E4407EB0C0904EB0C08F444F4
:10C2D00099F8D89098F8D8809CF8D8C002F83F8C8C
:10C2E00002F8409C02F83ECC10F87FCC07EB0C091A
:10C2F00004EB0C08F44499F8D89098F8D8809CF88E
:10C30000D8C002F83C9C02F83B8C02F83ACC10F8FA
:10C3100078CC07EB0C0904EB0C08F44499F8D8909E
:10C3200098F8D8809CF8D8C001F8409C01F83F8C60
:10C3300001F83ECC10F877CC67446444E64497F8A3
:10C34000D87094F8D84001F83C7C01F83B4C9EF83A
:10C35000D84001F83A4C95F8397015F807EC0BEB1A
:10C36000870710F87ECC0BEB8E0ED7F8D044DEF8A2
:10C37000D068D7F8D070DEF8D0EC34441F4403EB1B
:10C3800024449E4407EB0C0904EB0C08F44499F890
:10C39000D89098F8D8809CF8D8C002F8378C02F86A
:10C3A000389C02F836CC10F87DCC07EB0C0904EB76
:10C3B0000C08F44499F8D89098F8D8809CF8D8C024
:10C3C00002F8349C02F8338C02F832CC10F876CCA8
:10C3D00007EB0C0904EB0C08F44499F8D89098F892
:10C3E000D8809CF8D8C001F8389C01F8378C01F847
:10C3F00036CC10F875CC67446444E64497F8D8709E
:10C4000001F8347C94F8D8709EF8D84001F8337C59
:10C4100001F8324C95F83A7015F806EC0BEB8707EB
:10C4200010F87CCC0BEB8E0ED7F8D044DEF8D06839
:10C43000D7F8D070DEF8D0EC34441F4403EB24442A
:10C440009E4407EB0C0904EB0C08F44499F8D890CF
:10C4500098F8D8809CF8D8C002F82F8C02F8309C4D
:10C4600002F82ECC10F87BCC07EB0C0904EB0C087F
:10C47000F44499F8D89098F8D8809CF8D8C002F87D
:10C480002C9C02F82B8C02F82ACC10F874CC07EB09
:10C490000C0904EB0C08F44499F8D89098F8D8806B
:10C4A0009CF8D8C001F8309C01F82F8C01F82ECCF4
:10C4B00010F873CC6444E644674497F8D8C094F805
:10C4C000D8709EF8D84001F82CCC01F82B7C01F8EC
:10C4D0002A4C95F83B7015F805EC0BEB870710F824
:10C4E0007ACC0BEB8E0ED7F8D044DEF8D068D7F8B4
:10C4F000D070DEF8D0EC34441F4403EB24449E4457
:10C5000007EB0C0904EB0C08F44499F8D89098F860
:10C51000D8809CF8D8C002F8278C02F8289C02F832
:10C5200026CC10F879CC07EB0C0904EB0C08F4448A
:10C5300099F8D89098F8D8809CF8D8C002F8249C34
:10C5400002F8238C02F822CC10F872CC07EB0C090D
:10C5500004EB0C08F44499F8D89098F8D8809CF82B
:10C56000D8C001F8289C01F8278C01F826CC10F8D7
:10C5700071CC6444E644674494F8D8C09EF8D8402F
:10C5800097F8D87001F8224C039C01F823CCA04204
:10C5900001F8247C7FF47CAE029A0AF5C07A40321E
:10C5A0000292009A40320092019A02F5C072019202
:10C5B000049A013A04927FF464AE0DA801F02CFEB7
:10C5C0000EA801F029FE099C47F29442002147F28F
:10C5D0008843A154E358DFE5099D47F2204147F223
:10C5E0008C426C58A858E41A00F004FD47F20C4144
:10C5F00005F5E94306460E906D581A68002D02EBCA
:10C60000C404DDDD074B1F46214630463B68082247
:10C610009847013D04F1400406F10806F4D1CFE744
:10C6200044990090B40300204C880090099E47F282
:10C63000204147F28C427158B058CD1A00F0DAFC14
:10C6400047F20C4206F5E9430E90B4581968002CE5
:10C6500001EBC501B4DD00F12002DFF858B2944BC4
:10C6600091F88070013C087802F120020BEB8707FB
:10C6700091F84060184401F1C001D7F8D0500BEB9D
:10C680008606054495F8D85002F8405CD7F8D07477
:10C69000D6F8D0583D4400EB254595F8D85002F81F
:10C6A0003F5CD6F8D05C284490F8D80002F83E0CE5
:10C6B00011F83F7C11F8BF0C0BEB870711F87F6C6A
:10C6C0001844D7F8D0500BEB8606054495F8D8509F
:10C6D00002F83C5CD7F8D074D6F8D0583D4400EB53
:10C6E000254595F8D85002F83B5CD6F8D05C284434
:10C6F00090F8D80002F83A0C11F83E7C11F8BE0C04
:10C700000BEB870711F87E6C1844D7F8D0500BEB71
:10C710008606054495F8D85002F8385CD7F8D074EE
:10C72000D6F8D0583D4400EB254595F8D85002F88E
:10C73000375CD6F8D05C284490F8D80002F8360C64
:10C7400011F83D7C11F8BD0C0BEB870711F87D6CDF
:10C750001844D7F8D0500BEB8606054495F8D8500E
:10C7600002F8345CD7F8D074D6F8D0583D4400EBCA
:10C77000254595F8D85002F8335CD6F8D05C2844AB
:10C7800090F8D80002F8320C11F83C7C11F8BC0C7F
:10C790000BEB870711F87C6C1844D7F8D0500BEBE3
:10C7A0008606054495F8D85002F8305CD7F8D07466
:10C7B000D6F8D0583D4400EB254595F8D85002F8FE
:10C7C0002F5CD6F8D05C284490F8D80002F82E0CE4
:10C7D00011F83B7C11F8BB0C0BEB870711F87B6C55
:10C7E0001844D7F8D0500BEB8606054495F8D8507E
:10C7F00002F82C5CD7F8D074D6F8D0583D4400EB42
:10C80000254595F8D85002F82B5CD6F8D05C284422
:10C8100090F8D80002F82A0C11F83A7C11F8BA0CFA
:10C820000BEB870711F87A6C1844D7F8D0500BEB54
:10C830008606054495F8D85002F8285CD7F8D074DD
:10C84000D6F8D0583D4400EB254595F8D85002F86D
:10C85000275CD6F8D05C284490F8D80002F8260C63
:10C8600011F8397C11F8B90C0BEB870711F8796CCA
:10C870001844D7F8D0500BEB8606054495F8D850ED
:10C8800002F8245CD7F8D074D6F8D0583D4400EBB9
:10C89000254595F8D85002F8235CD6F8D05C28449A
:10C8A00090F8D80002F8220C7FF4DAAE88E600BFD8
:10C8B000449900904C880090099D47F2204147F22E
:10C8C0008C426C58A858E41A00F094FB47F20C41D3
:10C8D00005F5E942E3000E906958126800290191BC
:10C8E0007FF76EAE03F14005843300F12006DFF8D8
:10C8F0008CB2D7181544A04B05F180023C4629465E
:10C9000002950092324694F83CE0403114F8048CD1
:10C9100020320BEB8E0E11F880CC0BEB8808043420
:10C92000DEF8D004D8F8D058DEF8D0E0D8F8D08CB3
:10C9300028449E4403EB204098440EEB0C0A00EB85
:10C940000C09C4449AF8D8A099F8D8909CF8D8C09B
:10C9500002F83F9C02F840AC02F83ECC11F87FCCC4
:10C960006044E044E6449EF8D8C090F8D8E098F8D7
:10C97000D80002F83CCC02F83BEC02F83A0C94F8F0
:10C9800039E014F8078C0BEB8E0E11F87ECC0BEB14
:10C990008808DEF8D004D8F8D058DEF8D0E0D8F80F
:10C9A000D08C28449E4403EB204098440EEB0C0AA4
:10C9B00000EB0C09C4449AF8D8A099F8D8909CF8D8
:10C9C000D8C002F8379C02F838AC02F836CC11F81F
:10C9D0007DCCE0446044E64490F8D8C09EF8D8E0AE
:10C9E00098F8D80002F833CC02F834EC02F8320C94
:10C9F00094F83AE014F8068C0BEB8E0E11F87CCC10
:10CA00000BEB8808DEF8D004D8F8D058DEF8D0E078
:10CA1000D8F8D08C28449E4403EB204098440EEB79
:10CA20000C0A00EB0C09C4449AF8D8A099F8D890E5
:10CA30009CF8D8C002F82F9C02F830AC02F82ECC3B
:10CA400011F87BCC6044E044E6449EF8D8C090F8EE
:10CA5000D8E098F8D80002F82CCC02F82BEC02F8B9
:10CA60002A0C94F83BE014F805CC0BEB8E0E0BEB84
:10CA70008C0CDEF8D004DCF8D058DEF8D0E0284486
:10CA8000DCF8D08C9E4411F87ACC03EB204098441B
:10CA90000EEB0C0A00EB0C09C4449AF8D8A09CF8E1
:10CAA000D8C099F8D89002F828AC02F8279C02F870
:10CAB00026CC11F879CC6044E644E0449EF8D8C016
:10CAC00090F8D8E098F8D80002F824CC02F8220CAC
:10CAD000009802F823EC81427FF415AF019A4036AA
:10CAE000029D07F58077013A05F5807501927FF484
:10CAF00003AF65E5002DACBF4FF0FF0E4FF0000E09
:10CB0000FFF7C8BA002AACBFFF230023FFF726BBFC
:10CB10000028ACBFFF230023FFF712BB0028ACBFE7
:10CB2000FF200020FFF7FEBA002DACBFFF24002439
:10CB3000FFF7EABA002DACBFFF250025FFF7D6BAF4
:10CB4000002EACBFFF250025FFF7C2BA002DACBFF9
:10CB5000FF260026FFF7AEBA089B07990133403144
:10CB60001A4608930B9B07911B689A42BFF63FAB8E
:10CB70000D991346FFF7FFB8449900904C88009038
:10CB8000099C47F2204147F28C426558A058ED1AA3
:10CB900000F030FA47F290430D900646E05800F05E
:10CBA00029FA072D0E9075DC04F5E943196801EBAD
:10CBB000C5026B1047F20C44099DDB002C59002C78
:10CBC00005947FF7FAAC7F33341D013ADFF808B1E2
:10CBD000CB180394041D029204933E4B049F04F16E
:10CBE0002002029907F14008039E01F1080C8E46CD
:10CBF00001920097009A043418F8011F043612F8C5
:10CC0000015F0BEB81011EF8010F0BEB8505009214
:10CC1000D1F8D024D5F8D078D1F8D010D5F8D05CA0
:10CC20003A44194403EB22421D4401EB000A02EB93
:10CC3000000928449AF8D8A090F8D80099F8D8901C
:10CC400006F808AC06F8079C06F8060C1CF8010F5D
:10CC500002440144054491F8D80092F8D81095F8A0
:10CC6000D82004F8080C04F8062C04F8071C019AD4
:10CC7000A242BFD1039A20320392049A02F5807235
:10CC80000492029A02F580720292059A013A059284
:10CC9000A4D192E4099B05F0070203F5E943196862
:10CCA00001EBC202403284E7099B04F0070A03F556
:10CCB000E9431A6802EBCA0A0AF1800AFFF7C8BA08
:10CCC00047F27C43099AD05800F094F9206007900D
:10CCD000FFF737B8449900904C8800902DE9F04F49
:10CCE000B84B97B0834610221B68002112A89847C2
:10CCF00047F240435BF80320002A40F3F48047F2F8
:10CD000048430021DFF8C8A218460D9102915BF854
:10CD100003300BEB00010A91002B40F3DE8047F259
:10CD2000744247F22D3100230A985A449946984696
:10CD30000C920BEB010205930B92029A0390D20125
:10CD40000192039B47F2B83553F8044F03930BEB62
:10CD500004070C9B2601186800F04CF984460890E3
:10CD600047F22530A30016A9384441F6C242079382
:10CD7000CB1890F800E041F6FE410BEB060053F8AB
:10CD8000103C7244214405444B440BEB82025BF897
:10CD900021402968526804910992049A05999342A6
:10CDA000CDF83CC00C4480F2E08047F2BC3212580F
:10CDB000944280F2DA8047F2C03247F2C4310693DF
:10CDC0000244014412680868049200F013F92968CB
:10CDD000069B049A01FB0431119002FB01050BEB49
:10CDE000060147F2783604930E443268934249DADA
:10CDF00047F27C325258944244DA47F2843001F5CB
:10CE0000E742084412680068069200F0F3F83168BF
:10CE1000049B069A01FB0434109002FB04F40619EB
:10CE200031D085B3015B019A0898674B8418864618
:10CE300001987E221B682EF80010A91CA01C9847A0
:10CE400062493F2202E0013A00F0A78011F8013D5B
:10CE500034F81330002BF6D009995D4801EB4201FC
:10CE6000024433B1B1F800E010781EFB03F324F85C
:10CE700010305245A1F1020105D012F8013D34F8FD
:10CE80001330EEE700260F9B13B10FA801F0C4F991
:10CE900015B111A801F0C0F916B110A801F0BCF944
:10CEA0000B9B029A1B780132012B02925FD047F252
:10CEB0001D3309F101093B441B78994561D00A9B58
:10CEC00008F10108019A1B688032434501923FF73F
:10CED00038AF47F2404252F80B200D990131914290
:10CEE0000D91FFF619AF47F22D331BF80320012AED
:10CEF00070D0002A35D047F22E3047F2F83347F28F
:10CF00002131012A1BF800000BEB80055844EC5836
:10CF1000405C0444EC5024D047F22F30022A1BF826
:10CF200000000BEB80055844EC58405C0444EC5086
:10CF300017D047F23030032A1BF800000BEB8005B6
:10CF40005844EC58405C0444EC500AD047F231326B
:10CF50001BF802200BEB82005A44C458525C224456
:10CF6000C250002017B0BDE8F08F002537E716AAA1
:10CF7000079B13441A4653F8103C013342F8103C07
:10CF80009DE747F22133059A3B4401321B78059215
:10CF90009A4209D04FF0000991E709990C4801EB3A
:10CFA0004201238802445CE716AA079B134453F806
:10CFB000102C4A444FF0000943F8102CCDF814907F
:10CFC0007DE700BFB8030020B40300208C880090E8
:10CFD0004C88009047F22E3347F2F83100201BF8BE
:10CFE00003300BEB83035A5801325A5017B0BDE897
:10CFF000F08F00BF084AD169536B013110B4D16181
:10D0000003EBC00413F83020013203F830206068CD
:10D010005DF8044B0830704760E4032047F2784322
:10D020002DE9F04F804695B0C058FFF7E3FF47F277
:10D030004043129058F80330002B40F31E8347F210
:10D040004044002347F2344247F23841254647F234
:10D050007444089347F24840264604931C4608EB64
:10D060000203DFF8B894C3460D9308EB010309935C
:10D0700008EB00030A9308EB05030E9308EB060385
:10D080000B930D9B1B6823B1099B1B68002B00F0C1
:10D090006D860A9A1368002B40F3E282002C40F060
:10D0A000DF82049B05920C93DB010693059B47F2FC
:10D0B00032351A4652F8043F1C4600930B9B0592EA
:10D0C0001868FFF797FF0BEB040347F2253441F68E
:10D0D000C2421E460193DBF8243035443444C3F386
:10D0E0000721139095F80080069D247800EB050A2F
:10D0F0004FF45075224405FB08110BEB82020BEB39
:10D1000081015268D1F8BC580292002DC0F2DD8234
:10D110004FF45062DBF8287002FB08B808EB0502F8
:10D1200092F8BC6CBF1B002FCBF8287040F3A18392
:10D13000C6F12006F341CBF82430002D40F0A48244
:10D140002946009A47F2643047F23634129D0BEBC1
:10D15000820201261044019A2244144602681144B6
:10D16000029A0160128812FB01F20499AAF80020C9
:10D17000695C227800914FF4507101FB02F84FF482
:10D18000506101FB02B20192C3F3072242440BEB50
:10D190008202D2F8BC48002CC0F22881019A2244B5
:10D1A00092F8BC5C7F1B002FCBF8287040F37B818A
:10D1B000C5F1200263FA02F2CBF82420231114F007
:10D1C0000F0450D0002B00F00B819F193F2F00F36C
:10D1D0004382009AB24240F30481921B9342A8BF5B
:10D1E0001346002B00F0FD80721E0020CB4E9918D4
:10D1F00009EB0203494413F8012F8B422AF812006D
:10D20000F9D1DBF828200123C4F11005DBF8241044
:10D21000121BA34021FA05F0002A03F1FF35CBF8D9
:10D22000282005EA000540F37B81C4F12003D941A1
:10D23000CBF8241006EB8404236DAB4202DDD4F856
:10D2400090301D44029BF25D33F8173013FB05F557
:10D250002AF812507E1C402E00F09F80DBF824300C
:10D26000DBF8287090E70F2B40F09780302E00F30A
:10D27000F381009BB34240F3B6809B1B102BA8BFE9
:10D280001023002B00F0AF8019F80620012B06F1C7
:10D2900001012AF8124000F0A680A04A022B515C3E
:10D2A00006F102022AF8114000F09D809B49032BF1
:10D2B000895C06F103022AF8114000F09480974936
:10D2C000042B895C06F104022AF8114000F08B80DF
:10D2D0009249052B895C06F105022AF8114000F0FD
:10D2E000828019F80200062B4FF0000206F10601B9
:10D2F0002AF8102077D019F80100072B06F1070152
:10D300002AF810206FD019F80100082B06F1080147
:10D310002AF8102067D019F80100092B06F109013D
:10D320002AF810205FD019F801000A2B06F10A0133
:10D330002AF8102057D019F801000B2B06F10B0129
:10D340002AF810204FD019F801000C2B06F10C011F
:10D350002AF8102047D019F801000D2B06F10D0115
:10D360002AF810203FD019F801000E2B06F10E010B
:10D370002AF8102037D019F801100F2B06F10F07EB
:10D380002AF811203FF466AF7E1C19F807300022FE
:10D39000402E2AF813207FF461AF009BB3420ADDD0
:10D3A000591E731E002049444B4413F8012F994223
:10D3B0002AF81200F9D1049913A8129B069A5E5418
:10D3C0004B1C80321C460493069200F025FF0A9BFA
:10D3D0000C991A68631A9A423FF768AE00243FE13D
:10D3E00037464E4E0DE706F10F0733E7083F002F93
:10D3F000CBF8287040F3CE804FEA3362CBF824207C
:10D40000234639460FE04FEAF272CBF824202B1B5B
:10D4100043440BEB8303D3F8BC3D002B3FDADBF82E
:10D420002420DBF8281001395D42C2F3C034002902
:10D43000CBF82810E7DCDBF800200DF14701584657
:10D44000904770BB9DF84770FF2F00F0D880DBF845
:10D4500000300DF147015846984710BB9DF8473002
:10D46000FF2B00F0DD811904DBF82830DBF82420E5
:10D47000C3F11F0E584262FA0EF203F1200E103370
:10D4800092B2CBF8283042EA076747EA010303FA71
:10D4900000F023FA0EF30343CBF82430B7E71C4621
:10D4A0008CE6FF24B3E70DF1470358461946039372
:10D4B000DBF80030984700287FF480AE9DF8477075
:10D4C000DBF80030FF2F00F05F8103995846984742
:10D4D00000287FF473AE9DF84730FF2B079300F0D0
:10D4E000C7821904DBF82800DBF824202B18C0F1D0
:10D4F000000E00F120051030C3F12003CBF8280006
:10D5000062FA03F39BB243EA0763194301FA0EF38D
:10D51000E9400B43CBF8243050E600BF4C88009024
:10D520000DF14703584619460393DBF8003098473E
:10D5300070BB9DF84730FF2B0793DBF8003000F0FD
:10D54000488103995846984710BB9DF84720FF2A09
:10D5500000F011841004DBF82820DBF8243004EB01
:10D56000020E514202F1200C1032CEF1200ECBF807
:10D57000282063FA0EF3079A9BB243EA026303433F
:10D5800003FA01F123FA0CF30B43CBF8243051E6F4
:10D59000FF254FE60DF14703584619460393DBF884
:10D5A00000309847002852D19DF84730FF2B079351
:10D5B000DBF8003000F09281039958469847002824
:10D5C00045D19DF84750FF2D00F026832904DBF854
:10D5D0002830DBF82420C3F11805584203F1100766
:10D5E000EA4103F12005079B92B242EA036211432C
:10D5F00001FA00F2E9400A43CBF8242000E7DBF807
:10D6000000200DF147015846904700287FF449AFAC
:10D610009DF8470000283FF41AAF9BF82120042A08
:10D620003FF415AF531C0BEB0201DBB28BF821303A
:10D63000042B4877C349CBF8001000F09482911C6A
:10D640000BEB0302BF4B8BF82110577701E7DBF898
:10D650002420DBF82870D3E613A8012400F0DCFDB9
:10D66000089A099801320368114608920E9A013B04
:10D67000126803608A423FF704AD12A800F0CCFDA7
:10D68000002015B0BDE8F08F0122C5F110017F1B0D
:10D69000AA4023FA01F1002FCBF8287002F1FF32E3
:10D6A00001EA0202039240F384811146C5F120028F
:10D6B000D341CBF8243009EB85052A6D8A427FF7E8
:10D6C00040ADD5F8905029443BE5DBF82870083F81
:10D6D000002FCBF8287040F337814FEA3363CBF843
:10D6E00024304FF4507202FB08F80DE04FEAF37358
:10D6F0002246CBF82430B21A42440BEB8202D2F815
:10D70000BC5D002DBFF619AD013F6E42C3F3C034BE
:10D71000002FCBF82870E9DCDBF800300DF1470171
:10D720005846984750BB9DF84750FF2D00F079812F
:10D73000DBF800700DF147015846B847F0B99DF885
:10D740004770FF2F00F08E823B04DBF828702246E2
:10D75000DBF82410C7F11F047842E14107F12004EF
:10D76000103789B2CBF8287041EA05652B4303FADC
:10D7700000F0E3400343CBF82430BCE7DBF824306F
:10D78000FF22DBF82870B6E703995846984700282F
:10D790007FF414AD9DF84700002800F0C6809BF888
:10D7A0002120042A00F0C180531C0BEB0201DBB2E4
:10D7B0008BF82130042B48776249CBF8001000F039
:10D7C00024820BEB030102325E4B8BF821204F7752
:10D7D0007BE603995846984700287FF4D9AE9DF818
:10D7E0004700002800F06D819BF82120042A00F0FA
:10D7F0006881531C0BEB0201DBB28BF82130042B48
:10D8000048775049CBF8001000F0EB8202320BEB66
:10D8100003014C4B8BF821209DF81C204A7790E6A1
:10D82000DBF800200DF14701584603939047039B16
:10D8300000287FF436AE9DF847E0BEF1000F7DD0A2
:10D840009BF82110042979D04A1C0BEB0100D2B2BD
:10D850008BF82120042A80F81DE03A48CBF800001C
:10D860006CD0881C5A444FF47F018BF82100537709
:10D87000FAE50DF14704DBF8003058462146984799
:10D88000002855D19DF84780DBF80030B8F1FF0F34
:10D8900000F09981214658469847002848D19DF8C4
:10D8A0004770FF2F00F061813904DBF82870DBF846
:10D8B0002430F219784207F120041037C2F1200217
:10D8C000CBF82870D3419BB243EA08630B4303FAB9
:10D8D00000F0E3400343CBF824302EE4039958468C
:10D8E000984700287FF4B3AE9DF84700002800F069
:10D8F00074829BF82120042A00F06F82531C0BEBEA
:10D900000201DBB28BF82130042B48770D49CBF8AC
:10D91000001000F05F8202320BEB0301094B8BF821
:10D9200021209DF81C204A7746E6DBF80030CCE544
:10D93000DBF82430DBF82870FFF7FFBB4FF47F01E2
:10D9400092E500BFFD9505900DF14704DBF800302E
:10D95000584621469847002840F000819DF84730FE
:10D96000FF2B0393DBF8003000F0D18021465846AE
:10D970009847002840F0F2809DF84760FF2E00F0A5
:10D98000A3803204DBF82870DBF82430C7F11800DC
:10D99000039C7942C34107F1200010379BB243EA50
:10D9A0000463134303FA01F1C3400B43CBF8243063
:10D9B00097E60DF14704DBF80030584621469847BA
:10D9C000002840F09B819DF84780DBF80030B8F1DB
:10D9D000FF0F00F06D81214658469847002840F01F
:10D9E0008D819DF84760FF2E00F08E813004DBF8BA
:10D9F0002870DBF82430EC197A4207F12006103742
:10DA0000C4F120040399CBF82870E3419BB243EAA8
:10DA10000863034303FA02F2F3401343CBF82430C4
:10DA200049E6DBF800300DF14701584698470028D9
:10DA30007FF4A4AE9DF8470000283FF479AE9BF830
:10DA40002120042A3FF474AE531C0BEB0201DBB21D
:10DA50008BF82130042B4877C349CBF8001000F035
:10DA6000B38102325B440F468BF821205D7761E67B
:10DA700003995846DBF80030984700287FF49EABA6
:10DA80009DF84700002800F0AF819BF82120042A70
:10DA900000F0AA81531C0BEB0201DBB28BF82130A2
:10DAA000042B4877B049CBF8001000F09D8102327A
:10DAB0005B444FF47F018BF821209DF81C205A779E
:10DAC00010E5DBF800303CE52146DBF80030584635
:10DAD0009847002842D19DF8470000286DD09BF858
:10DAE0002110042969D04B1C0BEB0102DBB28BF82F
:10DAF0002130042B50779C4ACBF800205DD00231B6
:10DB00005B444FF47F028BF821105E773AE72146A1
:10DB10005846984710BB9DF8470000284AD09BF80C
:10DB20002120042A46D0531C0BEB0201DBB28BF8F8
:10DB30002130042B48778C49CBF8001038D00232C2
:10DB40000BEB03015846884B8BF821209DF80C20E5
:10DB50004A772146984700283FF40EAFDBF824307F
:10DB6000DBF82870BDE5804B73E42146DBF800301C
:10DB70005846984700287FF4DBAE9DF84700F8B17F
:10DB80009BF82120042A1BD0531C0BEB0201DBB2B3
:10DB90008BF82130042B48777349CBF800100FD055
:10DBA00002325B444FF47F018BF821205F777CE6E3
:10DBB0006D4BDBE6DBF80030D8E64FF47F02E1E6A0
:10DBC0004FF47F0171E621465846984700287FF4BC
:10DBD000AFAE9DF84700E0B19BF82120042A18D091
:10DBE000531C0BEB0201DBB28BF82130042B48777E
:10DBF0005D49CBF800100AD00BEB030102325A4BFF
:10DC00008BF8212081F81D8044E6574B5DE4564B8C
:10DC100040E6DBF800303DE603995846DBF800307B
:10DC2000984700287FF413AD9DF84700002800F0C6
:10DC30008D809BF82120042A00F08880531C0BEB78
:10DC40000201DBB28BF82130042B48774649CBF830
:10DC500000107BD002325B444FF47F018BF821200F
:10DC60005D77B4E4DBF800300DF147015846984782
:10DC700000287FF483AD9DF8470000286CD09BF806
:10DC80002120042A68D0531C0BEB0201DBB28BF875
:10DC90002130042B48773449CBF800105CD0911C1C
:10DCA0000BEB03024FF47F038BF8211057774CE501
:10DCB00021465846984708BB9DF84700002850D099
:10DCC0009BF82120042A4CD0531C0BEB0201DBB241
:10DCD0008BF82130042B48772349CBF800103ED035
:10DCE0000BEB03010232204B58468BF8212081F8C0
:10DCF0001D802146984700283FF473AEDBF824309E
:10DD0000FF21DBF82870D6E42146DBF800305846C6
:10DD100098470028F2D19DF84700D0B19BF8212008
:10DD2000042A16D0531C0BEB0201DBB28BF8213016
:10DD3000042B48770C49CBF800100AD002325B4420
:10DD40004FF47F008BF821205E7750E64FF47F017F
:10DD50003DE44FF47F004AE64FF47F03F5E4024BC5
:10DD600039E6DBF8003036E6FD950590584600F0C0
:10DD70006DFAFFF78EB903995846DBF800300F9221
:10DD800098470F9A00287FF403AC9DF847E0BEF156
:10DD9000000F1BD09BF82110042917D04B1C0BEB54
:10DDA0000100DBB28BF82130042B80F81DE0104815
:10DDB000CBF800000AD002315B444FF47F008BF8AF
:10DDC00021105A77FFF7C7BB094FB3E44FF47F0028
:10DDD000FFF7C1BB064BFFF7EFBBDBF80030FFF7E7
:10DDE000EBBB034BFFF7ADBB4FF47F01FFF77ABBF3
:10DDF000FD9505902DE9F04F044683B00D460026B1
:10DE0000236801A92046984718B113E02368984772
:10DE100080B99DF8043001A92046FF2BF6D103E01C
:10DE20009DF80430FF2B09D1236801A920469847AB
:10DE30000028F5D0012003B0BDE8F08F002BDFD023
:10DE4000CC2B2B70F6D04AD9DA2B40F21381DD2B84
:10DE500000F01781EE2B00F0B980DB2B00F043813E
:10DE600023680DF10301204698470028C8D1236894
:10DE700001A9204698470028C2D19DF803809DF84B
:10DE8000043043EA0828A8F10208B8F1000FB7DD12
:10DE9000A26990454FF000031ADD217FC2EB08080C
:10DEA000002940F07481E36867684FF4805201A94B
:10DEB000A068B847002800F06D81E3680246A061C1
:10DEC00090451844019BE06063614FF00003E4DC7F
:10DED0006369C8EB02024344A261636190E7C72B08
:10DEE00000F24F81C52BA6D2C32B40F2BC800DF1AE
:10DEF0000307236820463946984700289AD12368AB
:10DF000001A920469847002894D19DF803909DF8D8
:10DF1000043043EA0929A9F10209B9F1100F7FF78A
:10DF20006FAF236801A920469847002882D19DF849
:10DF30000420C2F3001302F00F0202EB8303072B4D
:10DF40008DF804303FF676AF03EB03124FF001017A
:10DF50002344804602F1300A224483F82C10A24464
:10DF600082F834000AF1050B0AF1150A22683946D5
:10DF70002046904700287FF45DAF9DF803200BF802
:10DF8000012BD3459044F1D1B8F1FF0FA9F111094C
:10DF90003FF750AFC8453FF74DAF9DF8043004EB55
:10DFA0000323BC33B8F1000F00F0218103EB080A12
:10DFB00002E0D34500F01B8103F1010B19462268F2
:10DFC000204690475B460028F3D033E723680DF1E5
:10DFD00003012046984700287FF42CAF236801A94D
:10DFE0002046984700287FF425AF9DF803209DF830
:10DFF000043043EA02230D2B7FF71CAFA2694FF0D8
:10E000000B0890454FF000031ADD217FC2EB080892
:10E01000002940F0C480E36867684FF4805201A98A
:10E02000A068B847002800F0BD80E3680246A06100
:10E0300090451844019BE06063614FF00003E4DC0D
:10E040006769C8EB0202236801A94744A261204620
:10E050006761984700287FF4EDAE9DF80430012BEE
:10E060007FF4E8AECCE6C02BBFF4E5AE012B3FF465
:10E07000E1AEF5E6D82BBFF4DEAECF2B3FF6DAAE3D
:10E08000D9E60DF103072368204639469847002852
:10E090007FF4D0AE236801A92046984700287FF47A
:10E0A000C9AE9DF803209DF8043043EA0223042BF7
:10E0B0007FF4C0AE394623682046984700287FF495
:10E0C000B9AE236801A92046984700287FF4B2AE74
:10E0D00047F234439DF803109DF80420234442EA9C
:10E0E00001221A608CE60DF10307236820463946A9
:10E0F000984700287FF49EAE236801A920469847E0
:10E1000000287FF497AE9DF803A09DF8043043EA01
:10E110000A2AAAF1020ABAF1000F75DD23680DF18F
:10E1200002012046984700287FF484AE9DF8023013
:10E1300003F00F011A0903298DF802103FF67AAE99
:10E1400004EBC11047F2081941F6C24381440B4465
:10E1500009F1040804EB8303C3F804803ABB09F116
:10E16000020809F1820905E09DF8043028F8023F11
:10E17000C84546D0236801A9204698470028F3D017
:10E1800058E6C82B3FF456AE03B0BDE8F08FE6600A
:10E19000267789E6A269002A7FF47BAE30E6E66046
:10E1A000267739E7A269002A7FF42BAF42E6DFF831
:10E1B00064B00BF1400912E0236801A9204698479A
:10E1C00000287FF437AE1BF8012F9DF803109DF84F
:10E1D0000430D94543EA012328F812300ED02368D1
:10E1E00039462046984700287FF424AEE4E7C8EB80
:10E1F0000909B9F1100F3FF794AE01E6AAF1810ABF
:10E2000089E7AAF1410A86E7BAF1000F3FF4F8ADB9
:10E2100010E600BF4B88009003680B4A30B40446F8
:10E2200053F8085C506B10F83530012B03D9D169D5
:10E2300009B10139D1610022013B00F835301046A7
:10E24000226030BC704700BF60E40320F0B5054693
:10E2500083B04FF4FA6405E09DF80730FF2B0DD032
:10E26000013C07D02B680DF1070128462646984748
:10E270000028F1D00124204603B0F0BD2B680DF139
:10E2800007012846984704460028F3D19DF8073037
:10E29000FF2B02D1013EF1D1ECE747F23C46AA59EF
:10E2A000D0329342E6D147F21C32114B47F2643030
:10E2B0002146AA5C10271B68284492009847AB5956
:10E2C00047F2344147F23842013347F2304069584F
:10E2D00003F007032C50A95028463946AB51AF62D2
:10E2E00000F008F83946284600F004F8C3E700BFFC
:10E2F000B80300202DE9F0410123846AC1F1100523
:10E30000466A641A8B4026FA05F582B0013B002C60
:10E310000246846205EA030508DDC1F120012846B2
:10E3200066FA01F1516202B0BDE8F0810C46036863
:10E330000DF107010646984728BB9DF80780336812
:10E34000B8F1FF0F21D00DF1070130469847D0B941
:10E350009DF80770FF2F38D0B16A2846726A63189B
:10E3600001F120054C421031C3F12003B162DA41C2
:10E3700092B242EA086242EA074303FA04F4EB402D
:10E3800023437362CFE7FF20CDE70DF1070130464D
:10E3900098470028F7D19DF80700A0B196F8211002
:10E3A000042910D04A1C7718184BD2B2042A86F8D8
:10E3B000212078773360C6D00231324486F82110AC
:10E3C00082F81D80BFE73368BDE70DF107013368B0
:10E3D000304698470028D6D19DF807000028BBD0CA
:10E3E00096F82120042AB7D0531CB118DFF81CE09E
:10E3F000DBB2042B86F821304877C6F800E0ABD0BA
:10E400000232334486F821205F77A5E7FD95059019
:10E410000101000D04000000ACE40590020A0103B4
:10E4200004000000F8D90590030401030600000071
:10E4300038DD05900709000408000000E888059011
:10E44000060C0102080000000C8905900A0A00036E
:10E450000B000000F43A0590090A01030A000000CD
:10E46000283B05900204010303000000A4E105908D
:10E47000050D010306000000E4830590050D00036F
:10E48000060000000C840590050602030800000049
:10E49000E0C0059007060107080000002CB60590B3
:10E4A0000303000B0400000070DF05900402000865
:10E4B00004000000A8E105900202010B0400000026
:10E4C00034E40590060B0103070000004097059017
:10E4D000070A000308000000F4690590040A01031C
:10E4E00008000000E4BC0590060A010308000000D3
:10E4F000FC9D0590070A0003080000001C6A0590B7
:10E50000070A000308000000446A0590070A000398
:10E51000080000006C6A0590070A0003080000006C
:10E52000946A0590060A0103080000001C9E0590ED
:10E53000070A000308000000BC6A0590070A0003F0
:10E5400008000000E46A05900207010604000000CC
:10E5500038DF0590030800060400000010C3059092
:10E560000707010608000000B4AA05900705010787
:10E5700008000000F8BC059007070106080000002D
:10E58000D0AA0590070A0003080000000C6B059054
:10E59000090A00030A0000005C3B05900A0A000318
:10E5A0000A000000903B0590070A010308000000E4
:10E5B000346B05900A0A00030B000000C43B059071
:10E5C000080A01030A0000005C6B0590060A0103BB
:10E5D000070000003C9E0590050A010306000000AC
:10E5E0005C9E05900A0A00030B000000F83B0590B2
:10E5F000070A010309000000846B0590020A010369
:10E600000400000004DA0590060A00030700000079
:10E610007C9E0590080A010309000000AC6B059080
:10E62000050A0103060000009C9E05900A0A0103EA
:10E630000C0000002C3C0590080A01030A000000B1
:10E64000D46B05900A0A00030B000000603C0590A3
:10E65000070A010308000000FC6B05900A0A010389
:10E660000B000000943C0590070A0103080000001D
:10E67000246C0590070A0003070000004C6C05900D
:10E68000060A000306000000BC9E0590070A01036D
:10E6900009000000746C0590090A000309000000DD
:10E6A000C83C05900C0A00030C000000000E059009
:10E6B000090A000309000000FC3C0590080A000359
:10E6C000080000009C6C0590060A0003060000008C
:10E6D000DC9E0590040D01030600000090B3059038
:10E6E000060B01030700000064970590040D010369
:10E6F00006000000ACB30590060501030800000009
:10E70000E0C405900701000E07000000ACE1059091
:10E71000040301020700000078DF059008070006E7
:10E7200009000000ECAA0590070A01030900000097
:10E73000C46C0590080700060800000008AB0590AF
:10E74000080A000309000000EC6C059008070006A9
:10E750000800000024AB0590040A00030400000038
:10E760000CBD0590080A000609000000146D059014
:10E77000060A010308000000FC9E0590020A01033E
:10E780000300000010DA0590030D000304000000F0
:10E79000C8B30590060A0103070000001C9F0590FE
:10E7A000020A0103030000001CDA05900B070106B2
:10E7B0000D0000008C6705900607010608000000A8
:10E7C000DCBA0590080700060900000040AB059080
:10E7D000070A0106090000003C6D0590080A0006C2
:10E7E00009000000646D05900407010605000000A3
:10E7F000F0C505900707FF06060000005CAB05901A
:10E80000050AFF03040000003C9F0590060701066F
:10E8100008000000F4BA0590070700060700000092
:10E8200078AB05900B0700060B000000B867059059
:10E83000080700060700000094AB0590070A0006D1
:10E84000070000008C6D059005070006060000001B
:10E850000CBB0590050D01030700000034840590F2
:10E86000020D03030700000030C70590050D0003EB
:10E87000070000005C840590060301080800000002
:10E8800008DC05900101000D04000000B0E40590D3
:10E89000020A01060400000028DA059006090104B6
:10E8A0000800000098B10590090AFF030800000065
:10E8B000303D05900908FF0508000000B46D059083
:10E8C000080A000308000000DC6D0590020B030439
:10E8D00007000000B0D90590070D000308000000F4
:10E8E0000C340590050201030700000080DF05904D
:10E8F0000A0A00030A000000643D059004040003B6
:10E900000500000040DD059005050007050000003A
:10E91000F0C40590070400070800000020C305901C
:10E920000402000804000000B0E105900A0A000398
:10E930000A000000983D0590050201040700000050
:10E9400088DF0590030401040500000048DD059000
:10E950000708010608000000FC9A05900406000361
:10E9600005000000D0D705900506FF030500000054
:10E97000F4C00590040302020700000090DF059038
:10E98000060A0106080000005C9F0590070B0003C3
:10E9900009000000845B05900202010904000000E8
:10E9A00038E405900304020C0700000050DD0590D8
:10E9B0000306010305000000DCD7059005040003F1
:10E9C00005000000E8D705900505000705000000D8
:10E9D00000C50590090A01030B000000CC3D05901D
:10E9E000090A01030B000000003E05900C0A000319
:10E9F0000C0000003C0E0590060A0106080000000D
:10EA00007C9F05900A0D00000A000000A000059000
:10EA10000A0D00000A000000E40005900A0C000145
:10EA20000A000000780E05900A0C00010A000000A0
:10EA3000B40E05900B0CFF010A000000BCE7049027
:10EA4000090D00000A000000280105900D0AFF03CF
:10EA50000D000000ACF404900B0D00030B0000004F
:10EA600030DD0490060D010007000000848405904D
:10EA7000060D010007000000AC840590070C0001A2
:10EA800007000000F4480590060C01010700000093
:10EA900030890590050DFF0004000000D484059026
:10EAA000050D000004000000FC840590060CFF0129
:10EAB0000400000054890590050CFF0104000000CB
:10EAC00078890590090A00030A000000343E059089
:10EAD000080C01010A000000244905900A0D0000FD
:10EAE0000B0000006C0105900A0D00000B000000F7
:10EAF000B00105900A0C00010B000000F00E05901B
:10EB00000A0C00010B0000002C0F05900A0C0001FC
:10EB10000B000000680F05900707010608000000C1
:10EB2000B0AB05900A0C00020B000000A40F05908A
:10EB3000070D01000900000040340590070D010099
:10EB40000900000074340590070C01010900000061
:10EB500054490590070C0101090000008449059003
:10EB6000080D000008000000A8340590070A010302
:10EB700008000000046E0590070A01030900000068
:10EB80002C6E0590080B000209000000B05B059098
:10EB9000080B000209000000DC5B0590080A000376
:10EBA00009000000546E0590080A000309000000E7
:10EBB0007C6E0590080A000309000000A46E059011
:10EBC000080B000209000000085C05900E07000613
:10EBD0000E000000EC450590080A00060800000041
:10EBE000CC6E0590080B000208000000345C059014
:10EBF000080B000208000000605C0590080A000392
:10EC000008000000F46E0590080A000308000000E8
:10EC10001C6F0590050BFF0203000000889705900C
:10EC2000040B00020300000014B90590060AFF035C
:10EC3000030000009C9F0590050AFF0303000000ED
:10EC4000BC9F0590080A000309000000446F05906E
:10EC5000060A010308000000DC9F0590080B000273
:10EC6000090000008C5C0590080B00020900000000
:10EC7000B85C0590080A0003090000006C6F05905D
:10EC8000080A000309000000946F0590080A0003B9
:10EC900009000000BC6F059007080106080000008D
:10ECA0001C9B059008090005090000009C8905903F
:10ECB000060B010208000000AC970590060B01024C
:10ECC00008000000D0970590060A01030800000024
:10ECD000FC9F0590060A0103080000001CA0059097
:10ECE000070E000207000000BC240590070D010379
:10ECF00009000000DC340590090DFF030700000047
:10ED0000F4010590020701060300000040DF0590B2
:10ED1000060A0003060000003CA00590040A000358
:10ED20000400000020BD05900E0A00030E00000044
:10ED3000F4F404900E0700060E0000002046059033
:10ED4000070C000107000000B4490590070AFF0303
:10ED500006000000E46F0590080C000108000000A8
:10ED6000E4490590060C000106000000C0890590EA
:10ED7000060A0003060000005CA00590070D0003D2
:10ED8000080000001035059006020103070000008E
:10ED900098DF05900602010307000000A0DF059040
:10EDA0000502010407000000A8DF05900503010328
:10EDB0000700000014DC05900202030307000000B6
:10EDC0003CE40590030402020700000058DD0590B2
:10EDD0000303020D07000000B0DF059005030103E7
:10EDE0000700000020DC0590060301020700000078
:10EDF0002CDC05900A0A00030A000000683E05901A
:10EE0000060A0106080000007CA005900A07FF061C
:10EE1000080000002096059004020008040000008D
:10EE2000B4E105900602010807000000B8DF059074
:10EE30000C0200080D000000F4D705900303010345
:10EE400004000000C0DF059003030103040000007C
:10EE5000C8DF05900303010B04000000D0DF05901C
:10EE6000050302030700000038DC059005030103D9
:10EE70000700000044DC05900503010B07000000BB
:10EE800050DC0590060D0103080000002485059064
:10EE9000060D0103080000004C85059004040307DB
:10EEA0000800000060DD05900B02010B0D00000062
:10EEB00000D805900F0A00031000000010DA04903B
:10EEC000030500070300000034DA0590030500077E
:10EED0000300000040DA0590060AFF03020000006C
:10EEE0009CA00590080AFF03070000000C70059025
:10EEF000070A000307000000347005900C06FF03AA
:10EF00000D000000E48905900A0A00030A000000D1
:10EF10009C3E05900B0A00030C000000E00F0590DA
:10EF2000070A0003080000005C700590090A00034E
:10EF300009000000D03E05900A0B00030A00000003
:10EF40008C290590070C000308000000144A059066
:10EF5000070201090800000068DD0590060AFF03AA
:10EF600002000000BCA0059002020109040000009C
:10EF700040E40590080D00020800000044350590AB
:10EF8000090401070B00000034BD0590050D0002C7
:10EF900005000000748505900704010708000000C3
:10EFA00030C3059007080105080000003C9B059050
:10EFB0000609010408000000B4B105900609010427
:10EFC00008000000D0B10590070B01030800000005
:10EFD000E45C0590060A000307000000DCA0059031
:10EFE000060A000307000000FCA0059007090004C2
:10EFF00007000000088A05900101000C04000000D1
:10F00000B4E40590010A0102040000004CDA059006
:10F01000030401020500000070DD0590070A0002EC
:10F020000700000084700590060C00010700000036
:10F030002C8A05900A0A00020A000000043F05908D
:10F04000080A01020A000000AC70059001040102E8
:10F0500003000000B8E10590040E01020600000064
:10F06000CCAB0590040E000206000000E8AB059052
:10F07000050501020800000010C5059007070005FE
:10F080000800000004AC05900203000A0400000020
:10F09000C4E30590040100080400000044E4059066
:10F0A0000102010A0400000048E40590060B010279
:10F0B00007000000F4970590060A0102070000000F
:10F0C0001CA10590030A01020700000048BD05903D
:10F0D000060A0102070000003CA10590070A000291
:10F0E00007000000D4700590070A00020700000026
:10F0F000FC700590070A00020700000024710590CB
:10F10000070A0002070000004C710590060A010280
:10F11000070000005CA10590060A0102070000003C
:10F120007CA10590070A0002070000007471059099
:10F13000010701050400000048DF059002080005F2
:10F140000400000078DD05900707010508000000B5
:10F1500020AC0590070401070800000040C305909B
:10F1600007070105080000003CAC0590050A0102F4
:10F17000070000009CA105900A0A00020A00000096
:10F18000383F0590090A0002090000006C3F059015
:10F19000060A010207000000BCA105900A0A01024C
:10F1A0000A000000A03F0590080A010209000000C3
:10F1B0009C710590060A010207000000DCA1059081
:10F1C000050A010206000000FCA105900A0A0102DE
:10F1D0000B000000D43F0590070A0102090000005F
:10F1E000C4710590010A01020300000058DA05907D
:10F1F000050A0002060000001CA20590070A010291
:10F2000008000000EC710590050A010206000000EC
:10F210003CA205900A0A01020C000000084005907B
:10F22000080A01020A00000014720590090A01028E
:10F230000B0000003C400590060A01020700000098
:10F240005CA205900B0A01020B0000001C10059047
:10F25000060A0102080000007CA20590050A0102CE
:10F26000070000009CA20590070AFF0206000000AC
:10F270003C720590060A010208000000BCA205903D
:10F28000090A000209000000704005900C0A000203
:10F290000C00000058100590080A00020800000049
:10F2A00064720590070A0002080000008C72059045
:10F2B000070A000206000000B4720590040D020265
:10F2C00006000000E4B30590060B010207000000F1
:10F2D00018980590040D00020600000000B4059087
:10F2E000060501020800000020C505900701000D79
:10F2F00007000000BCE105900403020207000000C3
:10F30000D8DF0590080700050900000058AC0590FB
:10F31000070A010209000000DC72059008070005D9
:10F320000800000074AC0590080A00020900000003
:10F3300004730590080700050800000090AC0590D4
:10F34000040A0002040000005CBD0590080A0005E4
:10F35000090000002C730590060A01020800000055
:10F36000DCA20590010A01020300000064DA0590A6
:10F37000030DFF02030000001CB40590060A010201
:10F3800007000000FCA20590010A01020300000032
:10F3900070DA05900A0701050C00000044960590FC
:10F3A000060701050800000024BB059008070005BA
:10F3B00008000000ACAC0590070A01050900000038
:10F3C00054730590080A0005090000007C7305903D
:10F3D000040701050400000000C6059005070005AC
:10F3E000060000003CBB0590050AFF020400000077
:10F3F0001CA30590060701050800000054BB0590FA
:10F400000707000507000000C8AC05900A070005C3
:10F410000A00000068960590060700050600000037
:10F420006CBB0590070A000507000000A473059057
:10F43000050700050500000084BB0590040D0202CD
:10F440000600000038B40590010D0302070000001B
:10F4500040C70590040D01020600000054B4059059
:10F460000602010808000000E0DF05900101000C21
:10F4700004000000B8E40590010901050400000043
:10F480005CDC0590060801030700000044B6059007
:10F49000070A000207000000CC730590080800046A
:10F4A000070000005C9B0590070A000207000000AF
:10F4B000F4730590010B030307000000BCD905900D
:10F4C000060D0102080000009C850590030202025F
:10F4D00007000000C0E105900A0A00020A000000CF
:10F4E000A440059005040002050000000CD805901A
:10F4F00004050006050000007CDA059007040007FB
:10F500000800000050C3059004010008040000003A
:10F510004CE405900A0A00020A000000D840059059
:10F520000501010307000000C8E30590040301037F
:10F5300005000000E8DF059007080004080000004F
:10F540007C9B0590030601020500000018D8059079
:10F55000040600020500000024D8059004030202FE
:10F5600007000000F0DF0590060A01050800000012
:10F570003CA30590070B000208000000105D0590F9
:10F58000010201070400000050E405900304020B8F
:10F590000700000080DD0590030600020500000062
:10F5A00030D80590040401020500000088DD0590B4
:10F5B000040500060500000088DA05900A0A00022A
:10F5C0000A0000000C4105900A0A00020A0000002F
:10F5D000404105900A0A01020B00000074410590A9
:10F5E000060A0105070000005CA30590090C000055
:10F5F0000900000094100590090C000009000000AB
:10F60000D0100590090C0000090000000C110590B5
:10F61000090C00000900000048110590090C0000C9
:10F620000900000084110590090C00000900000089
:10F63000C01105900C0A00020C000000FC1105909E
:10F640000A0D01020A00000038020590060C0100B4
:10F6500007000000508A0590060C0100070000001A
:10F66000748A0590060C010007000000988A059036
:10F67000050C010007000000BC8A0590040CFF0087
:10F68000030000005CB60590040C000003000000BD
:10F6900074B60590050CFF0003000000E08A059099
:10F6A000030C0000030000008CB60590090A00025C
:10F6B00009000000A8410590080C01000A000000A4
:10F6C000444A0590090C01000B0000003812059017
:10F6D000090C01000B00000074120590090C0100D8
:10F6E0000B000000B0120590090C01000B00000097
:10F6F000EC120590090C01000B0000002813059086
:10F700000707010508000000E4AC0590090C0101A1
:10F710000B00000064130590060C010008000000B7
:10F72000048B0590060C010008000000288B059052
:10F73000060C0100080000004C8B0590060C01002F
:10F7400008000000708B0590070C00000800000006
:10F75000744A0590060A0102070000007CA3059088
:10F76000060A0102080000009CA30590080A000296
:10F77000090000001C740590080A0002090000003E
:10F7800044740590080A0002090000006C7405909A
:10F79000080A00020900000094740590080A00029B
:10F7A00009000000BC740590080A0002090000006E
:10F7B000E47405900E0700050F0000005446059004
:10F7C000080A0005080000000C750590080A0002F0
:10F7D0000800000034750590080A000208000000C7
:10F7E0005C750590080A0002080000008475059009
:10F7F000080A000208000000AC750590040AFF0228
:10F800000300000070BD0590040B00010300000020
:10F810002CB90590060AFE0203000000BCA3059067
:10F82000030A00020300000084BD0590080A0002DC
:10F8300008000000D4750590060A010208000000C7
:10F84000DCA30590080A000208000000FC75059082
:10F85000080A00020800000024760590080A000249
:10F86000080000004C760590080A0002080000001D
:10F8700074760590080A0002080000009C76059046
:10F88000070700050800000000AD05900809000406
:10F8900008000000948B0590060A01020800000091
:10F8A000FCA30590060B0101080000003C980590A0
:10F8B000060A0102080000001CA40590060A0102C5
:10F8C000080000003CA40590070E0001070000009E
:10F8D000F4240590070D0102090000007835059019
:10F8E000070D000207000000AC3505900107010577
:10F8F0000300000050DF0590060A00020600000029
:10F900005CA40590040A00020300000098BD059065
:10F910000D0A01020F0000003CF504900E070005DF
:10F920000F00000088460590050C0100070000004C
:10F93000B88B0590060A0002060000007CA4059022
:10F94000070C000008000000A44A0590070C000006
:10F9500006000000D44A0590060A000205000000D7
:10F960009CA40590070D000207000000E0350590FB
:10F970000602010207000000F8DF059006020102FE
:10F980000700000000E005900501010307000000EA
:10F99000CCE30590050201020700000008E0059095
:10F9A000010203020700000054E405900303020271
:10F9B0000700000010E005900303020C07000000A0
:10F9C00018E00590050301020700000068DC0590BF
:10F9D000050301010700000074DC05900A0A00021B
:10F9E0000A000000DC410590060A0105080000003D
:10F9F000BCA4059008070005080000001CAD059098
:10FA0000040100080400000058E405900601000805
:10FA100007000000D0E305900C0100080D00000075
:10FA200020E005900203010204000000D4E30590E9
:10FA30000203010204000000D8E305900203010A5A
:10FA400004000000DCE3059004030202060000004D
:10FA500028E00590040301020600000030E0059054
:10FA60000403010A0600000038E00590070C0002BC
:10FA700008000000044B0590070C0002080000007D
:10FA8000344B0590030302060600000040E0059099
:10FA90000902020A0D00000094DA05900E0A000225
:10FAA0000F00000084F50490030501060300000028
:10FAB000A0DA05900305010603000000ACDA05900A
:10FAC000050AFE0202000000DCA40590080AFF02FD
:10FAD00007000000C4760590060B00010700000037
:10FAE000609805900B0600020D000000DC8B05906D
:10FAF0000A0A00020A000000104205900B0A0002E8
:10FB00000C000000A0130590060B01010700000087
:10FB100084980590080A000209000000EC76059020
:10FB20000A0B000209000000C4290590070B00021F
:10FB3000070000003C5D0590070101080800000077
:10FB4000C4E10590050AFE0202000000FCA4059035
:10FB500001020107040000005CE40590080E0100AA
:10FB6000080000002C250590090501050B00000088
:10FB700064B50590050E000005000000E4670590DF
:10FB80000705010508000000ACBD05900707010549
:10FB90000800000038AD05900608010408000000C8
:10FBA000A4B6059007080004080000009C9B05907F
:10FBB000070B010208000000685D0590050A0002BD
:10FBC000060000001CA50590050A000206000000C2
:10FBD0003CA505900709000307000000008C059074
:10FBE0000101001907000000BCE4059002140305A0
:10FBF00007000000C0BD0590060802050A000000CD
:10FC0000BCB605900E1100070F0000004899049043
:10FC10000B1702040F0000009C78049012140105D9
:10FC200014000000C01E049012140105130000000F
:10FC3000741F0490020802050600000090DD059084
:10FC4000081B02050B00000018AB0490081B0105FF
:10FC50000B00000084AB04900909030510000000AC
:10FC6000745305900E0D010C100000009CC604900A
:10FC70000405011608000000B8DA0590070200111B
:10FC80000700000098DD059002030316080000003D
:10FC9000E0E305900B1602050E000000DC840490E2
:10FCA0000D1401050F0000007C6B04900614030581
:10FCB0000F000000DC1305900D1401050F0000007B
:10FCC000086C04900D1400050F000000946C049063
:10FCD0000E1400050F000000206D04900E140005A6
:10FCE0000F000000AC6D04900D1401050F00000022
:10FCF000386E04900B1402050F000000F88E04907B
:10FD00000D1401050F000000C46E04900D140105D0
:10FD10000F000000506F0490020E030B080000005B
:10FD200010C605900410010B08000000BC9B059054
:10FD30000D0E010B100000009CBB04900D07010F7D
:10FD400010000000BC4605900D0E010B10000000D5
:10FD500000BC04900C1401050E000000708F04908C
:10FD6000121401051400000028200490121400054C
:10FD700012000000DC2004900C1402050F000000AB
:10FD8000E88F0490131401051500000060FD039036
:10FD90000F14020513000000EC4304900B1402053D
:10FDA0000E000000609004900A1402050D0000008F
:10FDB0005CB504901514010516000000CCE7039013
:10FDC0000D14020511000000DC6F049002140205FE
:10FDD00006000000D4BD05900B1400050D000000C6
:10FDE000D89004900D1402050F0000006870049074
:10FDF0000A1402050C000000C0B50490141402059A
:10FE00001800000028FE03900F14020513000000E4
:10FE10008C4404901414010516000000F0FE0390B9
:10FE20000C1402050E0000005091049016140105F8
:10FE300017000000A8E803900D1402050F00000051
:10FE4000F47004900C1401050E000000C891049099
:10FE50000C1400050C000000409204900C140205E4
:10FE600011000000B8920490121400051200000066
:10FE70009021049017140005180000005CD3039033
:10FE800010140005100000002C450490101400050B
:10FE90000F000000CC4504900D1400050D0000007B
:10FEA00080710490071903050B00000024B604902C
:10FEB0000B1602050E00000060850490071901056D
:10FEC0000B00000088B604900B0A02051000000029
:10FED000181405900D02001A0D00000020C60590B0
:10FEE000070503050E000000E8BD05900F0E010B8D
:10FEF0001200000074A104900F140205120000000B
:10FF00006C4604900F0E010B10000000E4A1049059
:10FF10000F140105120000000C4704900E0E010B97
:10FF20001000000064BC04900714000507000000E6
:10FF300060DA04900F14010B12000000AC4704902B
:10FF40000D140205110000000C7204900214020549
:10FF500006000000FCBD05900519FF050700000024
:10FF60005CE504900B1402050D0000003093049032
:10FF7000021402050600000010BE0590150E020BCB
:10FF8000190000004C5204900D0E020B11000000ED
:10FF9000C8BC04900F0E010B1100000054A2049085
:10FFA0000F13020B12000000205404900F13010BDA
:10FFB00012000000B8540490070E020B0800000065
:10FFC000642505900A0E000B0C000000CCF504908F
:10FFD0000814000508000000B0DA04900D0E020BB2
:10FFE000110000002CBD04900D0E000B0D00000050
:10FFF00090BD0490140E000B140000009872049041
:02000004900169
:100000000C0E000B0D0000003CD104900D13000BF2
:100010000D0000004C7B04900B0E000B0B00000049
:1000200090D10490081B02050C000000F0AB049076
:10003000021A06050E00000070B40590081B0205A8
:100040000C0000005CAC04900C05021010000000D5
:100050005CA505900101001907000000C0E40590AF
:100060000214030B0700000024BE05900C110207C8
:100070000F0000008CB404900F1400050F00000066
:100080004C4804900E0E00090F000000F4BD0490CF
:100090000E1400050F0000002473049002160608D9
:1000A0000E00000044B905900D1A01051000000073
:1000B000981C0490070404050E00000060C305901E
:1000C0001414000515000000B8FF0390080A01058C
:1000D0000B00000014770590080A010D0A000000CB
:1000E0003C7705900D07010F10000000F0460590C9
:1000F0000702001107000000A0DD059014140005A0
:1001000015000000800004900A0203060E000000A3
:10011000C4DA0590080801070A000000DC9B05907E
:100120000E0F010B10000000B4AE0490080D010585
:100130000A00000014360590080D01050A000000B1
:1001400048360590070504050E00000038BE0590EE
:100150000B13020B0F000000EC9C04900E1700051F
:100160001000000000420490020303110800000088
:10017000E4E30590050604180E00000008C1059090
:10018000050C01050A000000248C0590090A0105F0
:100190000B00000044420590080A010D0A0000000F
:1001A00064770590141400051400000048010490C1
:1001B0001414000515000000100204901514010528
:1001C0001700000084E903900B13020B0E000000DF
:1001D000609D0490121900001200000074E2039068
:1001E000121900001200000058E3039012180001D9
:1001F00012000000F4EC039012180001120000003D
:10020000CCED039013180001120000004CD40390B1
:10021000131900001200000088C703901814FF058E
:10022000190000003CD503901319010515000000CA
:1002300084C803900B1902000E000000685F049050
:100240000B1902000E000000006004900B18020160
:100250000E000000DC6504900B1802010E00000087
:100260006C6604900819FE0006000000ECB60490CD
:10027000081900000600000050B704900B18FE019A
:1002800006000000FC66049006180001060000004D
:1002900004E80490111400051300000044220490A7
:1002A0000F18020113000000CC090490141901007A
:1002B0001600000080C90390141901001600000008
:1002C0007CCA039014180101160000002CD603907C
:1002D00014180101160000001CD703901418010126
:1002E000160000000CD803900D0D010C100000004A
:1002F000F8C60490141601041600000060EA03908A
:100300000C19020011000000986004900C19020002
:1003100011000000306104900C180201110000006F
:100320008C6704900C180201110000001C680490F6
:10033000101900000F000000D80204900C140205F0
:100340000E000000A89304900D1402051000000098
:10035000B07304900F14010512000000EC480490E3
:100360000F140105120000008C4904900F140105C0
:10037000120000002C4A04900F1301061200000026
:10038000505504900F14010512000000CC4A04904F
:100390000F140105120000006C4B04901C0E010BA1
:1003A0001D000000F80504900E13010B1000000062
:1003B000D47B04900E140105100000003C740490DE
:1003C0000E14010510000000C87404900E140105FD
:1003D00010000000547504900E1401051000000078
:1003E000E07504900815FE0406000000E4D10490B6
:1003F000081500040600000038D204900C14FD0516
:1004000006000000209404900714FF050600000079
:1004100000DB04900F140105110000000C4C049047
:100420000D130206110000005C7C04900F140105FE
:1004300011000000AC4C04900F14010511000000E5
:100440004C4D04900F14010511000000EC4D049078
:100450000F13010611000000E85504900F14010568
:10046000110000008C4E04900E0F010B10000000D4
:1004700020AF04900F10010A11000000FC880490C6
:100480000D150204110000008C6304900D15020488
:1004900011000000206404900D14020511000000FA
:1004A0006C7604900D14020511000000F87604909B
:1004B0000D1A00040D000000501D04900F190205D4
:1004C00012000000A00304900E1900050D000000AA
:1004D000E0270490020E020B0600000030C60590D3
:1004E0000C1400050C0000009894049007140005FB
:1004F0000700000050DB04901C1401051E000000E2
:1005000084B503901B0E010B1D000000BC06049077
:100510000C1801010E000000AC6804900B140005DB
:100520000C00000010950490101800010F0000004E
:100530008C0A04900D1800010D000000C83A0490C8
:100540000B1400050B000000889504900E1900059F
:100550000F000000902804900B0402050E0000001C
:10056000D4B605900B0402050E000000ECB6059011
:100570000A0203060E000000D0DA05900B04020503
:100580000E00000004B70590020406050E000000EE
:10059000C8E10590060604050E0000001CC1059088
:1005A000050605180E00000030C105900A0302067A
:1005B0000E00000030C505900B0603030E0000007E
:1005C000488C05901214010513000000F8220490D5
:1005D0000B13020B0F000000D49D04900F0E000BB4
:1005E0000F000000C4A204900702001107000000E1
:1005F000A8DD05900B0201110D0000003CD805900C
:10060000180201111A0000001CB70590040502052C
:1006100008000000DCDA0590040501050800000070
:10062000E8DA05900405011608000000F4DA0590E8
:10063000070503050B0000004CBE059007050205E9
:100640000B00000060BE0590070502160B000000BD
:1006500074BE05900C180205100000003C6904905F
:100660000C19020510000000C86104900606030C76
:100670000D00000044C10590140303161A00000089
:100680007CA505901C1401051E0000009CB603907B
:10069000050A010D060000009CA50590050A010D44
:1006A00006000000BCA505900A14FD05030000002B
:1006B000B4B704900F14FF050E0000002C4F0490F7
:1006C0000B1501040D0000007C8A0490160D000536
:1006D0001A000000EC6A04901214010513000000D7
:1006E000AC23049016140105180000003CEB0390A5
:1006F0000C1601030F000000E4850490101301069E
:10070000110000008056049011160106130000002D
:10071000680404900D1601060F000000E8520490D2
:100720000D0201121000000040C605900A14FD05DC
:100730000300000018B80490020303110800000031
:10074000E8E305900F1B01020F000000A4EE0390E8
:100750001208010D150000004CE80490091C00026D
:100760000A000000847704900D08010D0F000000BE
:100770009C2505900D0E020B0F00000058BE049042
:100780000E1001090F00000034A304900D100009A1
:100790000F000000A4A304900D1502050F00000037
:1007A000B46404900A1400050C0000007CB80490A6
:1007B0000A1400050C000000E0B804900D120007B8
:1007C0000D000000FC8A04900101000D04000000EF
:1007D000C4E40590020900040200000080DC0590DA
:1007E0000404000405000000B0DD059007090104C1
:1007F000070000006C8C0590070C00030700000048
:10080000644B05900A0900040A000000A4530590F7
:100810000909000409000000D453059002040004F3
:1008200002000000CCE10590040B0004040000006D
:100830005CB90590040B00040400000074B9059035
:10084000040300040400000048E0059007070105C8
:100850000800000054AD05900204010B04000000E4
:10086000D0E105900402000904000000D4E10590E5
:100870000202010B0400000060E40590070B000475
:1008800007000000945D05900709000407000000C0
:10089000908C0590040902040700000058C10590DF
:1008A0000709000407000000B48C05900709000444
:1008B00007000000D88C059008090004070000001C
:1008C000FC8C05900709000407000000208D0590AE
:1008D0000709000407000000448D05900609000484
:1008E00007000000ECB105900709000407000000B4
:1008F000688D059007090004070000008C8D0590A5
:10090000020601070400000050E0059002080107FC
:1009100004000000B8DD059007080104080000008D
:10092000FC9B0590070401070800000070C30590B8
:1009300007080104080000001C9C0590060900043B
:100940000600000008B20590090901040B00000030
:10095000045405900A09000409000000345405906D
:100960000709000407000000B08D05900A09000483
:100970000900000064540590090900040900000002
:10098000945405900709000407000000D48D0590D9
:100990000709000407000000F88D0590090900040C
:1009A00009000000C4540590090900040900000072
:1009B000F454059004090004040000006CC1059083
:1009C00007090004060000001C8E059009090004B8
:1009D00009000000245505900709000407000000E5
:1009E000408E05900C0900040C0000004C3205906C
:1009F0000A0900040A000000545505900A09000481
:100A00000900000084550590070900040700000054
:100A1000648E05900B0900040A00000084320590E2
:100A20000909000408000000B455059006090004F7
:100A30000600000024B2059006090004070000002B
:100A400040B205900909000408000000E455059033
:100A50000909000409000000145605900D0900045E
:100A60000C000000800D0590090900040900000039
:100A7000445605900809000408000000888E05907F
:100A80000809FF0407000000AC8E0590040B000469
:100A9000050000008CB9059005090104070000005D
:100AA0005CB20590040B000405000000A4B9059099
:100AB000080701040800000070AD05900701000E52
:100AC00006000000D8E105900404010206000000C1
:100AD000C0DD059008070006080000008CAD0590F9
:100AE0000809000408000000D08E059007070006E2
:100AF00007000000A8AD05900809000408000000E8
:100B0000F48E05900707000607000000C4AD0590AD
:100B1000040900040400000080C1059008090006D3
:100B200008000000188F0590080900040800000064
:100B30003C8F0590040900040400000094C1059056
:100B4000030B000403000000BCB905900709000472
:100B500007000000608F05900409000404000000F5
:100B6000A8C105900C0700060C0000001068059055
:100B70000807000608000000E0AD05900707000622
:100B800007000000FCAD0590080900060800000001
:100B9000848F05900809000608000000A88F0590C2
:100BA00005070006050000009CBB0590060700062F
:100BB00006000000B4BB0590040900040400000016
:100BC000BCC10590080700060800000018AE05909B
:100BD000070700060700000034AE05900B0700066B
:100BE0000B0000003C6805900707000607000000A6
:100BF00050AE05900709000607000000CC8F059055
:100C00000507000606000000CCBB0590040B00049D
:100C100004000000D4B90590020D03030800000091
:100C200050C70590040B000404000000ECB90590C7
:100C3000070301070800000048D805900101000DD6
:100C400004000000C8E4059002090006020000004C
:100C50008CDC0590060901040700000078B20590BD
:100C60000809FF0407000000F08F05900508010542
:100C70000700000034B705900809000407000000D1
:100C800014900590020B030408000000C8D90590D9
:100C9000050B000406000000A8980590040201045A
:100CA00006000000DCE105900A0900040A000000CB
:100CB00074560590050400040500000054D8059002
:100CC000040500070400000000DB0590080400078D
:100CD0000800000080C30590040200090400000021
:100CE000E0E105900A0900040A000000A4560590FE
:100CF000050201040600000058E005900304010409
:100D000005000000C8DD0590070701050800000088
:100D10006CAE059004050004040000000CDB059097
:100D2000040600040400000060D8059004030103D9
:100D30000600000060E005900809000608000000B9
:100D400038900590070B000406000000C05D059078
:100D5000020201080400000064E405900303010D91
:100D60000400000068E00590030601040400000090
:100D70006CD805900404000404000000D0DD059048
:100D8000040500070400000018DB059009090104B0
:100D90000A000000D4560590090901040A00000069
:100DA000045705900B0900040A000000BC320590AE
:100DB000060900060600000094B205900A0D000026
:100DC000090000007C0205900A0D000009000000E7
:100DD000C00205900A0C000109000000541405909F
:100DE0000A0C000109000000901405900A0B000293
:100DF00009000000FC2905900A0D00000900000010
:100E0000040305900C0900040C000000F432059066
:100E10000A0C000409000000CC140590070D000026
:100E2000070000007C360590070D00000700000059
:100E3000B0360590070C000107000000944B0590A8
:100E4000080CFF0207000000C44B0590040D0000D1
:100E5000040000008CB40590040D000004000000A4
:100E6000A8B40590060CFF01040000005C900590FA
:100E7000040B00020400000004BA059009090004F4
:100E800009000000345705900A0C00010A00000018
:100E9000081505900A0D00000900000048030590A0
:100EA0000A0D0000090000008C0305900A0C0001E7
:100EB00009000000441505900A0C0001090000001B
:100EC000801505900A0B000209000000342A0590E5
:100ED0000606010608000000D0C105900A0B0003B9
:100EE000090000006C2A0590090D000008000000B0
:100EF000D0030590090D00000800000014040590BF
:100F0000090C000108000000BC150590090B000247
:100F100008000000A42A0590080D00000800000049
:100F2000E436059007090004070000008090059052
:100F30000709000407000000A4900590080B0002B8
:100F400008000000EC5D0590080B0002080000009E
:100F5000185E0590080A0003080000008C770590D1
:100F6000080A000308000000B4770590080900048F
:100F700008000000C8900590080A0003080000005F
:100F8000DC7705900D0700060C0000002447059053
:100F9000070A00060700000004780590070B00020E
:100FA00007000000445E0590070B000207000000E8
:100FB000705E0590070A0003070000002C7805907A
:100FC0000909FF040700000064570590050BFF02A4
:100FD00004000000CC980590050BFF0204000000FF
:100FE000F0980590060AFF0304000000DCA50590B8
:100FF0000409000404000000E4C10590070900048E
:1010000007000000EC900590080A000308000000AB
:1010100054780590070B0002070000009C5E0590C5
:10102000070B000207000000C85E0590070A0003D6
:10103000070000007C780590070A00030700000005
:10104000A47805900709000407000000109105909E
:1010500007060105080000004CB7059007090005C8
:101060000700000034910590080B00020800000002
:10107000F45E0590080B000208000000205F059058
:10108000080A000308000000CC7805900809000455
:101090000800000058910590070D000207000000AD
:1010A00018370590080B0004080000004C5F0590FD
:1010B000080B000407000000785F05900407000695
:1010C0000400000050C60590070900040700000056
:1010D0007C9105900509FF0404000000B0B2059062
:1010E0000D0900040D000000C00D05900D0700065D
:1010F0000C00000058470590060C00010600000097
:10110000A0910590070AFF0306000000F4780590FF
:10111000090B000208000000DC2A0590080CFF0102
:1011200007000000F44B0590050A000306000000CC
:10113000FCA50590060B010407000000149905901A
:10114000060201030700000070E00590060301039A
:101150000700000098DC059005020104060000006D
:1011600078E005900503010306000000A4DC05906B
:10117000020201040300000068E405900303010378
:101180000500000080E005900203010C040000004F
:10119000ECE305900503010306000000B0DC0590B8
:1011A0000503010306000000BCDC05900A09FF04EA
:1011B0000900000094570590080900060800000087
:1011C000C49105900907FF06070000008C96059062
:1011D0000402000904000000E4E105900702000990
:1011E00006000000D8DD05900D0200090C0000008B
:1011F00060C605900204000402000000E8E10590CA
:101200000204000402000000ECE105900204000B5F
:1012100002000000F0E10590040400040500000055
:10122000E0DD05900404000405000000E8DD059001
:101230000404000B05000000F0DD0590070B01041D
:1012400007000000A45F0590070B010407000000E1
:10125000D05F0590040502050700000024DB05901F
:101260000A02010B0C00000030DB05900F0900049E
:101270000F00000094E8049002050007020000003F
:1012800050E10590020500070200000058E10590BA
:101290000609FE0401000000CCB205900809000414
:1012A00007000000E8910590060A00030600000010
:1012B0001CA605900B0500040C0000003CA6059040
:1012C0000A09FF0409000000C45705900B09000437
:1012D0000B0000002C330590070A000307000000F4
:1012E0001C79059008090004080000000C92059084
:1012F0000B0BFF040900000040FA0490070A0004E9
:10130000070000004479059007020108080000006A
:10131000F8DD05900609FE0401000000E8B2059022
:1013200002020108040000006CE40590080D0102AF
:10133000070000004C370590080501070A0000006F
:1013400088BE0590050D000205000000C4850590CB
:10135000060501070700000040C5059006070106C5
:1013600007000000E4BB0590060801050700000027
:1013700064B7059006080005070000007CB70590DB
:10138000070A0104070000006C79059007090004B2
:1013900006000000309205900709000406000000D6
:1013A00054920590060900040600000004B305905D
:1013B0000101000D04000000CCE40590010A0003C7
:1013C000020000003CDB0590020301030400000062
:1013D000F0E30590070A00030800000094790590E7
:1013E000060D010208000000EC8505900A0A0003C2
:1013F0000A00000078420590090A00030900000075
:10140000AC4205900103010302000000F4E30590E3
:10141000040B0103040000001CBA0590040B000338
:101420000400000034BA0590040400030400000026
:1014300000DE0590070701050900000088AE059051
:101440000203010B04000000F8E305900401000909
:101450000400000070E405900102020B040000008B
:1014600074E40590070D0103080000008037059023
:10147000060A0103080000005CA60590050A0203A5
:10148000080000007CA60590060A01030800000081
:101490009CA60590060A010308000000BCA6059062
:1014A000080A000308000000BC790590070A000341
:1014B00008000000E4790590070A00030800000016
:1014C0000C7A0590060A010308000000DCA60590CE
:1014D000060A010308000000FCA60590070A0003A5
:1014E00008000000347A059001060207040000009D
:1014F00088E00590020701070400000058DF05900E
:1015000007080104090000003C9C0590070301073F
:101510000900000078D805900708010409000000C0
:101520005C9C0590060A0003070000001CA70590BC
:101530000A0A01030C000000E04205900A0A0003B9
:101540000B00000014430590060A01030800000088
:101550003CA705900A0A00030A00000048430590D2
:10156000080A0103090000005C7A0590060A0103DD
:10157000070000005CA70590060A010307000000B1
:101580007CA705900A0A00030A0000007C4305902E
:10159000080A010309000000847A0590030A010388
:1015A000040000009CBE0590060A0003070000002E
:1015B0009CA70590080A010309000000AC7A059079
:1015C000050A010307000000BCA705900C0A0003F0
:1015D0000D000000F8150590090A01030A0000003B
:1015E000B04305900A0A00030A000000E443059096
:1015F000060A010308000000DCA705900B0A00039F
:101600000B00000034160590080A010308000000D2
:10161000D47A0590060A000307000000FCA7059095
:10162000070A000307000000FC7A0590080A01037E
:1016300009000000247B05900A0A00030A0000004C
:10164000184405900D0A00030E00000014F60490E3
:10165000090A00030A0000004C440590090A00032F
:101660000900000080440590070A000307000000FD
:101670004C7B0590030C01030400000094B7059017
:10168000050A0103080000001CA80590030C0003D4
:1016900004000000ACB70590080701030900000032
:1016A000A4AE05900701000E07000000F4E10590CC
:1016B000040301020500000090E005900807000601
:1016C00009000000C0AE0590090A000309000000EF
:1016D000B44405900807000607000000DCAE059042
:1016E000080A000309000000747B05900707000644
:1016F00008000000F8AE0590040A00030400000092
:10170000B0BE0590080A0006090000009C7B059009
:10171000080A000308000000C47B0590030A0003C8
:1017200003000000C4BE0590030DFF03030000008A
:10173000C4B40590070A000308000000EC7B059084
:10174000040AFF0304000000D8BE05900D07000640
:101750000D0000008C4705900807000609000000F6
:1017600014AF0590070700060800000030AF059091
:10177000090A000609000000E8440590080A00066E
:1017800009000000147C0590040700060500000015
:1017900070C605900507000605000000FCBB05901B
:1017A000050AFF03040000003CA805900807000696
:1017B000080000004CAF0590080700060800000074
:1017C00068AF05900C0700060C00000068680590E3
:1017D000070700060800000084AF0590080A00060D
:1017E000080000003C7C05900607FF06050000008D
:1017F00014BC0590030B0003040000004CBA0590D4
:10180000010D04030900000060C70590030B0003ED
:101810000400000064BA05900702010709000000F7
:1018200008DE05900101000D04000000D0E40590E1
:10183000010A00060200000048DB059006090103CA
:101840000800000020B30590080A0003080000000B
:10185000647C059006070105080000002CBC05907B
:10186000080A0003080000008C7C0590010B0404AA
:1018700009000000D4D90590050C00030600000003
:10188000789205900302010304000000F8E105903E
:10189000090A01030B0000001C4505900605000322
:1018A0000500000050C50590040500070400000075
:1018B00054DB05900904FF0709000000ECBE059009
:1018C000040100090400000078E40590090A0103FE
:1018D0000B000000504505900501010306000000C3
:1018E000FCE30590040501030500000060DB0590A2
:1018F0000707010509000000A0AF059004070003D9
:101900000500000080C605900407000305000000E4
:1019100090C60590040301030500000098E00590BF
:10192000080A000608000000B47C0590060B0103BD
:101930000700000038990590010202080400000029
:101940007CE405900303010D04000000A0E0059075
:101950000407000305000000A0C60590050500036C
:101960000400000060C505900405000704000000A5
:101970006CDB05900B0A00030B000000701605904D
:101980000B0A00030B000000AC1605900B0A0003C5
:101990000B000000E8160590050A0106070000008C
:1019A0005CA805900A0D00000B000000580405908B
:1019B0000A0D00000B0000009C0405900A0C0001B9
:1019C0000B000000241705900A0D00000B0000001A
:1019D000E00405900A0C00010B0000006017059060
:1019E0000A0D00000B000000240505900D0A0003FD
:1019F0000D0000005CF604900A0D00030A000000D0
:101A000068050590060D010007000000148605908A
:101A1000060D0100070000003C860590060C010140
:101A2000070000009C920590060C010107000000D1
:101A3000C0920590040D000004000000E0B4059081
:101A4000040D000004000000FCB40590050C00012A
:101A500004000000E4920590030C01010400000062
:101A6000C4B70590080A010309000000DC7C05905A
:101A7000090D01000A000000AC0505900A0D0000E8
:101A80000A000000F00505900A0D00000A000000A1
:101A9000340605900A0C00010A0000009C1705900E
:101AA0000A0D00000A000000780605900A0C0001EB
:101AB0000A000000D817059006060105090000007D
:101AC000F8C105900A0C00020A00000014180590E5
:101AD000080D010009000000B4370590080D010051
:101AE00009000000E8370590080C0101090000001A
:101AF000244C0590080C010109000000544C05908D
:101B0000090D000009000000BC060590060A01034B
:101B1000080000007CA80590070A000308000000E8
:101B2000047D0590080B000209000000FC5F059091
:101B3000080B00020900000028600590080A000355
:101B4000090000002C7D0590080A00030900000030
:101B5000547D0590080A0003090000007C7D059073
:101B6000080A000309000000A47D05900E07000686
:101B70000E000000C0470590080A0006070000009C
:101B8000CC7D0590070B0002080000005460059012
:101B9000070B00020800000080600590070A0003A0
:101BA00008000000F47D0590070A0003080000000B
:101BB0001C7E0590040BFF02030000007CBA059018
:101BC000040BFF020300000094BA0590050AFF030E
:101BD000030000009CA80590030A00030300000016
:101BE00000BF0590070A000308000000447E05902E
:101BF000080A0003090000006C7E0590070B000234
